:100000000C94B14B0C94E24B0C94E24B0C94E24BED
:100010000C94E24B0C94A6840C94E24B0C94E24BAF
:100020000C9427840C94E24B0C94E24B0C94C2E5A4
:100030000C94E24B0D940DD70C94E24B0C94E24BD4
:100040000C94E24B0D94A8390C94E24B0C94E24BC7
:100050000C94E24B0C94E24B0D9410500D9434CF61
:100060000C94E24B0C941D5C0C94E24B0C94E24B10
:100070000C94E24B0C94E24B0C94E24B0C94E24B4C
:100080000C94E24B0C94E24B0C94E24B0C94E24B3C
:100090000C94E24B0C94E24B0C94E24B0C94E24B2C
:1000A0000C94E24B0C94E24B0C94E24B0C94E24B1C
:1000B0000C94E24B0C94E24B0C94E24B0C94E24B0C
:1000C0000C94E24B0C94E24B0C94E24B0C945D5C70
:1000D0000C94E24B0C94E24B0C94E24B0C94E24BEC
:1000E0000C94E24B205B245B295B315B465B5F5BDE
:1000F000845BAE5B4901BB01D901E501E701510118
:10010000ED0139010302970159018301D701B701BC
:100110005501C5016901DF01F7017701BF013B010D
:10012000B901C701430147010702F901E901B30120
:10013000DB014D01DD01D301AD017F0181019101A1
:100140005D015D015D010102010201026B0193018C
:100150000102E101E30173016F010902FB01750175
:100160008B01F301B1016301FF01C301CD014F0117
:100170007501EB01D101A301D5015B010F02F10172
:100180009F01BD01CB01A9014B01650179018901E5
:1001900011026101BD016D0185018701084AD73B4C
:1001A0003BCE016E84BCBFFDC12F3D6C74319ABD46
:1001B00056833DDA3D00C77F11BED9E4BB4C3E916A
:1001C0006BAAAABE000000803F05A84CCDB2D44E59
:1001D000B93836A9020C50B9918688083CA6AAAA5B
:1001E0002ABE000000803F07634236B79BD8A71A9B
:1001F00039685618AEBAAB558C1D3CB7CC5763BDA9
:100200006DEDFD753EF6177231BF000000803F08AE
:10021000000000BE922449123EABAAAA2ABECDCC51
:10022000CC4C3E00000080BEABAAAAAA3E00000053
:1002300000BF000000803F0000000000084178D3AC
:10024000BB4387D1133D190E3CC3BD4282AD2B3E4B
:1002500068EC8276BED98FE1A93E4C80EFFFBE01EB
:10026000C4FF7F3F0000000000000D94A7620D94C2
:1002700088800D9413510D9499870D9408780D94EE
:10028000615D0D942D8E0D94C99D0D94FFD10D943B
:10029000E19D0D9495500D943FD10D941A9F0D94AE
:1002A000E4D00D94F5500D9484600D9471510D942B
:1002B00097BF0D941B510D9431D10D94C69F0D9491
:1002C00026AC0D9455D10D94B7D00D9443D10D9417
:1002D000F58A0D941A870D94CE9F0D945BD10D94E1
:1002E0007FD00D948F830D947AD00D940CD10D9402
:1002F00085870D9447D10D94656F0D94DF5E0D9445
:100300008D9F0D94B69F0D9429510D945FD10D943E
:1003100063D10D944DD10D949DD00D946FBC0D946F
:10032000FDB20D94BE9F0D94FC9F0D9487860D9495
:1003300019510D9498830D9454840D94C1720D94A9
:100340002AD10D944A730D9402D10D9496C40D9444
:1003500020640D9439D10D9446670D946A9F0D94D5
:100360004E760D94ADD00D94359E0D9415B40D942C
:1003700051510D94B3870D94A3500D9468D10D94F1
:100380008F870D9480850D94CBD00D9400870D94AC
:10039000CD870D94C8930D9435D10D94DAD00D947A
:1003A0008A3C0D94F8D00D944D9F0D942ED10D9450
:1003B00043510D94BF500D94529E0D943C9F0D944B
:1003C00037870D94D89F0D9475D00D94CD500D9412
:1003D000E7500D94219E0D94EED00D940F510D9485
:1003E000AA830D9424D10D94A5D00D949D160D943F
:1003F00056870D940D9E0D9493D00D9423820D94E9
:10040000C1D00D94EC9F0D9415510D94A1830D94C2
:10041000F89D0D9489D00D941C610D9422610D946A
:1004200020D10D9451D10D940D610D94CEB748613A
:100430007264636F6465642044656661756C7420E2
:1004400053657474696E6773204C6F6164656400F2
:1004500053746F7265642073657474696E6773207A
:1004600072657472696576656400202020452F44AA
:10047000203D20002020204D393030204B004C6999
:100480006E65617220616476616E63652073657468
:1004900074696E67733A0046696C616D656E7420AD
:1004A00073657474696E67733A2044697361626C32
:1004B0006564002020204D32303020440046696CB5
:1004C000616D656E742073657474696E67733A004C
:1004D0002020204D3230392053004175746F2D5249
:1004E0006574726163743A20533D3020746F2064E8
:1004F000697361626C652C203120746F20696E74A1
:1005000065727072657420657874727564652D6F9C
:100510006E6C79206D6F76657320617320726574DF
:100520007261637473206F72207265636F76657297
:10053000696573002046002020204D32303820535A
:10054000005265636F7665723A20533D4578747248
:1005500061206C656E67746820286D6D2920463AAD
:10056000537065656420286D6D2F6D2900205A0039
:100570002046002020204D32303720530052657431
:10058000726163743A20533D4C656E67746820282D
:100590006D6D2920463A537065656420286D6D2F76
:1005A0006D29205A3A205A4C69667420286D6D29AD
:1005B000002044002049002020204D3330342050BA
:1005C00000504944206865617462656420736574F5
:1005D00074696E67733A002044002049002020208F
:1005E0004D33303120500050494420736574746994
:1005F0006E67733A00205A0020590020204D323097
:1006000036205800486F6D65206F666673657420EC
:10061000286D6D293A00204500205A0020590020FD
:10062000580020420020540020204D323035205305
:1006300000416476616E636564207661726961620F
:100640006C65733A20533D4D696E20666565647232
:1006500061746520286D6D2F73292C20543D4D69E0
:100660006E2074726176656C206665656472617473
:100670006520286D6D2F73292C20423D6D696E69B0
:100680006D756D207365676D656E742074696D6539
:1006900020286D73292C20583D6D6178696D756D2A
:1006A000205859206A65726B20286D6D2F73292C94
:1006B00020205A3D6D6178696D756D205A206A65FC
:1006C000726B20286D6D2F73292C2020453D6D61A4
:1006D00078696D756D2045206A65726B20286D6D97
:1006E0002F73290020540020204D32303420530035
:1006F000416363656C65726174696F6E3A20533D46
:10070000616363656C65726174696F6E2C20543D22
:100710007265747261637420616363656C65726194
:1007200074696F6E00204500205A00205900202077
:100730004D3230312058004D6178696D756D204122
:100740006363656C65726174696F6E20286D6D2FCF
:100750007332293A00204500205A002059002020F9
:100760004D3230332058004D6178696D756D2066CB
:10077000656564726174657320286D6D2F73293A05
:1007800000204500205A0020590020204D393220F9
:10079000580053746570732070657220756E6974AB
:1007A0003A0053657474696E67732053746F726591
:1007B0006400454550524F4D204572726F720000E3
:1007C00020006D65736820626564206C6576656CD9
:1007D000696E673A200029002C20002C20007068E8
:1007E00079736963616C20636F6F7264696E6174A1
:1007F00065733A20280029002C20002C2000776FF8
:10080000726C6420636F6F7264696E617465733AB1
:100810002028002046002045004731205A004D3254
:1008200034004D32362053256C75004D3130362062
:10083000530047312046256400473120453120468A
:10084000343830004731205A0020463230303000F2
:1008500020590047312058004D383300506F7369DC
:1008600074696F6E20726561642066726F6D2065B9
:100870006570726F6D3A004D3233202573002E671C
:10088000636F0046656564726174653A0072656302
:100890006F7665725F6D616368696E655F737461C1
:1008A00074655F61667465725F706F7765725F70A3
:1008B000616E69632C20696E697469616C200072D5
:1008C00065636F7665725F6D616368696E655F739E
:1008D000746174655F61667465725F706F7765726D
:1008E0005F70616E69632C20696E697469616C2048
:1008F000007265636F7665725F6D616368696E65CE
:100900005F73746174655F61667465725F706F7741
:1009100065725F70616E69632C20696E69746961CC
:100920006C200063757272656E745F706F736974AA
:10093000696F6E5B5A5F415849535D3A0043757267
:1009400072656E7420706F736974696F6E20595F81
:10095000415849533A0043757272656E7420706F46
:10096000736974696F6E20585F415849533A00416A
:10097000667465722077616974696E6720666F724C
:100980002074656D703A00473120452D3120463482
:1009900038300047312045352046313230004D385F
:1009A00033004D31393020532564004D313039202A
:1009B0005325640047323820582059004731205AC7
:1009C00032352046383030004D31343020532564E4
:1009D000004D3130342053256400494E54340055C5
:1009E000564C4F202D20656E640073747073005553
:1009F000564C4F0020423A0020453A00543A005AE3
:100A0000206C6976652061646A757374206F7574F3
:100A1000206F662072616E67652E2053657474695D
:100A20006E6720746F20302E20436C69636B2074D6
:100A30006F20636F6E74696E75652E005A206C6945
:100A400076652061646A757374206F7574206F66B3
:100A50002072616E67652E2053657474696E67201D
:100A6000746F20300020573A0020453A00543A0075
:100A70004B494C4C3A20004175746F0020452F447F
:100A80003D00416476616E6365204B3D0022283253
:100A900029005400496E76616C6964205420636FAC
:100AA00064652E00496E76616C6964204D20636F29
:100AB00064652E004D3232302053256900203A20E3
:100AC00000004C414E472053454C20464F52434571
:100AD0004400222831290020453A00205A3A0020BB
:100AE000593A0020453A00205A3A0020593A005815
:100AF0003A004D31313320530020002E0020423A7D
:100B00000020453A00543A0020413A0020503A0073
:100B10002042403A0020403A00202F003A00205462
:100B200000202F0020423A00202F006F6B20543A03
:100B3000002569206D696E2C20256920736563008E
:100B4000496E76616C6964204D20636F6465004D69
:100B500065736820626564206C6576656C696E6794
:100B6000206E6F74206163746976652E000A002020
:100B700020000A4D6561737572656420706F696E3F
:100B800074733A000A5A207365617263682068655D
:100B9000696768743A20002C004E756D20582C59F6
:100BA0003A2000476F20686F6D652066696E697333
:100BB000686564004D65736820626564206C6576C5
:100BC000656C696E67206163746976617465640041
:100BD000557073616D706C652066696E69736865C8
:100BE0006400426564206C6576656C696E6720639D
:100BF0006F7272656374696F6E2066696E6973687F
:100C0000656400206D6963726F6E7300457863657B
:100C1000737369766520626564206C6576656C69BE
:100C20006E6720636F7272656374696F6E3A20003D
:100C30006261627973746570206170706C6965645B
:100C400000636C65616E2075702066696E697368FB
:100C50006564200000206F66667365743A20006D3D
:100C600065736820626564206C6576656C696E6783
:100C70003A2000473238205730003A200054656D42
:100C800070657261747572652063616C696272610E
:100C900074696F6E20646F6E652E20436F6E746989
:100CA0006E75652077697468207072657373696EFC
:100CB0006720746865206B6E6F622E0000205A20DA
:100CC000736869667420286D6D293A0050494E4456
:100CD000412074656D70657261747572653A2000AB
:100CE000002F3600537465703A200000205A20739C
:100CF0006869667420286D6D293A0050494E444158
:100D00002074656D70657261747572653A20002F8C
:100D1000362028736B6970706564290053746570A0
:100D20003A2000005A45524F3A2000007374617215
:100D3000742074656D70657261747572653A200017
:100D400050494E44412070726F62652063616C6946
:100D500062726174696F6E207374617274004732DD
:100D600038205730000A00205A3A200020593A20F3
:100D70000020583A20004732382C2066696E616C9A
:100D800020004732382C2066696E616C20004732A3
:100D9000382C2066696E616C20004732382C20693F
:100DA0006E697469616C20004732382C20696E6965
:100DB0007469616C200043524153485F4445544577
:100DC00043544544004D323900627573793A2070BE
:100DD000617573656420666F7220696E707574004A
:100DE000627573793A2070617573656420666F72FD
:100DF000207573657200627573793A2070726F6343
:100E0000657373696E67002055706C6F616420694B
:100E10006E2070726F677265737300696E697469B2
:100E2000616C207A737465707320616674657220DA
:100E300072657365743A2000696E697469616C202B
:100E40007A7374657073206F6E20706F776572208F
:100E500075703A2000466163746F72792052455371
:100E60004554004E6F762032362032303137004301
:100E70006F6D70696C65643A2000286E6F6E652C2A
:100E80002064656661756C7420636F6E666967299E
:100E9000004E6F7620323620323031372031393AE9
:100EA00030393A3339007374617274001B5B324A13
:100EB0001B5B313B31484F726967696E616C205032
:100EC000727573612069331B5B323B334850727516
:100ED000736120526573656172636800250020208C
:100EE0002020202000202020202020004552415397
:100EF000494E4720616C6C206461746100466163F7
:100F0000746F7279205245534554004352415348FF
:100F10005F5245434F5645520047323820590047EB
:100F20003238205800FFFFFF0000A0400000A04022
:100F30000000004000007F43000056439AD951430F
:100F400000000000000080C09A99193E00007F4315
:100F5000000052430000524300000000000080C027
:100F60009A99193E6563686F3A004572726F723ADA
:100F70000000002110422063308440A550C660E785
:100F800070088129914AA16BB18CC1ADD1CEE1EF3E
:100F9000F13112100273325222B5529442F772D6D6
:100FA00062399318837BB35AA3BDD39CC3FFF3DE8E
:100FB000E36224433420040114E664C774A4448526
:100FC000546AA54BB528850995EEE5CFF5ACC58DDE
:100FD000D55336722611163006D776F6669556B476
:100FE000465BB77AA719973887DFF7FEE79DD7BC2E
:100FF000C7C448E5588668A77840086118022823C6
:1010000038CCC9EDD98EE9AFF9488969990AA92B7D
:10101000B9F55AD44AB77A966A711A500A333A1215
:101020002AFDDBDCCBBFFB9EEB799B588B3BBB1ACD
:10103000ABA66C877CE44CC55C222C033C600C4165
:101040001CAEED8FFDECCDCDDD2AAD0BBD688D491D
:101050009D977EB66ED55EF44E133E322E511E70B5
:101060000E9FFFBEEFDDDFFCCF1BBF3AAF599F786D
:101070008F8891A981CAB1EBA10CD12DC14EF16F1E
:10108000E18010A100C230E3200450254046706783
:1010900060B9839893FBA3DAB33DC31CD37FE35EAF
:1010A000F3B1029012F322D23235421452776256D3
:1010B00072EAB5CBA5A89589856EF54FE52CD50DBF
:1010C000C5E234C324A01481046674476424540523
:1010D00044DBA7FAB79987B8975FE77EF71DC73C4F
:1010E000D7D326F2369106B0165766767615463473
:1010F000564CD96DC90EF92FE9C899E9898AB9AB5F
:10110000A94458654806782768C018E1088238A3C2
:10111000287DCB5CDB3FEB1EFBF98BD89BBBAB9AEE
:10112000BB754A545A376A167AF10AD01AB32A9212
:101130003A2EFD0FED6CDD4DCDAABD8BADE89DC9FE
:101140008D267C076C645C454CA23C832CE01CC162
:101150000C1FEF3EFF5DCF7CDF9BAFBABFD98FF88E
:101160009F176E367E554E745E932EB23ED10EF0B2
:101170001E7C3C3E5E2B3D3F2F5B5D3B2C2A225C60
:10118000004D383420582059205A2045004D323423
:10119000004D3233202573006175746F25692E6709
:1011A000000A002F000A002E0044656C6574696F08
:1011B0006E206661696C65642C2046696C653A2016
:1011C0000046696C652064656C657465643A002E40
:1011D000002E002E002E004E6F7720667265736819
:1011E0002066696C653A20004E6F7720646F696EE7
:1011F000672066696C653A20002220706F730022B8
:1012000020706172656E743A2200535542524F55F8
:1012100054494E452043414C4C20746172676574BB
:101220003A2200747279696E6720746F2063616C72
:101230006C207375622D67636F64652066696C65E9
:1012400073207769746820746F6F206D616E7920E8
:101250006C6576656C732E204D4158206C65766503
:101260006C2069733A00256920686F7572732025B8
:1012700069206D696E757465730054494D454F550D
:10128000543A004D3131300046756C6C2052582074
:101290004275666665720022206661696C65643A13
:1012A000204275666665722066756C6C2100456E1D
:1012B000717565696E6720746F2074686520667249
:1012C0006F6E743A2022002200456E717565696E5A
:1012D0006720746F207468652066726F6E743A20A0
:1012E000220022206661696C65643A204275666658
:1012F00065722066756C6C210022004D363030001E
:101300005072757361206933204D4B3320626572D2
:101310006569742E005072757361206933204D4BDE
:101320003320707265702E005072757361206933BE
:10133000204D4B332070726F6E74612E00507275A9
:101340007361206933204D4B33206F6B00507275F1
:101350007361206933204D4B332072656164792EAF
:10136000007A5F6D696E3A20007A5F6D61783A208D
:10137000005A204F666673657400795F6D696E3A36
:101380002000795F6D61783A20005920456E7466BF
:1013900065726E756E6720766F6D206D696E0044A4
:1013A000697374616E7A612059206461206D696E81
:1013B0003A005920767A64616C656E6F7374206FA1
:1013C00064206D696E3A00592064697374616E63BC
:1013D000652066726F6D206D696E3A004A61005338
:1013E0006900536900416E6F0059657300785F6D45
:1013F000696E3A2000785F6D61783A200058595A3A
:10140000204B616C2E2044657461696C73005859DF
:101410005A2043616C2E206465747461676C6900A6
:1014200044657461696C792058595A206B616C2E3F
:101430000058595A2063616C2E2064657461696C90
:101440007300496368207765726465206A65747A01
:101450007420646965205A204B616C696272696509
:1014600072756E672064757263686675656872650B
:101470006E2E00566F79206120686163657220438B
:10148000616C6962726163696F6E205A2061686F76
:1014900072612E0041646573736F206176766965B1
:1014A000726F20756E612043616C696272617A6946
:1014B0006F6E65205A2E004E796E692070726F76BD
:1014C000656475207A206B616C6962726163692E54
:1014D00000492077696C6C2072756E207A206361F8
:1014E0006C6962726174696F6E206E6F772E00494D
:1014F0006368207765726465206A65747A74206415
:1015000069652058595A2D4B616C69627269657220
:10151000756E672064757263686675656872656E5E
:101520002E20457320776972642063612E2031324A
:10153000204D696E7574656E2064617565726E000C
:1015400048617265206C612063616C6962726163DD
:10155000696F6E2058595A2E20546172646172610D
:10156000203132206D696E2E206170726F78696D46
:101570006164616D656E74652E0041646573736F9F
:10158000206176766965726F20756E612043616CAB
:10159000696272617A696F6E652058595A2E2050BF
:1015A000756F206475726172652063697263612072
:1015B0003132206D696E2E004E796E692070726F27
:1015C000766564752078797A206B616C69627261E6
:1015D00063692E205A616265726520746F20707293
:1015E00069626C697A6E65203132206D696E2E00F9
:1015F000492077696C6C2072756E2078797A206347
:10160000616C6962726174696F6E206E6F772E20F3
:1016100049742077696C6C2074616B65206170700F
:10162000726F782E203132206D696E732E004A65FC
:10163000747A7420776572646520696368206469D0
:1016400065204475657365206675657220504C4150
:1016500020766F726865697A656E2E2000566F7904
:1016600020612070726563616C656E7461722065C3
:101670006C206E6F7A7A6C65207061726120504CBC
:10168000412061686F72612E0041646573736F2041
:1016900070726572697363616C6465726F206C2728
:1016A0007567656C6C6F2070657220504C412E0020
:1016B0004E796E692070726564656872656A69202A
:1016C000747279736B752070726F20504C412E00CC
:1016D0004E6F7720492077696C6C20707265686561
:1016E0006174206E6F7A7A6C6520666F7220504C40
:1016F000412E0048616C6C6F2C2069636820626920
:101700006E206465696E204F726967696E616C2036
:10171000507275736120693320447275636B657212
:101720002E204D6F65636874656E20536965206D6A
:1017300065696E652048696C6665206475726368CA
:101740002064656E2053657475702D50726F7A65D4
:1017500073733F00486F6C612C20736F7920747530
:1017600020696D707265736F7261204F726967696D
:101770006E616C2050727573612069332E20517533
:101780006965726573207175652074652067756978
:1017900065206120747261766573206465206C61D8
:1017A00020636F6E66696775726163696F6E3F0073
:1017B0004369616F2C20736F6E6F206C61207475AC
:1017C00061207374616D70616E7465204F7269671A
:1017D000696E616C2050727573612069332E2047E9
:1017E00072616469726573746920616975746F20D0
:1017F0006174747261766572736F20696C207072A7
:101800006F636573736F20646920636F6E666967C9
:101810007572617A696F6E653F00446F62727920FC
:1018200064656E2C206A73656D2076617365207423
:1018300069736B61726E61204F726967696E616C6A
:101840002050727573612069332E2043686365747C
:1018500065206162796368205661732070726F76CB
:1018600065646C61206B616C69627261636E696D45
:101870002070726F636573656D3F0048692C204965
:1018800020616D20796F7572204F726967696E6192
:101890006C205072757361206933207072696E74A8
:1018A00065722E20576F756C6420796F75206C6996
:1018B0006B65206D6520746F20677569646520799C
:1018C0006F75207468726F7567682074686520731F
:1018D000657475702070726F636573733F00496340
:1018E00068207765726465206A65747A7420657211
:1018F000737465204C696E696520647275636B65ED
:101900006E2E205761656872656E64206465732071
:10191000447275636B6573206B6F656E6E656E20C8
:101920005369652064696520447565736520616C41
:101930006C6D6165686C6963682073656E6B656E5C
:1019400020696E64656D205369652064656E204B67
:101950006E6F70662064726568656E2C20626973B4
:101960002053696520646965206F7074696D616CCE
:101970006520486F65686520657272656963686592
:101980006E2E2055656265727072756566656E2093
:10199000536965206469652042696C6465722069D9
:1019A0006E20756E736572656D2048616E64627538
:1019B000636820696D204B61706974656C204B61B0
:1019C0006C696272696572756E6700566F79206125
:1019D00020636F6D656E7A6172206120696D70722F
:1019E000696D6972206C61206C696E656120792077
:1019F00074752062616A6172617320656C206E6F1C
:101A00007A7A6C65206772616475616C6D656E745D
:101A10006520616C20726F74617220656C206D614D
:101A20006E646F2C20686173746120717565206C21
:101A30006C65677565732061206C6120616C7475DD
:101A40007261206F7074696D612E204D6972612022
:101A50006C617320696D6167656E65732064656C88
:101A6000206361706974756C6F2043616C69627288
:101A70006163696F6E20656E20656C206D616E75A7
:101A8000616C2E0041646573736F20696E697A69B9
:101A900065726F2061207374616D7061726520756D
:101AA0006E61206C696E6561206520747520646FBD
:101AB0007672616920616262617373617265206C24
:101AC000277567656C6C6F20706F636F207065722F
:101AD00020766F6C74612072756F74616E646F2014
:101AE0006C61206D616E6F706F6C612073696E6FD9
:101AF0002061207261676769756E67657265207520
:101B00006E6120616C74657A7A61206F7474696D9E
:101B1000616C652E20506572206661766F7265205B
:101B200064616920756E6F207367756172646F20E0
:101B3000616C6C27696D6D6167696E652064656CA9
:101B4000206E6F7374726F206D616E75616C652CA1
:101B5000206361702E43616C696272617A696F6E95
:101B6000652E005A61636E75207469736B6E6F75B4
:101B700074206C696E6B75206120567920627564E3
:101B800065746520706F737475706E6520736E690F
:101B90007A6F76617420747279736B75206F7461DB
:101BA00063656E696D20746C616369746B61206438
:101BB0006F6B7564206E65646F7361686E657465C4
:101BC000206F7074696D616C6E69207679736B79C2
:101BD0002E2050726F686C65646E65746520736941
:101BE000206F6272617A6B792076206E6173692052
:101BF00070726972756363652076206B61706974B9
:101C00006F6C65204B616C6962726163650049208D
:101C100077696C6C20737461727420746F207072B9
:101C2000696E74206C696E6520616E6420796F75D1
:101C30002077696C6C206772616475616C6C7920C7
:101C40006C6F77657220746865206E6F7A7A6C6548
:101C500020627920726F746174696E6720746865A0
:101C6000206B6E6F622C20756E74696C20796F75B5
:101C7000207265616368206F7074696D616C2068A3
:101C800065696768742E20436865636B20746865B6
:101C900020706963747572657320696E206F757248
:101CA0002068616E64626F6F6B20696E206368618B
:101CB000707465722043616C6962726174696F6EE1
:101CC0002E004A65747A74207765726465206963B2
:101CD000682064656E2041627374616E64207A7757
:101CE00069736368656E2044756573656E737069AA
:101CF000747A6520756E6420447275636B626574D6
:101D000074206B616C696272696572656E2E005633
:101D10006F7920612063616C6962726172206C610D
:101D20002064697374616E63696120656E747265A5
:101D3000206C612070756E74612064656C206E6F1C
:101D40007A7A6C652079206C612073757065726693
:101D500069636965206465206C61206865617462EF
:101D600065642E0041646573736F207461726572DF
:101D70006F206C6F2073746163636F2066726120E3
:101D80007567656C6C6F2065207375706572666928
:101D900063652064656C2070696174746F2E004EF9
:101DA000796E69207A6B616C696272756A692076F6
:101DB0007A64616C656E6F7374206D657A69206BEF
:101DC0006F6E63656D20747279736B79206120701A
:101DD0006F76726368656D206865617462656475AD
:101DE0002E004E6F7720492077696C6C2063616C00
:101DF0006962726174652064697374616E636520E1
:101E00006265747765656E20746970206F662074F2
:101E10006865206E6F7A7A6C6520616E64206865F3
:101E2000617462656420737572666163652E005A21
:101E3000756E616563687374206675656872652088
:101E40006963682064656E2053656C6273747465A1
:101E5000737420647572636820756D2064696520F1
:101E6000686165756669677374656E2050726F622C
:101E70006C656D65206265692064657220417566D8
:101E8000626175207A75207565626572707275651C
:101E900066656E2E005072696D65726F2C206861E8
:101EA000726520656C2053656C6674657374207070
:101EB00061726120636F6D70726F626172206C6F0E
:101EC000732070726F626C656D6173206465206D44
:101ED0006F6E74616A65206D617320636F6D756EDE
:101EE00065732E00416E7A69747574746F20617623
:101EF000766965726F20696C2053656C6620546545
:101F000073742070657220636F6E74726F6C6C6195
:101F1000726520676C69206572726F7269206469EE
:101F200020617373656D626C616767696F207069AA
:101F30007520636F6D756E692E004E656A647269F7
:101F40007620706F6D6F63692073656C667465735E
:101F50007475207A6B6F6E746F6C756A69206E652C
:101F60006A63617374656A73692063687962792052
:101F7000767A6E696B616A69636920707269207331
:101F80006573746176656E69207469736B61726ED6
:101F9000792E0046697273742C20492077696C6C25
:101FA0002072756E207468652073656C6674657345
:101FB0007420746F20636865636B206D6F73742089
:101FC000636F6D6D6F6E20617373656D626C7920E8
:101FD00070726F626C656D732E00446572206C6167
:101FE0007566656E646520417373697374656E749C
:101FF000206C6F65736368742064696520616B741D
:1020000075656C6C65204B616C696272696572659F
:10201000726765626E6973736520756E6420776997
:10202000726420766F6E20416E66616E6720616E0D
:1020300020626567696E6E656E2E20466F727473DE
:1020400065747A656E3F00456A65637574617220D8
:10205000656C2057697A61726420626F7272617276
:1020600061206C6F732076616C6F7265732064659C
:102070002063616C6962726163696F6E2061637471
:1020800075616C6573207920636F6D656E7A61721E
:1020900061206465206E7565766F2E20436F6E74C7
:1020A000696E7561723F00536520617676692069BB
:1020B0006C2057697A617264207065726465726120
:1020C00069206C612063616C696272617A696F6E0C
:1020D00065207072656573697374656E74652065DB
:1020E00020646F76726169207269636F6D696E63D7
:1020F000696172652064616C6C27696E697A696FC9
:102100002E20436F6E74696E756172653F00537067
:10211000757374656E692057697A6172646120769F
:10212000796D617A6520756C6F7A656E6520767958
:10213000736C65646B79207673656368206B616C82
:1021400069627261636920612073707573746920BC
:102150006B616C69627261636E692070726F636536
:1021600073206F64207A616361746B752E20506FE9
:102170006B7261636F7661743F0052756E6E696E4B
:10218000672057697A6172642077696C6C20646596
:102190006C6574652063757272656E742063616C22
:1021A0006962726174696F6E20726573756C7473A5
:1021B00020616E642073746172742066726F6D208A
:1021C00074686520626567696E6E696E672E20436C
:1021D0006F6E74696E75653F004D6F6563687465F9
:1021E0006E205369652064656E206C65747A746531
:1021F0006E205363687269747420776965646572D0
:10220000686F6C656E20756D2064656E2041627329
:1022100074616E64207A7769736368656E204475B3
:1022200065736520756E6420447275636B626574B6
:1022300074206E65752065696E7A757374656C6C53
:10224000656E3F00517569657265732072657065D2
:1022500074697220656C20756C74696D6F20706193
:10226000736F2070617261207265616A7573746149
:1022700072206C612064697374616E636961206EA1
:102280006F7A7A6C652D686561746265643F00449D
:1022900065736964657269207269706574657265D9
:1022A000206C27756C74696D6F2070617373616742
:1022B00067696F20706572206D69676C696F726104
:1022C0007265206C612064697374616E7A61206646
:1022D0007261207567656C6C6F2065207069617430
:1022E000746F3F00436863657465206F70616B6F46
:1022F00076617420706F736C65646E69206B726FA9
:102300006B206120706F7A6D656E697420767A64D7
:10231000616C656E6F7374206D657A692074727973
:10232000736B6F75206120686561746265643F003E
:10233000446F20796F752077616E7420746F2072FE
:102340006570656174206C617374207374657020AE
:10235000746F20726561646A757374206469737444
:10236000616E6365206265747765656E206E6F7A55
:102370007A6C6520616E6420686561746265643F93
:1023800000536965206B6F656E6E656E20696D6DBB
:1023900065722064656E204173697374656E74653F
:1023A0006E20696D204D656E75206E6575206175B6
:1023B00066727566656E3A204B616C69627269651A
:1023C00072756E67202D3E20417373697374616E60
:1023D00074005369656D707265207075656465730E
:1023E000206163636564657220616C206173697349
:1023F00074656E74652064657364652043616C69FF
:1024000062726163696F6E202D3E2057697A617236
:1024100064004520706F73736962696C6520707227
:102420006F73656775697265206C61206775696493
:10243000652057697A61726420696E207175616CDC
:102440007369617369206D6F6D656E746F2061745F
:10245000747261766572736F2043616C6962726138
:102460007A696F6E65202D3E2057697A6172642EFD
:102470000057697A61726461206D757A65746520B0
:102480006B64796B6F6C6976207A6E6F76752073EA
:10249000707573746974207A206D656E7520436160
:1024A0006C6962726174696F6E202D3E2057697A83
:1024B00061726400596F752063616E20616C776191
:1024C000797320726573756D65207468652057692E
:1024D0007A6172642066726F6D2043616C6962720A
:1024E0006174696F6E202D3E2057697A6172642E87
:1024F00000497374206573207769726B6C69636837
:1025000020504C412046696C616D656E743F0045FA
:102510007320656C2066696C616D656E746F205008
:102520004C413F00452071756573746F20756E20B6
:1025300066696C616D656E746F20646920504C41F2
:102540003F004A6520746F20504C412066696C61E1
:102550006D656E743F00497320697420504C4120B2
:1025600066696C616D656E743F004675656872657D
:102570006E2053696520626974746520504C412057
:1025800046696C616D656E7420696E2064656E20AD
:10259000457874727564657220756E642062657327
:1025A000746165746967656E205369652064656E42
:1025B000204B6E6F706620756D206573207A7520D4
:1025C0006C6164656E2E00496E73657274612C20B7
:1025D000706F72206661766F722C2066696C616D17
:1025E000656E746F20504C4120656E20656C2065CF
:1025F00078747275736F722E20446573707565738D
:102600002068617A20636C69632070617261206365
:1026100061726761726C6F2E005065722066617620
:102620006F726520696E7365726973636920696C86
:102630002066696C616D656E746F20646920504C12
:1026400041206E656C6C276573747275736F72656B
:102650002C20706F69207072656D69206C61206D2F
:10266000616E6F706F6C612070657220636172695A
:10267000636172652E0050726F73696D20766C6FA6
:102680007A746520504C412066696C616D656E748A
:1026900020646F206578747275646572752C207083
:1026A0006F20746520737469736B6E657465207434
:1026B0006C616369746B6F2070726F207A617665EC
:1026C00064656E692066696C616D656E74752E0057
:1026D000506C6561736520696E7365727420504C2F
:1026E000412066696C616D656E7420746F2074683A
:1026F000652065787472756465722C207468656EE7
:10270000207072657373206B6E6F6220746F206C23
:102710006F61642069742E004269747465206C6175
:1027200064656E2053696520504C412D46696C618B
:102730006D656E7420756E642066616872656E20CA
:10274000536965206D69742064656D2041737369F8
:102750007374656E74656E20666F72742C20696E7A
:1027600064656D205369652064656E2044727563ED
:102770006B6572206E6575207374617274656E2E60
:102780000043617267612066696C616D656E746F8C
:1027900020504C412C20706F72206661766F722C35
:1027A0002079207265696E69636961206C612069B6
:1027B0006D707265736F7261207061726120636FFA
:1027C0006E74696E75617220636F6E20656C205740
:1027D000697A61726400506572206661766F726515
:1027E000206361726963612066696C616D656E74F6
:1027F0006F20646920504C412065207269707265B9
:102800006E646920696C2057697A61726420646F14
:10281000706F206176657220726961767669617485
:102820006F206C61207374616D70616E74652E0031
:1028300050726F73696D207A61766564746520509B
:102840004C412066696C616D656E74206120706F0B
:10285000207465206F626E6F7674652057697A61A7
:1028600072646120737469736B6E7574696D207224
:102870006573657420746C616369746B612E0050BC
:102880006C65617365206C6F616420504C412066FB
:10289000696C616D656E7420616E64207468656E2C
:1028A00020726573756D652057697A617264206264
:1028B00079207265626F6F74696E67207468652035
:1028C0007072696E7465722E00566F726865697AEF
:1028D000656E206465722044756573652E204269BB
:1028E0007474652077617274656E2E005072656332
:1028F000616C656E74616E646F206E6F7A7A6C6560
:102900002E2045737065726120706F72206661764B
:102910006F722E0053746F207072657269736361F9
:102920006C64616E646F206C277567656C6C6F2ECC
:1029300020506572206661766F72652061747465DF
:102940006E64692E00507265646568726976616DA7
:1029500020747279736B752E2050726F73696D20BD
:1029600063656B656A74652E005072656865617495
:10297000696E67206E6F7A7A6C652E20506C656187
:10298000736520776169742E0049737420646173E4
:102990002046696C616D656E742067656C61646565
:1029A0006E3F004573746120656C2066696C616DD3
:1029B000656E746F206361726761646F3F00496C7C
:1029C0002066696C616D656E746F2065207374613B
:1029D000746F20636172696361746F3F004A6520A0
:1029E00066696C616D656E74207A61766564656E8A
:1029F0003F0049732066696C616D656E74206C6F71
:102A0000616465643F00416C6C6573207775726426
:102A10006520676574616E2E205669656C20537061
:102A2000617373206265696D20447275636B656EB6
:102A300021005465726D696E61646F212046656C7A
:102A4000697A20696D70726573696F6E21004265E5
:102A50006E20666174746F2E2042756F6E612073F4
:102A600074616D70612100567365206A6520686F1E
:102A7000746F766F2E00416C6C20697320646F6EEA
:102A8000652E204861707079207072696E74696E6D
:102A90006721004269747465207265696E696765B3
:102AA0006E2053696520646173204865697A6265A8
:102AB000747420756E642064727565636B656E2036
:102AC0005369652064616E6E2064656E204B6E6F85
:102AD00070662E004C696D706961206C61207375A1
:102AE0007065726669636965206465206C61206841
:102AF0006561746265642C20706F72206661766F08
:102B0000722C20792068617A20636C6963005065BB
:102B100072206661766F72652070756C6973636987
:102B200020696C2070696174746F2C20706F69204B
:102B30007072656D69206C61206D616E6F706F6C75
:102B4000612E0050726F73696D206F6369737465D5
:102B500074652068656174626564206120737469BE
:102B6000736B6E65746520746C616369746B6F2E32
:102B700000506C6561736520636C65616E206865EB
:102B8000617462656420616E64207468656E207093
:102B90007265737320746865206B6E6F622E0042DD
:102BA00069747465207565626572707275656665B5
:102BB0006E2053696520756E7365722048616E647E
:102BC0006275636820756E64206265686562656E13
:102BD00020536965206461732050726F626C656D6B
:102BE0002E2046616872656E205369652064616EAF
:102BF0006E206D69742064656D2041737369737410
:102C0000656E74656E20666F72742C20696E6465E3
:102C10006D205369652064656E20447275636B6531
:102C200072206E6575207374617274656E2E004C2F
:102C3000656520656C206D616E75616C2079207210
:102C4000657375656C766520656C2070726F626C5B
:102C5000656D612E20446573707565732C207265F7
:102C6000696E69636961206C6120696D707265735A
:102C70006F7261207920636F6E74696E7561206375
:102C80006F6E20656C2057697A61726400506572BE
:102C9000206661766F726520636F6E73756C746108
:102CA00020696C206E6F7374726F206D616E756138
:102CB0006C6520706572207269736F6C76657265E1
:102CC00020696C2070726F626C656D612E20506F90
:102CD000692072697072656E646920696C20576939
:102CE0007A61726420646F706F2061766572207201
:102CF000696176766961746F206C61207374616DAF
:102D000070616E74652E0050726F73696D206E6114
:102D1000686C65646E65746520646F206D616E75A6
:102D2000616C752061206F707261767465207072BD
:102D30006F626C656D2E20506F207465206F626E1F
:102D40006F7674652057697A61726461207265627A
:102D50006F6F746F76616E696D207469736B6172E9
:102D60006E792E00506C6561736520636865636BD6
:102D7000206F75722068616E64626F6F6B20616E88
:102D80006420666978207468652070726F626C6573
:102D90006D2E205468656E20726573756D652074A4
:102DA00068652057697A6172642062792072656271
:102DB0006F6F74696E6720746865207072696E74D5
:102DC00065722E0057697A617264002057617463DE
:102DD00068646F6720526573657400496E666F7230
:102DE0006D6174696F6E004D6F6E69746F72697A90
:102DF00061720053636865726D61746120696E660B
:102E00006F00496E666F726D61636500496E666F33
:102E10002073637265656E0045727374652D53632C
:102E20006869636874204B616C0043616C2E20708C
:102E300072696D657261206361702E0043616C2E52
:102E4000207072696D6F206C617965722E004B6124
:102E50006C2E207072766E692076727374767900AB
:102E60004669727374206C617965722063616C2E9F
:102E70000057617274652061756620757365722EE6
:102E80002E2E004573706572616E646F206F7264E0
:102E9000656E657300417474656E64656E646F2061
:102EA0007574656E7465005761697420666F722071
:102EB000757365722E2E2E004265696D2044727501
:102EC000636B2062656E75747A7465005573616416
:102ED0006F20656E20696D70726573696F6E005545
:102EE00073617469206E656C6C61207374616D70C0
:102EF0006100506F757A69746520626568656D2040
:102F00007469736B75005573656420647572696EBE
:102F100067207072696E740046696C616D656E74CD
:102F200020656E746C6164656E00536F6C746172C1
:102F30002066696C616D656E746F005363617269C0
:102F400063612066696C616D656E746F0056796AA5
:102F50006D6F75742066696C616D656E7400556E79
:102F60006C6F61642066696C616D656E74004669A2
:102F70006C616D656E742061757377657266656EE0
:102F800000536F6C74616E646F2066696C616D656F
:102F90006E746F0052696C6173632E2066696C6198
:102FA0006D656E746F005679736F7576616D20660E
:102FB000696C616D656E7400556E6C6F6164696EED
:102FC000672066696C616D656E7400556E6B6E6F1F
:102FD000776E20636F6D6D616E643A2022004665E6
:102FE000696E65696E7374656C6C756E6700416AB5
:102FF0007573746172005265676F6C61004C616437
:1030000069740054756E65005344204B6172746599
:10301000205B466C6173684169725D0053442063B4
:10302000617264205B466C73684169725D00534451
:10303000204B61727465205B6E6F726D616C5D0018
:1030400053442063617264205B6E6F726D616C5DCE
:103050000054656D702E204B616C2E205B4F4E5DD1
:103060000043616C2E2074656D702E205B4F4E5DA9
:103070000043616C2E2074656D702E205B4F4E5D99
:10308000005465706C2E206B616C2E205B4F4E5D82
:103090000054656D702E2063616C2E205B4F4E5D79
:1030A0000054656D702E204B616C2E205B4F4646A0
:1030B0005D0043616C2E2074656D702E205B4F4661
:1030C000465D0043616C2E2074656D702E205B4F51
:1030D00046465D005465706C2E206B616C2E205B43
:1030E0004F46465D0054656D702E2063616C2E2046
:1030F0005B4F46465D0054656D702E204B616C69D8
:103100006272696572756E67206665727469672E92
:10311000204B6C69636B656E20756D2077656974F3
:103120006572207A7520676568656E2E0043616C54
:1031300069627261636F6E2074656D70657261742F
:10314000757261207465726D696E6164612E2048CC
:10315000617A20636C6963207061726120636F6EB5
:1031600074696E7561722E0054617261747572615A
:103170002074656D7065726174757261207465721A
:103180006D696E6174612E204661726520636C69A1
:10319000636B2070657220636F6E74696E75617207
:1031A000652E005465706C6F746E69206B616C697C
:1031B000627261636520646F6B6F6E63656E612E12
:1031C00020506F6B726163756A74652073746973E4
:1031D0006B656D20746C616369746B612E0054655E
:1031E0006D70657261747572652063616C6962727D
:1031F0006174696F6E2069732066696E69736865B2
:10320000642E20436C69636B20746F20636F6E744F
:10321000696E75652E0054656D70204B616C696236
:103220002E2020202020202020200043616C2E20F2
:1032300074656D702E20202020202020202020006A
:1032400043616C2E2074656D702E2020202020207C
:1032500020202020005465706C2E206B616C2E2085
:103260002020202020202020200054656D702E205A
:1032700063616C2E2020202020202020202000545C
:10328000656D706572617475720054656D706572FC
:1032900061747572610054656D70657261747572E8
:1032A00061005465706C6F74610054656D70657277
:1032B000617475726500536F706F72746500506F42
:1032C00064706F726100537570706F727400447235
:1032D00075636B2061626272656368656E00446548
:1032E00074656E657220696D70726573696F6E00CA
:1032F00041727265737461207374616D7061005AFC
:1033000061737461766974207469736B0053746FB0
:1033100070207072696E7400474553544F5050547A
:103320002E200050415241444100415252455354D5
:1033300041544F2E0053544F505045442E200053BB
:103340007465707261746520746F6F206869676856
:103350003A2000497320737465656C207368656555
:1033600074206F6E20686561746265643F00546FFD
:1033700074616C6520447275636B7A6569743A0098
:103380005469656D706F20746F74616C203A0054DD
:10339000656D706F207374616D706120746F743A25
:1033A0000043656C6B6F767920636173203A00543B
:1033B0006F74616C207072696E742074696D652021
:1033C0003A00476573616D7466696C616D656E7412
:1033D0003A0046696C616D656E746F20746F74613C
:1033E0006C3A0046696C616D656E746F20746F7421
:1033F0003A0046696C616D656E742063656C6B653F
:103400006D203A00546F74616C2066696C616D6563
:103410006E74203A00447275636B7A6569743A2061
:1034200020005469656D706F20646520696D702E91
:103430003A0054656D706F206469207374616D701B
:10344000613A00436173207469736B75203A2020E0
:10345000005072696E742074696D653A20200046D0
:10346000696C616D656E74766572627261756368B0
:103470003A0046696C616D656E746F2075736164A6
:103480006F3A20200046696C616D656E746F20751F
:103490007361746F3A0046696C616D656E74203AB1
:1034A00020200046696C616D656E742075736564DB
:1034B0003A20200053746174697374696B656E20DF
:1034C00000457374616469737469636173202000DB
:1034D00053746174697374696368650053746174CB
:1034E000697374696B61202000537461746973742B
:1034F0006963732020004572726F72202D207374EF
:1035000061746963206D656D6F72792068617320E5
:103510006265656E206F7665727772697474656E28
:1035200000476573636877696E6469676B65697482
:103530000056656C6F63696461640056656C6F6307
:1035400069746100527963686C6F737400537065BD
:1035500065640020536F66747761726520526573ED
:103560006574004C656963687465722053636872A2
:103570002E3A00496E636C2E206C65676765726138
:103580003A004C65686B65207A6B6F73656E693ABB
:1035900000536C6967687420736B65773A004D6FF0
:1035A000646520202020205B6C656973655D004D9B
:1035B0006F646F2020205B73696C656E63696F5D5B
:1035C000004D6F646F205B73696C656E7A696F7311
:1035D0006F5D004D6F64202020202020205B7469E7
:1035E0006368795D004D6F646520202020205B7347
:1035F000696C656E745D004D6F6465205B486F6833
:1036000065204C656973745D004D6F646F205B725B
:10361000656E642E706C656E6F5D004D6F64652025
:1036200020202020205B666F7274655D004D6F6402
:1036300020205B7679732E2076796B6F6E5D004D5E
:103640006F6465205B6869676820706F7765725D7D
:1036500000456E64736368616C74657220537461B5
:10366000742E00456E73656E6120746F7065206600
:10367000696E616C00537461746F2066696E656376
:103680006F7273610053746176206B6F6E632E20CE
:103690007370696E2E0053686F7720656E642073B7
:1036A000746F70730053636877657265722053633B
:1036B00068722E3A00496E632E2072696C657661DD
:1036C0006E74653A0054657A6B65207A6B6F73652A
:1036D0006E693A0053657665726520736B65773A5B
:1036E0000054656D702E2065696E7365747A656E21
:1036F0000045737461626C656365722074656D70FA
:103700002E3A00496D706F7374612074656D706539
:10371000726174757261004E6173746176746520B4
:103720007465706C6F74753A005365742074656DC0
:1037300070657261747572653A0045696E7374657F
:103740006C6C756E67656E00436F6E666967757247
:103750006163696F6E00496D706F7374617A696F30
:103760006E69004E6173746176656E6900536574AD
:1037700074696E6773005665726472616874756E01
:10378000676665686C6572004572726F7220646569
:1037900020636F6E6578696F6E004572726F726537
:1037A000206361626C616767696F00436879626179
:1037B000207A61706F6A656E6900576972696E6719
:1037C000206572726F720053656C627374746573F6
:1037D000742073746172742000496E6963696F208C
:1037E00053656C6674657374004176766961206117
:1037F00075746F746573740053656C6620746573BB
:10380000742073746172742020004269747465209E
:103810007072756566653A00436F6E74726F6C61A5
:10382000203A00566572696669636172653A005AAA
:103830006B6F6E74726F6C756A7465203A00506CB1
:103840006561736520636865636B203A0053656C3E
:1038500062737474657374204F4B004175746F7498
:10386000657374204F4B0053656C662074657374E8
:10387000204F4B004E6963687420616E6765736307
:10388000686C6F7373656E004E6F2068617920639A
:103890006F6E6578696F6E2020004E6F6E20636FCB
:1038A0006E6E6573736F004E657A61706F6A656ED8
:1038B0006F20202020004E6F7420636F6E6E656352
:1038C000746564004D6F746F7265004D6F746F7234
:1038D00000486F74656E640052697363616C642E96
:1038E0002F5465726D6973742E004865617465723A
:1038F0002F546865726D6973746F72004C756566DC
:103900007465727465737400546573742076656EA3
:1039100074696C61646F7265730050726F766120B8
:1039200064656C2076656E74696C61746F720054A6
:103930006573742076656E74696C61746F7275005E
:1039400046616E20746573740053656C62737474A1
:10395000657374206D6973736C756E672E004661B4
:103960006C6C6F2053656C6674657374004175747C
:103970006F746573742066616C6C69746F00536555
:103980006C66746573742073656C68616C202000CC
:1039900053656C6674657374206661696C65642038
:1039A00020004C696E6B6572204C7565667465729B
:1039B0003F0056656E742E20697A71756965726470
:1039C0006F3F0056656E742053582073756C6C27DA
:1039D0007567656C6C6F3F004C6576792076656E17
:1039E00074206E61207472797363653F004C656664
:1039F0007420686F74656E642066616E3F00536565
:103A00006C6274657374204665686C657221004150
:103A100075746F74657374206572726F72210041E2
:103A200075746F74657374206E6567617469766F01
:103A30000053656C6674657374206572726F7220D2
:103A40002100456E6465206E696368742067657443
:103A5000726F662E00546F7065206E6F20616C630C
:103A6000616E7A61646F0046696E65632E206675CB
:103A70006F726920706F722E00456E6473746F7080
:103A8000206E6F742068697400456E6473636861AA
:103A90006C74657200546F7065732066696E616C3A
:103AA00065730046696E65636F7273612028322901
:103AB00000456E6473746F707300546F7065206698
:103AC000696E616C0046696E65636F727361004573
:103AD0006E6473746F7000566F72646572657220E5
:103AE0004C7565667465723F0056656E742E20666F
:103AF000726F6E74616C3F0056656E74206469204D
:103B00007374616D706120616E742E3F0050726538
:103B1000646E69207469736B6F76792076656E7454
:103B20003F0046726F6E74207072696E7420666119
:103B30006E3F00507275656665205A204163687358
:103B4000652020202000436F6E74726F6C20746FAC
:103B50007065205A005665726966696361206173F9
:103B60007365205A004B6F6E74726F6C61205A201F
:103B700061786973202000436865636B696E672014
:103B80005A2061786973202000507275656665203F
:103B9000592041636873652020202000436F6E74B4
:103BA000726F6C20746F706520590056657269667B
:103BB00069636120617373652059004B6F6E747285
:103BC0006F6C61205920617869732020004368651B
:103BD000636B696E672059206178697320200050FB
:103BE00072756566652058204163687365202020E2
:103BF0002000436F6E74726F6C20746F7065205874
:103C00000056657269666963612061737365205847
:103C1000004B6F6E74726F6C61205820617869730D
:103C2000202000436865636B696E672058206178C7
:103C30006973202000507275656665204475657350
:103C40006500436F6E74726F6C20686F74656E648C
:103C500020005665726966696361207567656C6CE2
:103C60006F004B6F6E74726F6C6120686F74656E5D
:103C700064202000436865636B696E6720686F7419
:103C8000656E6420200050727565666520456E641F
:103C9000736368616C746572202000436F6E747288
:103CA0006F6C20746F706573005665726966696326
:103CB000612066696E65636F727361004B6F6E742D
:103CC000726F6C6120656E6473746F70730043680B
:103CD00065636B696E6720656E6473746F707300E3
:103CE000507275656665204265747420202020201E
:103CF00020202000436F6E74726F6C2068656174C1
:103D0000626564005665726966696361206C6574FA
:103D1000746F004B6F6E74726F6C6120626564200B
:103D20002020202000436865636B696E6720626510
:103D300064202020202000416C6C65732072696330
:103D4000687469672020202000546F646F206269C6
:103D5000656E004E657373756E206572726F726565
:103D600000567365204F4B2020202020202020204B
:103D7000202000416C6C20636F7272656374202098
:103D8000202020200042657474202F204865617433
:103D900065720048656174626564004C6574746F97
:103DA0002F52697363616C642E00426564202F207A
:103DB0004865617465720041786973206C656E674F
:103DC000746800417869730053656C62737474653C
:103DD0007374202020202020200053656C667465B9
:103DE0007374004175746F746573740053656C6609
:103DF000746573742020202020202020200057721A
:103E00006974696E6720746F2066696C653A20007A
:103E1000766F6C756D652E696E6974206661696C6C
:103E20006564002053697A653A2000534420656E2A
:103E3000746665726E7420005461726A65746120E4
:103E400072657469726164610053442072696D6FB8
:103E5000737361004B617274612076796A6D757459
:103E60006100436172642072656D6F766564005312
:103E700044207072696E74696E672062797465207F
:103E8000006F70656E206661696C65642C20466900
:103E90006C653A20006F70656E526F6F74206661BA
:103EA000696C65640053442065696E676573657469
:103EB0007A74005461726A65746120696E73657208
:103EC0007461646100534420696E73657269746142
:103ED000004B6172746120766C6F7A656E6100438D
:103EE00061726420696E7365727465640053442066
:103EF000696E6974206661696C0046696C6520733F
:103F0000656C65637465640046696C65206F7065F7
:103F10006E65643A20006572726F72207772697400
:103F2000696E6720746F2066696C65005344206376
:103F3000617264206F6B0043616E6E6F7420656EFA
:103F4000746572207375626469723A200052656309
:103F50006874733A004465737472613A0050726118
:103F600076793A0052696768743A00447275636BF7
:103F700020776569746572676568656E0052656172
:103F80006E7564617220696D70726573696F6E0021
:103F90005374616D706120696E207269707265730F
:103FA00061004F626E6F766F76616E69207469731F
:103FB0006B7500526573756D696E67207072696EFE
:103FC0007400447275636B20666F72746765736505
:103FD000747A7400526573756D69656E646F2069DB
:103FE0006D70726573696F6E0052697072656E6490
:103FF00069207374616D7061004F626E6F76656EDB
:1040000069207469736B7500526573756D696E67AD
:10401000207072696E7400466F72747365747A658D
:104020006E005265616E7564617220696D707265B3
:10403000732E0052697072656E6469207374616DCD
:10404000706100506F6B7261636F766174005265CE
:1040500073756D65207072696E7400526573656E5C
:10406000643A2000506C656173652072656D6F76EF
:104070006520737465656C2073686565742066726D
:104080006F6D20686561746265642E00426C6163C7
:104090006B6F7574206F636375727265642E205246
:1040A00065636F766572207072696E743F00526549
:1040B000636F766572696E67207072696E74202016
:1040C000202000686F77746F2E707275736133648F
:1040D0002E637A00686F77746F2E70727573613318
:1040E000642E636F6D00666F72756D2E70727573DE
:1040F0006133642E637A00666F72756D2E7072750F
:10410000736133642E636F6D007072757361336415
:104110002E637A00707275736133642E636F6D0065
:10412000447275636B2070617573696572740049C0
:104130006D70726573696F6E20656E207061757346
:1041400061005374616D706120696E2070617573D8
:1041500061005469736B20706F7A61737461766566
:104160006E005072696E74207061757365640044EE
:104170007275636B206162676562726F6368656EFA
:1041800000496D70726573696F6E2063616E63655F
:104190006C616461005374616D70612061626F7263
:1041A00074697461005469736B2070726572757301
:1041B000656E005072696E742061626F727465641E
:1041C000005072696E74657220646973636F6E6EFD
:1041D000656374656400756E64204B6E6F70662055
:1041E00064727565636B656E0048617A20636C6903
:1041F00063006520636C696363617265206D616E45
:104200006F706F6C61006120737469736B6E65749D
:104210006520746C616369746B6F00616E642070FB
:104220007265737320746865206B6E6F62004475ED
:1042300065736520566F72776165726D656E0050AB
:10424000726563616C656E746172206578747275F5
:10425000736F72005072657269732E207567656C9A
:104260006C6F210050726564656872656A746520C0
:10427000747279736B752100507265686561742082
:10428000746865206E6F7A7A6C652100566F72775C
:104290006165726D656E0050726563616C656E7408
:1042A00061720050726572697363616C6461005081
:1042B00072656465687265760050726568656174E0
:1042C00000506F776572557000426974746520778D
:1042D000617274656E00506F72204661766F722055
:1042E000457370657261720041737065747461002A
:1042F00050726F73696D2063656B656A74650050F9
:104300006C656173652077616974004269747465D6
:10431000206C6164656E20536965207A75657273DF
:104320007420504C412046696C616D656E742E009E
:10433000436172676120656C2066696C616D656EB2
:10434000746F20504C41207072696D65726F2070DF
:104350006F72206661766F722E0050657220666102
:10436000766F7265207072696D6120636172696336
:104370006172652066696C616D656E746F20646939
:1043800020504C412E004E656A6472697665207A31
:1043900061766564746520504C412066696C616D7E
:1043A000656E742070726F73696D2E00506C65615C
:1043B0007365206C6F616420504C412066696C61AC
:1043C0006D656E742066697273742E004973742073
:1043D000504C412046696C616D656E742067656C58
:1043E0006164656E3F004573746120656C20666989
:1043F0006C616D656E746F20504C41206361726713
:1044000061646F3F00496C20504C412065207374FB
:1044100061746F20636172696361746F3F004A6504
:1044200020504C412066696C616D656E74207A6124
:10443000766564656E3F00497320504C4120666983
:104440006C616D656E74206C6F616465643F002003
:1044500020506C616E6E6572427566666572427957
:104460007465733A2000506C6561736520706C61EF
:10447000636520737465656C207368656574206F6F
:104480006E20686561746265642E0050494E444137
:10449000206572776165726D656E0043616C656E53
:1044A00074616E646F2050494E44410052697363D9
:1044B000616C642E2050494E4441004E616872691F
:1044C00076616E692050494E44410050494E444146
:1044D0002048656174696E670054656D706572612E
:1044E000747572207775726465206E6963687420D4
:1044F0006B616C69627269657274004C61207465ED
:104500006D70657261747572612064652063616CA1
:104510006962726163696F6E206E6F2068612073DB
:1045200069646F20616A75737461646100546172BB
:1045300061747572612064656C6C612074656D7066
:1045400065726174757261206E6F6E20616E636F4B
:104550007261206573656775697461005469736B76
:1045600061726E61206E6562796C61207465706C39
:104570006F746E65207A6B616C6962726F76616EC2
:10458000610054656D706572617475726520636158
:104590006C6962726174696F6E20686173206E6FFE
:1045A00074206265656E2072756E207965740050A6
:1045B0004944204B616C69622E0043616C2E20508F
:1045C000494420202020202020202020200043615A
:1045D0006C2E2050494400504944206B616C2E20C1
:1045E000202020202020202020200050494420632B
:1045F000616C2E2020202020202020202020005010
:104600004944204B616C69622E206665727469674B
:104610000043616C2E20504944207465726D696EB0
:104620006164610043616C2E2050494420636F6DCA
:10463000706C65746100504944206B616C2E20756C
:104640006B6F6E63656E61005049442063616C2E30
:104650002066696E697368656400504944204B6147
:104660006C696272696572756E670043616C69623C
:10467000726163696F6E205049440043616C6962E6
:1046800072617A696F6E6520504944005049442038
:104690006B616C69627261636500504944206361BB
:1046A0006C6962726174696F6E00447275636B202D
:1046B000756E74657262726563682E005061757301
:1046C000617220696D70726573696F6E004D6574FB
:1046D000746920696E20706175736100506F7A6132
:1046E000737461766974207469736B0050617573BB
:1046F00065207072696E74004C6567656E2065692F
:104700006E20426C6174742050617069657220750E
:104710006E746572206469652044756573652077E1
:1047200061656872656E6420646572204B616C69B6
:104730006272696572756E67206465722065727356
:1047400074656E20342050756E6B74652E2057652D
:104750006E6E2064696520447565736520646173BD
:10476000205061706965722065696E6B6C656D6D56
:10477000742C20447275636B657220736F666F7260
:104780007420617573736368616C74656E00436F48
:104790006C6F63617220756E6120686F6A6120645E
:1047A0006520706170656C20736F627265206C614A
:1047B0002073757065726669636965206465206938
:1047C0006D70726573696F6E20647572616E746569
:1047D000206C612063616C6962726163696F6E2035
:1047E0006465206C6F73207072696D65726F7320E1
:1047F000342070756E746F732E205369206C6120A5
:10480000626F7175696C6C61206D75657665206588
:104810006C20706170656C2C206170616761722022
:10482000696D707265736F726120696E6D65646920
:104830006174616D656E74652E00506F72726520D3
:10484000756E20666F676C696F20736F74746F206C
:104850006C277567656C6C6F20647572616E74652A
:10486000206C612063616C696272617A696F6E6548
:1048700020646569207072696D6920342070756EDE
:1048800074692E20496E206361736F206C277567F1
:10489000656C6C6F206D756F766120696C20666F3A
:1048A000676C696F20737065676E657265207072E2
:1048B0006F6E74616D656E7465206C6120737461D8
:1048C0006D70616E74652E00556D697374657465E5
:1048D000206C69737420706170697275206E61203C
:1048E000706F646C6F7A6B752061207564727A7575
:1048F0006A7465206A656A20706F642074727973C7
:104900006B6F7520626568656D206D6572656E6997
:10491000207072766E696368203420626F64752E31
:1049200020506F6B756420747279736B61207A61AB
:1049300063687974692070617069722C207679706F
:104940006E657465207469736B61726E752E0050AC
:104950006C6163652061207368656574206F6620F3
:10496000706170657220756E646572207468652070
:104970006E6F7A7A6C6520647572696E67207468F0
:10498000652063616C6962726174696F6E206F6625
:10499000206669727374203420706F696E74732E90
:1049A00020496620746865206E6F7A7A6C65206392
:1049B00061746368657320746865207061706572E6
:1049C0002C20706F776572206F6666207468652092
:1049D0007072696E74657220696D6D656469617469
:1049E000656C792E006F6B004F6666004B65696ED3
:1049F00065204265776567756E672E0053696E2086
:104A00006D6F76696D69656E746F004E6573737551
:104A10006E206D6F76696D656E746F2E004E6F201F
:104A20006D6F76652E004B65696E65205344204B93
:104A300061727465004E6F20686179207461726ADA
:104A4000657461205344004E657373756E61205325
:104A500044005A61646E61205344206B617274613A
:104A6000004E6F2053442063617264004475657387
:104A700065005567656C6C6F00547279736B6100EB
:104A80004E6F7A7A6C650046696C2E206E69636899
:104A9000742067656C6164656E0046696C2E206EDB
:104AA0006F20696E74726F64756369646F00466924
:104AB0006C2E206E6F6E20636172696361746F008B
:104AC00046696C616D656E74206E657A61766564A9
:104AD000656E0046696C616D656E74206E6F742042
:104AE0006C6F6164656400466172626520756E6B0F
:104AF0006C617200436F6C6F72206E6F20686F6D17
:104B00006F67656E656F00436F6C6F7265206E6FC7
:104B10006E207075726F004261727661206E656EF4
:104B20006920636973746100436F6C6F72206E6FEC
:104B30007420636C656172004E65696E004E65009D
:104B40004E6F00426974746520616B7475616C69A5
:104B500073696572656E2E0041637475616C697A64
:104B6000617220706F72206661766F72005072659C
:104B7000676120616767696F726E612E0050726FA6
:104B800073696D20616B7475616C697A756A74659F
:104B90002E00506C65617365207570677261646585
:104BA0002E004E657565204669726D7761726520CD
:104BB00056657273696F6E20766572667565676299
:104BC00061723A004E7565766F206669726D776125
:104BD000726520646973706F6E69626C653A004E2D
:104BE000756F76612076657273696F6E6520646596
:104BF0006C206669726D7761726520646973706F8D
:104C00006E6962696C65005679736C61206E6F76AF
:104C100061207665727A65206669726D776172656A
:104C20003A004E6577206669726D7761726520760D
:104C3000657273696F6E20617661696C61626C6523
:104C40003A00426577656765205A004D6F76657258
:104C5000205A004D756F7669205A00506F73756E3B
:104C60006F7574205A004D6F7665205A0042657743
:104C70006567652059004D6F7665722059004D7546
:104C80006F7669205900506F73756E6F7574205977
:104C9000004D6F766520590042657765676520583D
:104CA000004D6F7665722058004D756F76692058FB
:104CB00000506F73756E6F75742058004D6F766578
:104CC00020580045787472756972004D756F766969
:104CD000204573747275736F7265004578747275D0
:104CE00064657200416368736265776567756E67B6
:104CF000004D6F76657220656A6573004D756F763D
:104D000069206173736500506F73756E6F757420E1
:104D10006F7375004D6F76652061786973004D651E
:104D200073682042657474204C6576656C696E67A3
:104D3000004D657368206C6976656C2E206C657417
:104D4000746F004D65736820426564204C6576651C
:104D50006C696E67004B616C696272696572756E31
:104D6000670043616C6962726163696F6E004361E1
:104D70006C696272617A696F6E65004B616C696221
:104D8000726163650043616C6962726174696F6E20
:104D90000020766F6E203900206465203900207372
:104DA00075203900207A203900206F662039004DA7
:104DB000657373656E206465722052656665726501
:104DC0006E7A686F65686520646573204B616C69F5
:104DD000627269657270756E6B746573004D69649B
:104DE00069656E646F20616C747572612064656CB6
:104DF0002070756E746F2064652063616C696272E7
:104E00006163696F6E004D69737572617265206CC4
:104E100027616C74657A7A612064692072696665BD
:104E200072696D656E746F2064656C2070756E7448
:104E30006F2064692063616C696272617A696F6E68
:104E400065004D6572696D207265666572656E6399
:104E50006E69207679736B75206B616C6962726123
:104E6000636E69686F20626F6475004D656173756C
:104E700072696E67207265666572656E636520682B
:104E80006569676874206F662063616C696272612E
:104E900074696F6E20706F696E740053636872611D
:104EA00065676C6175663A00496E636C2E206D69AA
:104EB0007375726174613A004D6572656E65207A32
:104EC0006B6F73656E693A004D65617375726564E9
:104ED00020736B65773A0048617570746D656E7507
:104EE00065004D656E75207072696E636970616CE6
:104EF000004D656E75207072696E636970616C65D6
:104F000000486C61766E69206E616269646B610055
:104F10004D61696E004D32323120496E76616C69A7
:104F20006420657874727564657220004D32313882
:104F300020496E76616C6964206578747275646569
:104F40007220004D32303020496E76616C696420E9
:104F5000657874727564657220005265706F727442
:104F6000696E6720656E6473746F7020737461740A
:104F70007573004D3131372045727374652D53635D
:104F80006869636874204B616C2E004D31313720A5
:104F900043616C2E207072696D657261206361706F
:104FA0002E004D3131372043616C2E207072696DB7
:104FB0006F206C617965722E004D313137204B6165
:104FC0006C2E207072766E6920767273747679001A
:104FD0004D313137204669727374206C6179657286
:104FE0002063616C2E004649524D574152455F4E39
:104FF000414D453A4D61726C696E2056312E302E0E
:10500000323B20537072696E7465722F6772626CE6
:10501000206D617368757020666F722067656E36EB
:10502000204649524D574152455F55524C3A68749B
:105030007470733A2F2F6769746875622E636F6D91
:105040002F707275736133642F50727573612D699F
:10505000332D506C75732F2050524F544F434F4C8B
:105060005F56455253494F4E3A312E30204D414301
:1050700048494E455F545950453A50727573612006
:105080006933204D4B332045585452554445525FA7
:10509000434F554E543A3120555549443A303030FB
:1050A00030303030302D303030302D303030302D09
:1050B000303030302D3030303030303030303030F3
:1050C000300A004D31303920496E76616C696420B8
:1050D000657874727564657220004D3130352049F1
:1050E0006E76616C6964206578747275646572208F
:1050F000004D31303420496E76616C6964206578EA
:1051000074727564657220004C6F73652052696516
:105110006D656E7363686569626500506F6C65618B
:10512000207375656C74610050756C6567676961A3
:10513000206C656E74610055766F6C6E656E6120D3
:1051400072656D656E69636B61004C6F6F7365208E
:1051500070756C6C65790046696C616D656E742064
:105160006C6164656E00496E74726F647563697218
:105170002066696C616D2E0043617269636120660F
:10518000696C616D656E746F005A61766573742029
:1051900066696C616D656E74004C6F616420666950
:1051A0006C616D656E740046696C616D656E74202E
:1051B0006C6561647400496E74726F6475636965CF
:1051C0006E646F2066696C616D2E00436172696365
:1051D000616E646F2066696C616D2E005A61766144
:1051E00064656E692066696C616D656E7475004CEE
:1051F0006F6164696E672066696C616D656E7400CD
:105200004C6164652046617262650043616D62694C
:10521000616E646F20636F6C6F72004361726963CB
:10522000616E646F20636F6C6F72650043697374A5
:10523000656E69206261727679004C6F6164696E97
:105240006720636F6C6F72004C696E6B733A00532A
:10525000696E69737472613A004C6576793A004CF4
:105260006566743A00576165686C652053707261B9
:105270006368650043616D6269616520656C2069E2
:1052800064696F6D610053656C657A696F6E61204A
:105290006C696E677561005679626572206A617A21
:1052A000796B610053656C656374206C616E677522
:1052B0006167650044657574736368004573706168
:1052C0006E6F6C004974616C69616E6F0043657349
:1052D00074696E6100456E676C697368004142478E
:1052E0004542524F4348454E2E20005041524144C2
:1052F0004120444520454D455247454E43494100D4
:10530000494E2054494C542E004B494C4C45442E98
:105310002000496E76616C696420657874727564EA
:1053200065720046696C616D656E742065696E6CAE
:105330006567656E00496E74726F6475636972208B
:1053400066696C616D656E746F00496E7365726934
:1053500072652066696C616D656E746F00566C6F66
:105360007A74652066696C616D656E7400496E7350
:105370006572742066696C616D656E740050726947
:105380006E742046414E3A20004E6F7A7A6C65204A
:1053900046414E3A00457874727564657220696EB4
:1053A000666F0020766F6E20340020646520340024
:1053B000207375203400207A203400206F6620345A
:1053C00000566572626573736572756E672042651B
:1053D0007474204B616C69627269657270756E6B72
:1053E00074004D656A6F72616E646F2070756E74C3
:1053F0006F2064652063616C6962726163696F6EBE
:1054000020686561746265640050657266657A69DA
:105410006F6E2E20696C206C6574746F2070756ED1
:10542000746F2064692063616C696272617A2E0016
:105430005A6C657073756A6920707265736E6F73EC
:1054400074206B616C69627261636E69686F20625F
:105450006F647500496D70726F76696E6720626562
:10546000642063616C6962726174696F6E20706F31
:10547000696E74004B616C69627269657265205A6D
:105480000043616C696272616E646F205A0043610F
:105490006C696272616E646F205A004B616C696264
:1054A00072756A69205A0043616C6962726174693D
:1054B0006E67205A004B616C696272696572756E25
:1054C00067204F4B0043616C6962726163696F6E64
:1054D000204F4B0043616C696272617A696F6E653F
:1054E000204F4B004B616C696272616365204F4BCA
:1054F0000043616C6962726174696F6E20646F6EE3
:1055000065004B616C696272696572656E205A0054
:1055100043616C6962726172205A0043616C696216
:105520007261205A004B616C6962726F76617420FF
:105530005A0043616C696272617465205A0041755A
:1055400066776165726D656E204F4B0043616C65D7
:105550006E74616D69656E746F2066696E616C2E24
:105560000052697363616C642E20636F6D706C65AB
:10557000746F005A6168726976616E69204F4B2EB4
:105580000048656174696E6720646F6E652E004126
:105590007566776165726D656E0043616C656E74EA
:1055A000616E646F2E2E2E0052697363616C6461AC
:1055B0006D656E746F2E2E2E005A61687269766169
:1055C0006E690048656174696E670046696C2E20DB
:1055D00073656E736F7220205B6F6E5D0046696C41
:1055E0002E2073656E736F72205B6F66665D0020A0
:1055F00046726565204D656D6F72793A200044658D
:105600007220447275636B657220777572646520D1
:105610006E6F6368206E69636874206B616C696289
:1056200072696572742E20426974746520666F6CAD
:1056300067656E20536965206461732048616E64FC
:10564000627563682C204B61706974656C204669D3
:105650007273742073746570732C20416273636875
:105660006E6974742043616C6962726174696F6EF3
:1056700020666C6F772E00496D707265736F726172
:10568000206E6F20657374612063616C6962726162
:10569000646120746F64617669612E20506F72209E
:1056A0006661766F722075736120656C206D616E26
:1056B00075616C2C206361706974756C6F2046692C
:1056C0007273742073746570732C2043616C69620B
:1056D000726174696F6E20666C6F772E005374610F
:1056E0006D70616E746520616E636F7261206E6FA4
:1056F0006E2063616C6962726174612E205369204F
:105700007072656761206469207365677569726589
:1057100020696C206D616E75616C652C2063617011
:1057200069746F6C6F205052494D4920504153535A
:10573000492C2073657A696F6E652064656C6C61B5
:105740002063616C696272617A696F6E652E0054C4
:1057500069736B61726E61206E6562796C61206A3B
:1057600065737465207A6B616C6962726F76616EC5
:10577000612E20506F73747570756A746520707235
:105780006F73696D20706F646C65206D616E7561FB
:105790006C752C206B617069746F6C61205A616349
:1057A000696E616D652C206F64737461766563202A
:1057B000506F73747570206B616C696272616365A0
:1057C0002E005072696E74657220686173206E6F6E
:1057D00074206265656E2063616C696272617465D4
:1057E00064207965742E20506C6561736520666F46
:1057F0006C6C6F7720746865206D616E75616C2CC0
:1058000020636861707465722046697273742073D6
:10581000746570732C2073656374696F6E204361C7
:105820006C6962726174696F6E20666C6F772E00AE
:105830004475726368666C75737300466C756A6F45
:1058400000466C7573736F00507275746F6B004611
:105850006C6F77004265776567756E672062656576
:105860006E64656E005465726D2E206D6F76696D85
:1058700069656E746F73004172726573746F20692D
:105880006E20636F72736F00446F6B6F6E636F7621
:10589000616E6920706F687962750046696E697320
:1058A00068696E67206D6F76656D656E7473002034
:1058B000766F6E20340020646520340020737520DC
:1058C0003400207A203400206F6620340053756342
:1058D00068656E2042657474204B616C6962726900
:1058E000657270756E6B740042757363616E646F80
:1058F0002070756E746F2064652063616C696272DC
:105900006163696F6E2068656174626564005269E5
:1059100063657263612064656C206C6574746F20CC
:1059200070756E746F2064692063616C6962726166
:105930007A2E00486C6564616D206B616C696272DF
:1059400061636E6920626F6420706F646C6F7A6B44
:105950007900536561726368696E672062656420CF
:1059600063616C6962726174696F6E20706F696ED9
:1059700074005265697465726163696F6E200052CC
:105980006569746572617A696F6E65200049746536
:10599000726163652000497465726174696F6E207D
:1059A00000446F6E6520736176696E672066696C6E
:1059B000652E00446F6E65207072696E74696E6743
:1059C0002066696C650049737420466172626520C7
:1059D0007265696E3F00457320656C206E75657653
:1059E0006F20636F6C6F72206E697469646F3F0023
:1059F000496C20636F6C6F7265206527206E697437
:105A000069646F3F004A6520626172766120636954
:105A10007374613F00497320636F6C6F7220636C15
:105A20006561723F0046696C616D656E742D5765E6
:105A3000636873656C0043616D62696172206669B9
:105A40006C616D656E746F0043616D622E206669D6
:105A50006C616D656E746F0056796D656E6974204A
:105A600066696C616D656E74004368616E67652080
:105A700066696C616D656E74004C756566746572FF
:105A80002D54656D706F0056656C6F636964616459
:105A90002056656E742E0056656C6F6369746120C4
:105AA00076656E742E00527963686C6F737420761D
:105AB000656E742E0046616E2073706565640065C6
:105AC0006E717565696E6720220045787472757312
:105AD0006F72004573747275736F726500457874E8
:105AE0007275646572002045787465726E616C2011
:105AF0005265736574005072696E746572207374B8
:105B00006F707065642064756520746F20657272B3
:105B10006F72732E204669782074686520657272F2
:105B20006F7220616E6420757365204D393939209C
:105B3000746F20726573746172742E202854656DC1
:105B40007065726174757265206973207265736522
:105B5000742E205365742069742061667465722008
:105B600072657374617274696E6729004E6F204CA0
:105B7000696E65204E756D62657220776974682064
:105B8000636865636B73756D2C204C617374204C76
:105B9000696E653A20004E6F20436865636B7375CC
:105BA0006D2077697468206C696E65206E756D6212
:105BB00065722C204C617374204C696E653A20002C
:105BC00020746F6F206C6F6E6720657874727573C8
:105BD000696F6E2070726576656E746564004C69DD
:105BE0006E65204E756D626572206973206E6F74EC
:105BF000204C617374204C696E65204E756D626532
:105C0000722B312C204C617374204C696E653A20E4
:105C1000005072696E7465722068616C7465642EE0
:105C2000206B696C6C28292063616C6C65642100B1
:105C300020636F6C6420657874727573696F6E2071
:105C400070726576656E74656400636865636B7316
:105C5000756D206D69736D617463682C204C617380
:105C600074204C696E653A20004645484C45523ACE
:105C7000004552524F52453A0043485942413A007A
:105C80004552524F523A00456E642066696C652059
:105C90006C697374006F70656E00545249474745D4
:105CA00052454400656E6473746F70732068697444
:105CB0003A200045696E656E204D6F6D656E7420EB
:105CC00062697474652E00456E206573706572613B
:105CD00000536F7370656E73696F6E652E2E2E00A4
:105CE000536C6565702E2E2E004D6F746F72656E4D
:105CF0002061757300417061676172206D6F746F10
:105D0000726573004469736162696C6974206D6FB8
:105D1000746F7269005679706E6F7574206D6F7450
:105D20006F72790044697361626C65207374657089
:105D30007065727300446174756D00446174610034
:105D4000446174756D3A00446174653A00416B7446
:105D500075656C6C65730041637475616C004174AA
:105D60007475616C6500506F757A6520616B747530
:105D7000616C6E690043757272656E740043726186
:105D80007368206465742E2020205B6F6E5D004375
:105D900072617368206465742E20205B6F66665D97
:105DA0000020436F756E7420583A20005765636871
:105DB00073656C206F6B3F0043616D626961646F56
:105DC00020636F72726563742E3F0043616D626978
:105DD00061746F20636F72722E3F0056796D656E2D
:105DE00061206F6B3F004368616E67656420636F7D
:105DF00072726563746C793F0041626B7565686CA3
:105E0000656E00456E667269617200526166667207
:105E100065646461005A63686C6164697400436F0F
:105E20006F6C646F776E00204C61737420557064E2
:105E3000617465643A2000576165686C656E205333
:105E4000696520457874727564657200456C656794
:105E50006972206578747275736F723A0053656C5D
:105E6000657A696F6E61206573747275736F7265A0
:105E70003A0056796265727465206578747275644B
:105E800065723A0043686F6F736520657874727548
:105E90006465723A005765636873656C2065726665
:105EA0006F6C67722E210043616D62696F20636FB2
:105EB00072726563746F0043616D62696F2072690D
:105EC00075736369746F21005A6D656E6120757317
:105ED0007065736E6121004368616E67652073753C
:105EE00063636573732100447275636B656E20761E
:105EF0006F6E205344004D656E75207461726A6543
:105F00007461205344005374616D7061206461209A
:105F10005344005469736B207A20534400507269D3
:105F20006E742066726F6D2053440054656D702E40
:105F3000206B616C696272696572656E0043616CA9
:105F40006962726163696F6E2074656D702E0054B2
:105F5000617261747572612074656D702E00546594
:105F6000706C6F742E206B616C6962726163650086
:105F700054656D702E2063616C6962726174696F23
:105F80006E0043616C6962726174696E67205A00C9
:105F90004B616C696272696572656E0043616C6920
:105FA000627261720043616C696272617265005A6B
:105FB0006B616C6962726F7661740043616C6962D7
:105FC000726174650052657365742058595A204B8C
:105FD000616C6962722E0052657365742058595A5B
:105FE000206B616C6962722E005265736574205873
:105FF000595A2063616C6962722E004B616C696250
:1060000072696572756E672058595A0043616C69F0
:106010006272612058595A0043616C696272612052
:1060200058595A004B616C69627261636520585916
:106030005A0043616C6962726174652058595A0054
:106040002042726F776E206F75742052657365748D
:1060500000426567696E2066696C65206C697374BF
:106060000058595A2D4B616C696272696572756E80
:106070006720756E67656E61752E204C696E6B6565
:106080007220766F726465726572204B616C696212
:106090007269657270756E6B7420697374207A759D
:1060A000207765697420766F726E652E0043616C8F
:1060B000696272617A696F6E2058595A20636F6DF8
:1060C00070726F6D65746964612E2050756E746FA7
:1060D0002066726F6E74616C20697A717569657281
:1060E000646F206E6F20616C63616E7A61626C65B3
:1060F0002E0043616C696272617A696F6E65205827
:10610000595A20636F6D70726F6D657373612E20C5
:1061100050756E746F20616E746572696F72652060
:1061200073696E697374726F206E6F6E207261672F
:106130006769756E676962696C652E004B616C6991
:1061400062726163652058595A206E65707265737A
:106150006E612E204C65767920707265646E6920C0
:10616000626F64206D6F63207670726564752E00B7
:1061700058595A2063616C6962726174696F6E204C
:10618000636F6D70726F6D697365642E204C656608
:10619000742066726F6E742063616C6962726174E0
:1061A000696F6E20706F696E74206E6F74207265F7
:1061B00061636861626C652E0058595A2D4B616CA1
:1061C000696272696572756E6720756E67656E616A
:1061D000752E20566F7264657265204B616C696222
:1061E0007269657270756E6B74652073696E642078
:1061F0007A75207765697420766F726E652E00431C
:10620000616C696272617A696F6E2058595A2063B5
:106210006F6D70726F6D65746964612E2050756E5C
:10622000746F732066726F6E74616C6573206E6F2D
:1062300020616C63616E7A61626C65732E004361EC
:106240006C696272617A696F6E652058595A206371
:106250006F6D70726F6D657373612E2050756E7403
:106260006920616E746572696F7269206E6F6E204D
:106270007261676769756E676962696C692E004B48
:10628000616C6962726163652058595A206E65704D
:106290007265736E612E20507265646E69206B6149
:1062A0006C69627261636E6920626F6479206D6FE0
:1062B00063207670726564752E0058595A206361A8
:1062C0006C6962726174696F6E20636F6D70726F5A
:1062D0006D697365642E2046726F6E742063616C05
:1062E0006962726174696F6E20706F696E74732079
:1062F0006E6F7420726561636861626C652E005810
:10630000595A204B616C696272696572756E6720BB
:10631000696E204F72646E756E672E20582F59205B
:1063200041636873656E2073696E6420657477617C
:1063300073207363686965662E0043616C696272DD
:106340006163696F6E2058595A20636F727265637A
:1063500074612E204C6F7320656A65732058202F5E
:10636000205920657374616E206C69676572616D78
:10637000656E746520696E636C696E61646F732EFF
:10638000204275656E2074726162616A6F210043FC
:10639000616C696272617A696F6E2058595A206324
:1063A0006F7272657474612E204173736920582F67
:1063B00059206C65676765726D656E7465207374CE
:1063C0006F7274692E2042656E20666174746F214D
:1063D000004B616C6962726163652058595A20767E
:1063E00020706F7261646B752E20582F59206F7367
:1063F00079206D69726E65207A6B6F73656E652E9C
:1064000020446F6272612070726163652100585987
:106410005A2063616C6962726174696F6E20616C8D
:106420006C2072696768742E20582F592061786536
:10643000732061726520736C696768746C7920736E
:106440006B657765642E20476F6F64206A6F6221E9
:106450000058595A204B616C696272696572756E99
:106460006720696E204F72646E756E672E205363CD
:10647000686965666865697420776972642061750A
:10648000746F6D617469736368206B6F7272696792
:10649000696572742E0043616C6962726163696F31
:1064A0006E2058595A20636F7272656374612E2092
:1064B0004C6120696E636C696E6163696F6E2073F5
:1064C0006520636F72726567697261206175746FB0
:1064D0006D61746963616D656E74652E0043616CF6
:1064E000696272617A696F6E2058595A20636F72BF
:1064F00072657474612E204C6120646973746F72CC
:1065000073696F6E6520766572726127206175749C
:106510006F6D61746963616D656E746520636F6D25
:1065200070656E736174612E004B616C696272619B
:1065300063652058595A207620706F7261646B75BC
:106540002E205A6B6F73656E6920627564652061D9
:1065500075746F6D617469636B79207679726F768B
:106560006E616E6F20707269207469736B752E0096
:1065700058595A2063616C6962726174696F6E2048
:10658000616C6C2072696768742E20536B6577208C
:1065900077696C6C20626520636F727265637465E5
:1065A00064206175746F6D61746963616C6C792EC0
:1065B0000058595A2D4B616C696272696572756E2B
:1065C00067206665686C67657363686C6167656E94
:1065D0002E20426574742D4B616C6962726965721C
:1065E00070756E6B74206E6963687420676566757C
:1065F0006E64656E2E0043616C6962726163696FDF
:106600006E2058595A2066616C6C6164612E20506E
:10661000756E746F732064652063616C696272616A
:1066200063696F6E20656E206865617462656420C1
:106630006E6F20656E636F6E747261646F732E008F
:1066400043616C696272617A696F6E652058595A4C
:106650002066616C6C6974612E20496C2070756EC7
:10666000746F2064692063616C696272617A696F1A
:106670006E652073756C206C6574746F206E6F6E20
:1066800020652720737461746F2074726F76617453
:106690006F2E004B616C6962726163652058595AB4
:1066A0002073656C68616C612E204B616C6962724D
:1066B00061636E6920626F6420706F646C6F7A6BC7
:1066C00079206E656E616C657A656E2E0058595A38
:1066D0002063616C6962726174696F6E20666169C2
:1066E0006C65642E204265642063616C696272612E
:1066F00074696F6E20706F696E7420776173206E9D
:106700006F7420666F756E642E0058595A2D4B6158
:106710006C696272696572756E67206F6B2E2058A6
:106720002F592D41636873656E2073696E64207301
:10673000656E6B7265636874207A7565696E616EEB
:106740006465722E20476C7565636B77756E736335
:1067500068210043616C6962726163696F6E2058E1
:10676000595A206F6B2E20456A657320582F592087
:1067700070657270656E646963756C617265732EA5
:1067800020456E686F72616275656E6121004361BC
:106790006C696272617A696F6E652058595A204F30
:1067A0004B2E20476C69206173736920582F592044
:1067B000736F6E6F2070657270656E6469636F6C65
:1067C0006172692E20436F6D706C696D656E7469BE
:1067D00021004B616C6962726163652058595A20CF
:1067E0007620706F7261646B752E20582F59206F60
:1067F0007379206A736F75206B6F6C6D652E2047FF
:10680000726174756C756A69210058595A20636108
:106810006C6962726174696F6E206F6B2E20582FE5
:1068200059206178657320617265207065727065AA
:106830006E646963756C61722E20436F6E6772615E
:1068400074756C6174696F6E73210058595A2D4BC1
:10685000616C696272696572756E67206665686CE5
:1068600067657363686C6167656E2E204269747436
:1068700065207363686175656E2053696520696E74
:10688000206461732048616E64627563682E004302
:10689000616C6962726163696F6E2058595A206633
:1068A000616C6C6164612E20436F6E73756C7461F2
:1068B00020656C206D616E75616C20706F72206652
:1068C00061766F722E0043616C696272617A696FE2
:1068D0006E652058595A2066616C6C6974612E206F
:1068E000536920707265676120646920636F6E73FD
:1068F000756C7461726520696C206D616E75616C78
:10690000652E004B616C6962726163652058595A4B
:106910002073656C68616C612E204E61686C6564E3
:106920006E65746520646F206D616E75616C752E87
:106930000058595A2063616C6962726174696F6EA4
:10694000206661696C65642E20506C6561736520FA
:10695000636F6E73756C7420746865206D616E75FD
:10696000616C2E0058595A2D4B616C6962726965D1
:1069700072756E67206665686C67657363686C61C5
:1069800067656E2E204C696E6B657220766F72643F
:1069900065726572204B616C6962726965727075AF
:1069A0006E6B7420697374207A7520776569742022
:1069B000766F726E652E0043616C69627261636905
:1069C0006F6E2058595A2066616C6C6164612E208C
:1069D00050756E746F2066726F6E74616C20697A88
:1069E0007175696572646F206E6F20616C63616E92
:1069F0007A61626C652E0043616C696272617A69CA
:106A00006F6E652058595A2066616C6C6974612EEE
:106A10002050756E746F20616E746572696F726557
:106A20002073696E697374726F206E6F6E2072616D
:106A3000676769756E676962696C652E004B616C8A
:106A40006962726163652058595A2073656C686188
:106A50006C612E204C65767920707265646E6920B9
:106A6000626F64206D6F63207670726564752E208E
:106A700053726F766E656A7465207469736B6172A8
:106A80006E752E0058595A2063616C696272617488
:106A9000696F6E206661696C65642E204C65667452
:106AA0002066726F6E742063616C696272617469D2
:106AB0006F6E20706F696E74206E6F7420726561E6
:106AC000636861626C652E0058595A2D4B616C6980
:106AD0006272696572756E67206665686C6765735A
:106AE00063686C6167656E2E20566F7264657265AF
:106AF000204B616C69627269657270756E6B74654A
:106B00002073696E64207A75207765697420766FCA
:106B1000726E652E0043616C6962726163696F6EAB
:106B20002058595A2066616C6C6164612E20507542
:106B30006E746F732066726F6E74616C6573206E15
:106B40006F20616C63616E7A61626C65732E0043C5
:106B5000616C696272617A696F6E652058595A205A
:106B600066616C6C6974612E2050756E7469206169
:106B70006E746572696F7269206E6F6E20726167E4
:106B80006769756E676962696C692E004B616C6933
:106B900062726163652058595A2073656C68616C34
:106BA000612E20507265646E69206B616C6962723F
:106BB00061636E6920626F6479206D6F6320767007
:106BC000726564752E2053726F766E656A746520E7
:106BD0007469736B61726E752E0058595A20636127
:106BE0006C6962726174696F6E206661696C65645C
:106BF0002E2046726F6E742063616C6962726174DC
:106C0000696F6E20706F696E7473206E6F7420727E
:106C10006561636861626C652E005A2D4B616C6919
:106C20006272696572756E67206665686C67657308
:106C300063686C672E2053656E736F72206E696394
:106C4000687420616E67657363686C6F7373656EDB
:106C50002E205761727465206175662052657365D8
:106C6000742E004E6976656C6163696F6E20666193
:106C70006C6C6164612E2053656E736F7220646565
:106C800073636F6E65637461646F206F206361620C
:106C90006C65732064616E61646F732E2045737040
:106CA0006572616E646F2072657365742E004C6945
:106CB00076656C6C616D656E746F206C6574746F55
:106CC0002066616C6C69746F2E2053656E736F72F1
:106CD0006520646973636F6E2E206F204361766F49
:106CE0002044616E6E2E20496E206174746573615C
:106CF0002064692072657365742E004B616C696253
:106D000072616365205A2073656C68616C612E2026
:106D100053656E736F72206A65206F64706F6A6569
:106D20006E79206E65626F20707265727573656E24
:106D300079206B6162656C2E2043656B616D206EFE
:106D4000612072657365742E00426564206C6576FF
:106D5000656C696E67206661696C65642E20536599
:106D60006E736F7220646973636F6E6E65637465B2
:106D700064206F72206361626C652062726F6B6564
:106D80006E2E2057616974696E6720666F7220727B
:106D9000657365742E005A2D4B616C2E20666568F4
:106DA0006C67657363686C672E2053656E736F72D2
:106DB000206E696368742061757367656C6F6573B5
:106DC000742E205363686D75747A69676520447505
:106DD0006573653F20576172746520617566205246
:106DE00065736574004E6976656C6163696F6E20CA
:106DF00066616C6C6164612E2053656E736F7220E6
:106E00006E6F2066756E63696F6E612E20457363C9
:106E10006F6D62726F7320656E206E6F7A7A6C652B
:106E20003F204573706572616E646F207265736593
:106E3000742E004C6976656C6C616D656E746F20A4
:106E40006C6574746F2066616C6C69746F2E4E6F24
:106E50005269737053656E736F7220526573696403
:106E60007569207375207567656C6C6F3F20496E7E
:106E70002061747465736120646920726573657440
:106E80002E004B616C696272616365205A207365E4
:106E90006C68616C612E2053656E736F72206E6535
:106EA0007365706E756C2E205A6E656369737465B8
:106EB0006E6120747279736B613F2043656B616D05
:106EC000206E612072657365742E00426564206CCB
:106ED0006576656C696E67206661696C65642E20F5
:106EE00053656E736F72206469646E742074726986
:106EF000676765722E20446562726973206F6E2029
:106F00006E6F7A7A6C653F2057616974696E67208D
:106F1000666F722072657365742E005A2D4B616C1A
:106F2000696272696572756E67206665686C67650F
:106F30007363686C672E2053656E736F72207A7569
:106F400020686F63682061757367656C6F65737423
:106F50002E205761727465206175662052657365D5
:106F6000742E004E6976656C6163696F6E20666190
:106F70006C6C6164612E2053656E736F7220667550
:106F80006E63696F6E612064656D61736961646FC2
:106F90002074656D7072616E6F2E2045737065721E
:106FA000616E646F2072657365742E004C6976653E
:106FB0006C6C616D656E746F206C6574746F2066A7
:106FC000616C6C69746F2E526973702073656E7397
:106FD0006F72652074726F70706F20707265737459
:106FE0006F496E20617474657361206469207265F5
:106FF0007365742E004B616C696272616365205A1F
:107000002073656C68616C612E2053656E736F72BE
:10701000207365706E756C207072696C6973207670
:1070200079736F6B6F2E2043656B616D206E6120ED
:1070300072657365742E00426564206C6576656CBC
:10704000696E67206661696C65642E2053656E7396
:107050006F722074726967676572656420746F6F00
:1070600020686967682E2057616974696E672066B9
:107070006F722072657365742E00426574742061AE
:107080007566776165726D656E0043616C656E74DF
:10709000616E646F20426173650052697363616C55
:1070A000642E206C6574746F005A61687269766131
:1070B0006E69206265640042656420486561746998
:1070C0006E670042657474204F4B00426173652007
:1070D0007072657061726164610050696174746F8F
:1070E00020666174746F2E00426564204F4B2E0041
:1070F00042656420646F6E65005265636874732036
:107100002020205B756D5D004465726563686120B9
:1071100020205B756D5D00446573747261202020D2
:10712000205B756D5D0056707261766F205B756DCA
:107130005D00526967687420736964655B756D5D95
:1071400000527565636B7365747A656E0052657382
:1071500065740048696E74656E202020205B756D33
:107160005D00547261736572612020205B756D5DF6
:1071700000526574726F20202020205B756D5D00C9
:10718000567A61647520205B756D5D005265617291
:107190002073696465205B756D5D004265747420C1
:1071A0006C6576656C204B6F7272656B7400436F13
:1071B00072722E206465206C612063616D610043F2
:1071C0006F7272657A2E206C69762E6C6574746F9E
:1071D000004B6F72656B636520706F646C6F7A6BC8
:1071E0007900426564206C6576656C20636F72720D
:1071F000656374004C696E6B7320202020205B75E2
:107200006D5D00497A71756965726461205B756DA9
:107210005D0053696E697374726120205B756D5DEA
:1072200000566C65766F20205B756D5D004C656661
:10723000742073696465205B756D5D00566F726EB6
:107240006520202020205B756D5D0046726F6E7496
:10725000616C2020205B756D5D0046726F6E7465F9
:10726000202020205B756D5D00567072656475206E
:107270005B756D5D0046726F6E7420736964655B4B
:10728000756D5D0042657474004865617462656483
:10729000004C6574746F004265640044657220415F
:1072A000627374616E64207A7769736368656E20B7
:1072B00064657220537069747A6520646572204435
:1072C0007565736520756E6420646572204265740F
:1072D0007420697374206E6F6368206E69636874CC
:1072E0002065696E67657374656C6C742E204269E5
:1072F00074746520666F6C67656E205369652064E1
:10730000656D2048616E64627563682C2046697201
:1073100073742073746570732C2073656374696F64
:107320006E204669727374206C61796572206361A6
:107330006C6962726174696F6E2E00446973746166
:107340006E63696120656E747265206C6120707572
:107350006E74612064656C206E6F7A7A6C6520793A
:10736000206C61207375706572666963696520645D
:1073700065206C6120686561746265642061756E6A
:10738000206E6F2066696A6164612E20506F7220E2
:107390006661766F72207369676120656C206D612C
:1073A0006E75616C2C206361706974756C6F20461A
:1073B000697273742073746570732C2046697273DC
:1073C00074206C617965722063616C6962726174AA
:1073D000696F6E2E0044697374616E7A61207472F5
:1073E00061206C612070756E74612064656C6C271F
:1073F0007567656C6C6F2065206C612073757065B6
:107400007266696369652064656C206C6574746F6D
:10741000206E6F6E20616E636F726120696D706F98
:107420007374612E205369207072656761206469EE
:10743000207365677569726520696C206D616E7572
:10744000616C652C2063617069746F6C6F20466994
:107450007273742073746570732C2073657A696F0E
:107460006E65204669727374206C61796572206361
:10747000616C6962726174696F6E2E004E656E692F
:10748000207A6B616C6962726F76616E6120767AC8
:1074900064616C656E6F737420747279736B79209C
:1074A0006F64207469736B6F766520706F646C6FA6
:1074B0007A6B792E20506F73747570756A746520BD
:1074C00070726F73696D20706F646C65206D616E92
:1074D00075616C752C206B617069746F6C61205ADA
:1074E0006163696E616D652C206F6473746176658C
:1074F00063204E6173746176656E69207072766E7A
:1075000069207672737476792E0044697374616EA3
:107510006365206265747765656E20746970206F9D
:107520006620746865206E6F7A7A6C6520616E647F
:107530002074686520626564207375726661636596
:1075400020686173206E6F74206265656E207365BC
:1075500074207965742E20506C6561736520666FA8
:107560006C6C6F7720746865206D616E75616C2C32
:107570002063686170746572204669727374207349
:10758000746570732C2073656374696F6E2046692F
:10759000727374206C617965722063616C696272C8
:1075A0006174696F6E2E005A2065696E7374656C24
:1075B0006C656E004D6963726F7061736F20456A10
:1075C00065205A00436F6D70656E73617A696F6EE6
:1075D00065205A00446F6C6164656E69206F737931
:1075E000205A004C6976652061646A757374205A6C
:1075F0000041646A757374696E67205A0053746140
:107600007274706F736974696F6E004C6C6576612B
:107610007220616C206F726967656E0054726F76BC
:1076200061206F726967696E65004175746F2068CB
:107630006F6D6500207C20417574686F723A200080
:10764000416C6C6500546F646F7300547574746999
:107650000056736500416C6C004163746976652067
:1076600045787472756465723A20004D133D132895
:1076700013151300136113691371137A138213C75F
:1076800013B2139F13C7138A13E913E513E213DF31
:1076900013DC13ED13F513311420140E143114FD03
:1076A00013D114B714941473144214F015B8157A46
:1076B000154015EF14D016B01689165D162E167BE0
:1076C000181A18B0175417F3160E1C631B841ACB24
:1076D00019DE18E21D9F1D641D0F1DC21C931F3A69
:1076E0001FE41E951E2F1E7A210E21A7204720DAA7
:1076F0001F3023E4228F224422D921B42471241282
:1077000024D22381235625422524250F25F124D078
:107710002676261926C7256A257F283028D6278170
:10772000271827692945291429EC28C928F229DDB9
:1077300029BE29A3298929762A672A4E2A322A06B0
:107740002A712B432B0E2BD42A932A642D072D8DBF
:107750002C2F2C9F2BC42DCB2D0C2E022EF32DE77E
:107760002DDB2D602E4E2E3C2E2A2E182EA72EA756
:107770002E952E832E712E062FF22EDF2ECC2EB8B4
:107780002E5E2F4D2F3B2F2A2F182FB82FA62F9468
:107790002F812F6E2FCB2F0330FD2FF62FEE2FDEF4
:1077A0002F1C301C301C301C300830403040304022
:1077B0003040302E3091308130713061305130E5C1
:1077C00030D430C330B230A130DE31A33168312D36
:1077D00031F6306A32553240322B321632AA32A29A
:1077E0003296328A327F32C632BE32C632B632C6A4
:1077F000320D33FF32F032DE32CE32353335332ABA
:1078000033233318333F335333AF33A1338F3380B4
:10781000336E330434F233E333D233C2335134435F
:1078200034323422341534A3349634853472345FC0
:1078300034E934DC34D034C134B434F6344D354416
:10784000353B353135213553359135823573359199
:10785000356335E535D335C135AF359E353F362DEA
:10786000361B360936F7359636853675366336510A
:1078700036D436C536B536D436A53629371737034C
:1078800037F136E1366D376337563748373A37BA0E
:1078900037AB379A3788377637F837F837E937D93B
:1078A00037C7373E382F38233818380A38673867D3
:1078B000385B3867384D38B638A7389A3888387406
:1078C00038CB38CB38C438CB38CB38EA38EA38D85C
:1078D00038D138EA3840392F391A390839FC38900C
:1078E000397E396D395E394939ED39D839C339B204
:1078F00039A239313A313A1F3A0F3AFE39793A7999
:107900003A673A553A423AB13AB13AA33A953A8986
:107910003ACF3ACF3AC53ABA3ACF3A223B0D3BF882
:107920003AE93AD73A773B653B553B463B333BCD4B
:107930003BBB3BAB3B9C3B893B233C113C013CF2BA
:107940003BDF3B743C623C523C423C353CCE3CBC51
:107950003CA93C9B3C863C253D133D043DF43CE06A
:107960003C733D613D533D493D373DAA3DAA3D9B9A
:107970003D933D853DB73DC33DEC3DEC3DE33DDAF8
:107980003DC83DFE3D103E233E623E543E493E38DA
:107990003E2B3E6F3E813E953EDF3ED13EC53EB31F
:1079A0003EA53EED3EFA3E083F163F2C3F373F6472
:1079B0003F5D3F553F643F4D3FB33FA23F903F7D0A
:1079C0003F6B3F0840F93FE93FD43FC23F4E404341
:1079D000403340224017405B4064408C40AE40D46E
:1079E00040C340D440D440D440F740E640F740F78D
:1079F00040F740144109411441144114416241527D
:107A00004142412F412041B341A541954181416F00
:107A100041C1411B420642F241E941D641784264EC
:107A20004254423F422E42B942AF42A34297428C57
:107A300042C142FF42F042E842D642C942AC4386CC
:107A4000435A4330430B4337441E440544E643CC7A
:107A5000434F446644CB44BB44AC449B448B448278
:107A6000455C452D45FB44D944EB45D745CE45BA49
:107A700045AF454846364624461146FF459A468C52
:107A8000467B466B465A46EC46DC46CD46BC46AA8B
:107A9000464F49C8483A488E47F846E549E8491DE7
:107AA0004A1D4A0B4AFC49EC49614A524A474A3549
:107AB0004A264A804A794A724A804A6C4AD34AC066
:107AC0004AAE4A9A4A874A284B174B074BF44AE773
:107AD0004A404B3D4B404B404B384B924B7D4B6D9E
:107AE0004B584B434B224C074CDF4BC44BA24B66CD
:107AF0004C5B4C534C4B4C424C914C864C7E4C76E0
:107B00004C6D4CBC4CB14CA94CA14C984CDB4CDBA3
:107B10004CCB4CC34CDB4C144D074DFC4CF14CE4AE
:107B20004C434D434D314D434D1E4D854D7B4D6E68
:107B30004D624D554DA94DA44D9E4D984D914D6BA7
:107B40004E424E064EDD4DAF4DC84EB84EA84EC803
:107B50004E9B4E104F014FF14EE24ED74E154F2C1B
:107B60004F434F5A4FD04FB94FA24F8B4F734FE6F1
:107B70004FC350DA50F1504A51375128511B510828
:107B80005199518951785166515751EF51DC51CB80
:107B900051B651A7513A522C521B520B5200525F10
:107BA0005259524F525F524852A4529752865274C1
:107BB000526552D552CD52C452BC52B452095309E7
:107BC000530053EB52DD5212536D535D534A5335FC
:107BD0005323537D5389539553BB53B653B053AA84
:107BE00053A353545430540954E253C153A7549BE4
:107BF000548E5481547454F154E454D454C554B53F
:107C000054325525551B55105502558155735561F4
:107C1000554C553E55C355B955A8559A558F55CB1A
:107C200055DD55EF55C2574F57DD567756FE554F28
:107C300058485841583B5830589B58885877586591
:107C4000585458C758C258BC58B658AF58525933F0
:107C5000590E59E858CD5896598D597F59725996F1
:107C600059A159B359155A055AF059D659C65969E7
:107C70005A585A485A365A255AB55AA65A975A87C0
:107C80005A795ABF5ADD5ADD5AD35ACA5ADD5AE6D2
:107C90005AF65A6C5B965BC05BDE5B115C305C4AEB
:107CA0005C805C795C715C805C695C875C955C9AEB
:107CB0005CA45CE05CE05CD15CC75CB35C245D15FB
:107CC0005D045DF55CE95C475D405D3B5D475D35AE
:107CD0005D755D665D5E5D575D4D5D7D5D8F5DA132
:107CE0005DE65DDB5DCB5DB85DAC5D1E5E155E0B7C
:107CF0005E035EF95D275E845E725E5D5E4C5E379C
:107D00005ED75EC85EB75EA75E955E1D5F135F06B9
:107D10005FF65EE75E705F5E5F4F5F3D5F2B5F8289
:107D20005FBB5FAF5FA55F9C5F905FE95FD75FE977
:107D30005FE95FC55F3260246018600C60FB5F40E4
:107D400060516070613C61F260AD606160BA627FF9
:107D5000623E62FF61B9610E64D1638F633A63FF73
:107D60006270652965DD6496645164CD66936640F2
:107D700066F665B1650A68D2678E6753670A673130
:107D8000690369C6688F684B68846A3D6AF769B79A
:107D9000696469DA6B8C6B4F6B156BC86A496DFB54
:107DA0006CAE6C636C1A6CCB6E826E336EE56D9646
:107DB0006D3770F56FAC6F636F1B6FB770A9709AFA
:107DC000708A707A70F070E870DA70CB70C37032BD
:107DD00071267117710871F9704D714D714D714DAA
:107DE0007141718C718071717162715371E271D1E5
:107DF00071BF71AE719B712D72217212720372F498
:107E000071757269725A724B723C72977297729165
:107E100072897284720A757C74D5733B739B72E3AA
:107E200075D475C475B475A775F1752A762A761C54
:107E3000760B76FD753476557651764B76457640E1
:107E4000765976457872656D65207370616E206F26
:107E50006620746865205A2076616C756573210010
:107E600043616C63756C6174696F6E206F6620741A
:107E70006865206D616368696E6520736B65772046
:107E8000616E64206F6666736574206661696C65F7
:107E9000642E00203C20005741524E494E473A2064
:107EA00046726F6E7420706F696E74206E6F7420EE
:107EB000726561636861626C652E205920636F6F23
:107EC0007264696E6174653A000049746572617428
:107ED000696F6E3A2000496E76616C696420626554
:107EE0006420636F7272656374696F6E206D617474
:107EF0007269782E20526573657474696E67207498
:107F00006F206964656E746974792E00496E7661BC
:107F10006C69642062656420636F72726563746962
:107F20006F6E206D61747269782E20582F59206110
:107F300078657320617265206661722066726F6D6C
:107F4000206265696E672070657270656E64696332
:107F5000756C61722E00496E76616C696420626591
:107F60006420636F7272656374696F6E206D6174F3
:107F70007269782E205368696674206F7574206F5B
:107F8000662072616E67652E005A65726F20706F91
:107F9000696E7420636F7272656374696F6E3A0004
:107FA000496E76616C69642062656420636F7272E9
:107FB000656374696F6E206D61747269782E204CF0
:107FC000656E677468206F66207468652059207636
:107FD0006563746F72206F7574206F662072616EB6
:107FE00067652E005920766563746F72206C656E2C
:107FF0006774683A00496E76616C696420626564F2
:1080000020636F7272656374696F6E206D61747244
:1080100069782E204C656E677468206F66207468DE
:1080200065205820766563746F72206F7574206FB9
:10803000662072616E67652E005820766563746FE6
:1080400072206C656E6774683A00556E6465666987
:108050006E65642062656420636F72726563746923
:108060006F6E206D61747269782E0000004041FFD0
:10807000FFBF4000005C43FFFFBF4000005C4300C7
:10808000004643000040410000464300004041FFDD
:10809000FFBF400000E442FFFFBF4000005743FF26
:1080A000FFBF40000057430000CC420000E4420004
:1080B00000CC42000040410000CC420000404100A2
:1080C0000046430000E442000046430000574300DE
:1080D0000046435A00205A3A00590020593A0058A5
:1080E0000020583A0024F4D43050C38E20C2A2405D
:1080F00017828B7011127A910D816CD90AA861E1F7
:1081000008C7586607615143061E4B5D05C145A768
:10811000041A411104093D9803713931034036DBDB
:108120000265339102D4305402802E1D02632CEE7E
:1081300001752AC501B028A001102781018F25648F
:10814000012B244B01E0223401AC211F018D200DB5
:1081500001801FFC00841EED00971DDF00B81CD2BB
:1081600000E61BC600201BBC00641AB200B219A8AE
:10817000000A19A0006A189900D117910040178BC6
:1081800000B516840031167E00B31579003A1573D8
:1081900000C7146F0058146A00EE1366008813635A
:1081A0000025135E00C7125B006C125700151254B5
:1081B00000C111510070114F0021114B00D6104920
:1081C000008D1047004610440002104200C00F40CE
:1081D00000800F3E00420F3C00060F3B00CB0E38E4
:1081E00000930E37005C0E3500270E3400F30D327D
:1081F00000C10D3100900D3000600D2E00320D2DAC
:1082000000050D2C00D90C2B00AE0C2900850C2983
:10821000005C0C2700350C27000E0C2600E80B2410
:1082200000C40B2400A00B23007D0B23005A0B215C
:1082300000390B2100180B2000F80A1F00D90A1E74
:1082400000BB0A1E009D0A1D00800A1D00630A1C57
:1082500000470A1B002C0A1B00110A1A00F7091A12
:1082600000DD091900C4091900AB091900920917AA
:10827000007B091800630917004C0916003609161F
:1082800000200916000A091500F5081500E0081479
:1082900000CC081400B8081400A4081400900813B7
:1082A000007D0812006B08130058081200460812DF
:1082B00000340811002308110012081100010811F0
:1082C00000F0071000E0071000D0071000C00710F2
:1082D00000B0070F00A107100091070E0083070FE1
:1082E0000074070F0065070E0057070E0049070EC0
:1082F000003B070D002E070E0020070D0013070D91
:108300000006070D00F9060C00ED060D00E0060C56
:1083100000D4060C00C8060C00BC060C00B0060C0D
:1083200000A4060B0099060C008D060B0082060BBC
:108330000077060B006C060B0061060A0057060B5F
:10834000004C060A0042060A0038060A002E060AF9
:108350000024060A001A060A001006090007060A89
:1083600000FD050900F4050900EB050900E2050917
:1083700000D9050900D0050900C7050900BE050997
:1083800000B5050800AD050800A50509009C050815
:1083900000940508008C050800840508007C050889
:1083A00000740508006C050700650508005D0507F9
:1083B00000560508004E0507004705070040050860
:1083C0000038050700310507002A050700230507C7
:1083D000001C050600160507000F05070008050626
:1083E0000002050700FB040600F5040700EE040682
:1083F00000E8040600E2040700DB040600D50406DA
:1084000000CF040600C9040600C3040600BD04062C
:1084100000B7040600B1040500AC040600A604067B
:1084200000A00405009B04060095040500900406C6
:10843000008A04050085040500800406007A04050E
:108440000075040500700405006B04050066040552
:1084500000610405005C0405005704050052040592
:10846000004D04050048040500430405003E0404D3
:10847000003A04050035040500300404002C04050E
:108480000027040400230405001E0404001A040449
:108490000016040500110404000D0404000904057D
:1084A000000404040000040400FC030400F80304B6
:1084B00000F4030400F0030400EC030400E80304E8
:1084C00000E4030400E0030400DC030400D8030418
:1084D00000D4030400D0030400CC030400C8030349
:1084E00000C503030024F404D9201BC40C5C0E98BF
:1084F00004C4095F0265077101F405F900FB04B3C8
:108500000048048700C10369005803550003034570
:1085100000BE023A008402310053022A00290225DB
:108520000004022000E4011C00C8011900AF01177B
:108530000098011400840113007101100061011002
:108540000051010E0043010D0036010B002B010B01
:108550000020010B00150109000C010900030108AE
:1085600000FB000800F3000800EB000700E4000631
:1085700000DE000600D8000600D2000600CC000590
:1085800000C7000500C2000500BD000400B90004DA
:1085900000B5000400B1000400AD000400A900040F
:1085A00000A5000300A20003009F0004009B00033D
:1085B0000098000300950002009300030090000360
:1085C000008D0002008B000300880002008600027C
:1085D0000084000300810002007F0002007D000291
:1085E000007B0002007900020077000100760002A3
:1085F000007400020072000100710002006F0002AE
:10860000006D0001006C0002006A000100690002B8
:1086100000670001006600010065000100640002BF
:10862000006200010061000100600001005F0002C3
:10863000005D0001005C0001005B0001005A0001C8
:1086400000590001005800010057000100560001C8
:1086500000550001005400010053000000530001C8
:10866000005200010051000100500001004F0001C4
:10867000004E0000004E0001004D0001004C0001C2
:10868000004B0000004B0001004A000100490001BE
:1086900000480000004800010047000100460000BB
:1086A00000460001004500000045000100440001B3
:1086B00000430000004300010042000000420001AE
:1086C000004100000041000100400001003F0000A7
:1086D000003F0001003E0000003E0001003D0000A0
:1086E000003D0001003C0000003C0000003C000197
:1086F000003B0000003B0001003A0000003A00018E
:108700000039000000390001003800000038000086
:10871000003800010037000000370001003600007B
:108720000036000000360001003500000035000072
:108730000035000100340000003400000034000166
:10874000003300000033000000330001003200005D
:108750000032000000320001003100000031000052
:108760000031000100300000003000000030000146
:10877000002F0000002F0000002F0000002F00013C
:10878000002E0000002E0000002E0001002D000031
:10879000002D0000002D0000002D0001002C000025
:1087A000002C0000002C0000002C0001002B000019
:1087B000002B0000002B0000002B0001002A00000D
:1087C000002A0000002A0000002A00010029000001
:1087D00000290000002900000029000000290001F4
:1087E00000280000002800000028000000280000E9
:1087F00000280001002700000027000000270000DB
:1088000000270000002700010026000000260000CD
:1088100000260000002600000026000100250000C0
:1088200000250000002500000025000000250000B4
:1088300000250001002400000024000000240000A6
:108840000024000000240001002300000023000099
:10885000002300000023000000230000002300008C
:10886000002300010022000000220000002200007E
:108870000022000000220000002200010021000070
:108880000021000000210000002100000021000064
:108890000021000000210001002000000020000055
:1088A0000020000000200000002000000020000048
:1088B0000020000000200001001F0000001F000039
:1088C000001F0000001F0000001F0000001F00002C
:1088D000001F0001001E0000001E0000001E00001E
:1088E000001E0000004572723A204D494E54454D1D
:1088F00050204245440054656D7065726174757214
:1089000065206865617465642062656420737769B9
:108910007463686564206F66662E204D494E544529
:108920004D50207472696767657265642021004547
:1089300072723A204D415854454D502042454400F2
:1089400054656D70657261747572652068656174D7
:108950006564206265642073776974636865642068
:108960006F66662E204D415854454D5020747269F3
:108970006767657265642021004572723A204D492F
:108980004E54454D50003A204578747275646572B6
:10899000207377697463686564206F66662E204D66
:1089A000494E54454D50207472696767657265641D
:1089B0002021004572723A204D415854454D5000D7
:1089C0003A204578747275646572207377697463B0
:1089D000686564206F66662E204D415854454D50A1
:1089E0002074726967676572656420210020484FB2
:1089F00054454E4420544845524D414C2052554E0A
:108A0000415741590020484541544245442054486B
:108A100045524D414C2052554E4157415900544802
:108A200045524D414C2052554E4157415900424507
:108A30004420544845524D414C2052554E415741D7
:108A4000590020544845524D414C2052554E4157F3
:108A500041592028205052454845415420484F5400
:108A6000454E44290020544845524D414C20525512
:108A70004E415741592028205052454845415420E5
:108A800048454154424544290050524548454154C7
:108A9000204552524F5200424544205052454845CD
:108AA0004154204552524F52004572723A20505262
:108AB000494E542046414E204552524F5200455295
:108AC000524F523A205072696E742066616E207364
:108AD00070656564206973206C6F776572207468B7
:108AE000656E206578706563746564004572723ADE
:108AF00020455854522E2046414E204552524F5246
:108B0000004552524F523A2045787472756465722E
:108B10002066616E207370656564206973206C6FD8
:108B2000776572207468656E20657870656374651A
:108B30006400202D20496E76616C6964206578742C
:108B40007275646572206E756D62657220210050C9
:108B50004944204175746F74756E652066696E694D
:108B600073686564212050757420746865206C6199
:108B70007374204B702C204B6920616E64204B6411
:108B800020636F6E7374616E74732066726F6D20F4
:108B900061626F766520696E746F20436F6E6669DF
:108BA0006775726174696F6E2E6800504944204188
:108BB00075746F74756E65206661696C65642120DB
:108BC00074696D656F75740020403A006F6B2054B6
:108BD0003A006F6B20423A00504944204175746F4F
:108BE00074756E65206661696C6564212054656DDD
:108BF000706572617475726520746F6F2068696743
:108C00006800204B643A2000204B693A2000204B3A
:108C1000703A200020436C617373696320504944AB
:108C200020002054753A2000204B753A2000206D1A
:108C300061783A2000206D696E3A200020643A2065
:108C40000020626961733A200010137D00201578BE
:108C50000060177300C0196E00401C6900E01E64BC
:108C60000080215F0040245A00F0265500902950D2
:108C700000202C4B00802E4600C0304100D0323CFA
:108C800000B034370050363200C0372D000039288C
:108C900000103A2300F03A1E00B03B1900503C147B
:108CA00000D03C0F00303D0A00803D0500C03D0073
:108CB00000F03DFBFF103EF6FF303EF1FF403EEC82
:108CC000FF503EE7FF603EE2FF703EDDFF703ED8A2
:108CD000FF1000C90210012C01400122017001188F
:108CE00001B0010E01F00104015002FA00B002F0DF
:108CF000003003E600D003DC009004D2007005C809
:108D000000A006BE000008B400B009AA00D00BA065
:108D100000600E960060118C00001582002019780A
:108D200000C01D6E00A0226400B0275A00902C5095
:108D30000000314600E0343C0010383200903A2800
:108D400000603C1E00A03D1400803E0A00203F0051
:108D50000070012C0190012701B0012201C0011D0A
:108D600001F00118011002130130020E0160020926
:108D70000190020401C002FF000003FA004003F565
:108D8000008003F000D003EB002004E6007004E153
:108D900000E004DC004005D700C005D2004006CD4D
:108DA00000D006C8008007C3003008BE00F008B934
:108DB00000C009B400B00AAF00B00BAA00D00CA5E7
:108DC00000000EA000500F9B00C0109600501291A2
:108DD0000000148C00C0158700B0178200B0197D08
:108DE00000D01B7800001E730040206E00902269A6
:108DF00000F024640040275F0090295A00E02B55C2
:108E000000102E500020304B0010324600E033415D
:108E10000090353C001037370070383200A0392DF3
:108E200000B03A2800A03B2300603C1E00103D1912
:108E300000903D1400103E0F00703E0A00C03E0539
:108E400000003F0000544D432044524956455220F3
:108E50004F56455254454D502000436F6E74696E15
:108E60007565207769746820616E6F74686572201B
:108E7000626F7764656E3F0053746174653A2000D9
:108E8000473736004D3435205A004D3435004738C9
:108E9000300020003E003E0020003E003E003E002C
:108EA0003E0020003E003E00200000002D2D2D2D14
:108EB0002D2D2D2D2D2D2D2D2D2D2D2D2D2D2D2DE2
:108EC000004E2F41004E2F41006D6D00004D373098
:108ED00031004D37303200496E76616C6964205044
:108EE00049442063616C2E20726573756C74732E17
:108EF000204E6F742073746F72656420746F204508
:108F00004550524F4D2E004D353030004731205ADC
:108F10003135204631353030004739310047312076
:108F200058353020593139302045302046373030DF
:108F30003000473930004D373032004D3730322065
:108F400043004D3730322055004D37303200473125
:108F5000205A31352046313530300047393100470D
:108F600031205835302059313930204530204637AE
:108F7000303030004D383300473930004D38340040
:108F80004D313034205330004D38340047312058B3
:108F900031302059313830204634303030004731BC
:108FA000205A31302046313330302E303030004DB1
:108FB000313430205330004D313034205330004DA7
:108FC00031303700473120452D302E3037353030A5
:108FD0002046323130302E303030303000473120B2
:108FE000583530205935352045332E363237373312
:108FF0000047312058323030205935352045302E49
:109000003439333836004731205832303020593720
:10901000352045332E363237373300473120583527
:1090200030205937352045302E3439333836004713
:109030003120583530205939352045332E363237D6
:1090400037330047312058323030205939352045E8
:10905000302E343933383600473120583230302002
:10906000593131352045332E3632373733004731C9
:109070002058353020593131352045302E343933A0
:1090800038360047312058353020593133352045A6
:10909000332E3632373733004731205832303020C4
:1090A000593133352045302E36363137340047318B
:1090B000205832303020593135352045322E363265
:1090C000373733004731205831303020593135356A
:1090D0002045320047312058373520593135352069
:1090E00045322E3500473120463130383000473187
:1090F000205835302059313535004731204634303D
:109100003030004D32303420533130303000473170
:10911000205A302E3135302046373230302E303024
:109120003000473120452D312E353030303020464B
:10913000323130302E3030303030004D383300474F
:10914000393000473231004739322045302E300067
:10915000473120583130302E30204531322E3520E5
:1091600046313030302E30004731205836302E30E6
:109170002045392E302046313030302E30004739EE
:10918000322045302E300047323800473837004D06
:109190003130392053323130004D313930205335A0
:1091A00035004D31343020533535004D31303420C9
:1091B00053323130004D31303700473930004731BC
:1091C000204531004D3832004731204531004D38BF
:1091D00033004D31303620532564004D323230207B
:1091E000532564003A200020202020202020202029
:1091F0002020202020202020202000203A20002095
:10920000202020202020202020202020202020205E
:10921000202020002020202020202020202020206E
:1092200020002573002020002D2D3A2D2D00200038
:10923000200020004C002020002046002D2D2D0075
:109240003E555342005344002D2D00252020202060
:1092500020002020002020000120002020202D2D93
:109260002D200020205A002020000120004D363003
:109270003000464C4558202D20203233302F3530D9
:109280000050502020202D20203235342F31303016
:109290000048495053202D20203232302F313030B9
:1092A0000050455420202D20203234302F393000FA
:1092B000504C4120202D20203231352F35350041B2
:1092C000425320202D20203235352F31303000669A
:1092D00061726D20202D20203235302F3430004D2A
:1092E0003234004D323320257300052E2E005800F5
:1092F00059005A00457874727564657200473939AF
:109300000044697361626C65206661726D206D6FE7
:1093100064653F0044697361626C65206661726DCB
:10932000206D6F6465004661726D206E756D6265BB
:1093300072004D3834005072696E742066616E3A66
:109340000045787472756465722066616E3A0041FA
:10935000786973206C656E677468206469666665F9
:1093600072656E63653A004D656173757265642060
:1093700061786973206C656E6774683A004D3834A3
:10938000004731205A3135004732382057005A30D3
:10939000005A31005930005931005830005831001E
:1093A000456E642073746F70732064696167004D4B
:1093B0003434004732382057004175746F2072658D
:1093C000636F7665722063726173680043686563DA
:1093D0006B2066616E73205B4449535D0043686592
:1093E000636B2066616E73205B454E5D0054656D56
:1093F000706572617475726573002D2D2D2D2D2D84
:109400002D2D2D2D2D2D00466C6173684169722024
:10941000495020416464723A002D2D2D2D2D2D2DA3
:109420002D2D2D2D2D004E6F7620323620323031ED
:1094300037002D2D2D2D2D2D2D2D2D2D2D2D004594
:109440003344763666756C6C0045494E595F30344E
:109450006100315F37356D6D5F4D4B33002D2D2D24
:109460002D2D2D2D2D2D2D2D2D0020332E302E3157
:10947000322D5243322062313133004669726D77AA
:109480006172653A0025642E25642E25642E2564BC
:10949000004661696C207374617473004661726D7B
:1094A000206E756D626572000072630062657461A2
:1094B00000616C70686100646576005052555341DC
:1094C0003344465700332E302E31322D5243320072
:1094D00000000A0B02090C0D0E080703040100002E
:1094E000000000000000000000000000000000007C
:1094F0000000000000000000000000001211100039
:10950000000000000000000000000000000000005B
:10951000000000000000000000000000000000004B
:109520000000000000000102102020080810204068
:109530001020408002010201080402010102040817
:1095400010204080804020100804020180040201A5
:1095500080402010080402010804020101020408EE
:1095600010204080010204081020408010080408E8
:10957000801020400440801020400480050505052F
:10958000070508080808020202020A0A080804047B
:1095900004040101010101010101030303030303A9
:1095A0000303040707070C0C0C0C0C0C0C0C020238
:1095B000020206060606060606060B0B0B0B0B0B35
:1095C0000B0B07070A0A0A0A0A0A05050504040420
:1095D0000808000020002300260029002C002F008E
:1095E0003200000100000301060109010000220011
:1095F000250028002B002E0031003400020100005D
:10960000050108010B0100002100240027002A00A9
:109610002D003000330001010000040107010A01A0
:10962000024E414E494E495459494E46CDCCCC3D4F
:109630000AD7233C17B7D13877CC2B329595E6243F
:109640001FB14F0A000020410000C84200401C46E4
:1096500020BCBE4CCA1B0E5AAEC59D7400407A1089
:10966000F35A00A0724E18090010A5D4E80000E8D3
:109670007648170000E40B54020000CA9A3B000031
:1096800000E1F505000080969800000040420F00C0
:109690000000A08601000000102700000000E80381
:1096A000000000006400000000000A00000000004C
:1096B0000100000000002C76D888DC674F0823DF0B
:1096C000C1DFAE59E1B1B796E5E3E453C63AE651DE
:1096D000997696E8E6C28426EB898C9B62ED407C05
:1096E0006FFCEFBC9C9F40F2BAA56FA5F490055AA1
:1096F0002AF75C936B6CF9676DC11BFCE0E40D47C6
:10970000FEF520E6B500D0ED902E030094357705E8
:109710000080841E080000204E0A000000C80C33A0
:109720003333330F986E12831141EF8D2114893B2F
:10973000E65516CFFEE6DB18D1844B381BF77C1DAF
:10974000901DA4BBE424203284725E228100C9F102
:1097500024ECA1E53D2778BE16E5F501CF01FD011A
:10976000A9BE11241FBECFEFD1E2DEBFCDBF00E006
:109770000CBF19E0A0E0B2E0E8E0FFEC03E00BBFB3
:1097800002C007900D92A83EB107D9F72CE1A8EED0
:10979000B9E001C01D92A934B207E1F717E9C0E6AC
:1097A000D7E900E006C022970109FE010BBF0F9424
:1097B00095DDC635D10780E00807A9F70F946DD76E
:1097C0000D9472E70C940000CF92DF92EF92FF921B
:1097D0000F931F93CF93DF938C01D42EC62FD72FD7
:1097E000D60EDC1671F1F801E080F180C990C70156
:1097F0000F9465E4C816F1F06C2DC7010F9495E441
:10980000C7010F9465E48C15A9F0E2EBF7E08491B1
:10981000882341F09091C00095FFFCCF8093C60053
:109820003196F5CF8091C00085FFFCCF8AE0809310
:10983000C60007C0F80180819181019691838083E1
:10984000D0CFDF91CF911F910F91FF90EF90DF90DC
:10985000CF900895EF92FF920F931F93CF93DF93D2
:109860001F92CDB7DEB78C017B01460FF8018081D6
:10987000918149830F9465E4F70181937F01F80199
:109880008081918101969183808349814E11EECF31
:109890000F90DF91CF911F910F91FF90EF9008955E
:1098A000FF920F931F93CF93DF93CDB7DEB72C9723
:1098B0000FB6F894DEBF0FBECDBF8C01F62E80E34D
:1098C00090E3A0E3B0E08D839E83AF83B8871C87CD
:1098D0000B8744E0BE016B5F7F4FCE010B9674DFB8
:1098E00040E163E979E1CE010B966EDF40E163EA86
:1098F00079E1CE010B9668DF40E163E879E1CE01C2
:109900000B9662DF44E06BE779E1CE010B965CDFFA
:1099100044E067E779E1CE010B9656DF44E06FE75C
:1099200079E1CE010B9650DF44E063E679E1CE01A8
:109930000B964ADF44E063EB79E1CE010B9644DFFE
:1099400044E067E679E1CE010B963EDF44E06BE64A
:1099500079E1CE010B9638DF44E06FE679E1CE0184
:109960000B9632DF44E063E779E1CE010B962CDF02
:109970004CE06EE37BE0CE010B9626DF44E067E32C
:109980007BE0CE010B9620DF44E06DEA72E0CE0171
:109990000B961ADF44E069EA72E0CE010B9614DF01
:1099A00044E065EA72E0CE010B960EDF44E06DE91B
:1099B00072E0CE010B9608DF44E069E972E0CE0167
:1099C0000B9602DF44E065E972E0CE010B96FCDE07
:1099D00080E290E09A87898742E0BE01675F7F4F0F
:1099E000CE010B96F1DE41E063E37BE0CE010B9606
:1099F000EBDE44E064E272E0CE010B96E5DE44E08B
:109A00006CE172E0CE010B96DFDE44E06EE27BE0BB
:109A1000CE010B96D9DE44E06AE27BE0CE010B96E4
:109A2000D3DE44E068E172E0CE010B96CDDE41E08A
:109A30006AE57BE0CE010B96C7DE44E064E472E0A9
:109A4000CE010B96C1DE89E08F1560F444E062EB35
:109A500073E1CE010B96B8DE44E06EEA73E1CE010D
:109A60000B96B2DE46E551E360E070E049835A832D
:109A70006B837C831C870B8744E0BE016F5F7F4F45
:109A8000CE010B96A1DEE4E6FFE08491882341F04D
:109A90009091C00095FFFCCF8093C6003196F5CF22
:109AA000E2EAF7E08491882341F09091C00095FFAD
:109AB000FCCF8093C6003196F5CF8091C00085FF22
:109AC000FCCF8AE08093C6002C960FB6F894DEBFD8
:109AD0000FBECDBFDF91CF911F910F91FF900895E1
:109AE0001F93CF93DF93182FC4E6DFE0FE0184912C
:109AF000882341F09091C00095FFFCCF8093C60071
:109B00003196F5CFE2E9F7E08491882341F0909116
:109B1000C00095FFFCCF8093C6003196F5CF8091B1
:109B2000C00085FFFCCF8AE08093C600FE018491CF
:109B3000E4E6FFE0882349F09091C00095FFFCCF58
:109B40008093C60031968491F5CF4091931950913E
:109B5000941960919519709196198AE897E00E947E
:109B600007644091971950919819609199197091D3
:109B70009A1987E897E00E94076440919B195091D9
:109B80009C1960919D1970919E1984E897E00E943C
:109B9000076440919F195091A0196091A11970918B
:109BA000A21981E897E00E9407648091C00085FFB8
:109BB000FCCF8AE08093C600FE018491E4E6FFE0DA
:109BC000882349F09091C00095FFFCCF8093C60098
:109BD00031968491F5CFE7E6F7E08491882341F050
:109BE0009091C00095FFFCCF8093C6003196F5CFD1
:109BF0008091C00085FFFCCF8AE08093C600FE0103
:109C00008491E4E6FFE0882349F09091C00095FF3D
:109C1000FCCF8093C60031968491F5CF4091A31973
:109C20005091A4196091A5197091A6198EE597E03D
:109C30000E9407644091A7195091A8196091A91931
:109C40007091AA198BE597E00E9407644091AB19C7
:109C50005091AC196091AD197091AE1988E597E0FB
:109C60000E9407644091AF195091B0196091B119E9
:109C70007091B21985E597E00E9407648091C00059
:109C800085FFFCCF8AE08093C600FE018491E4E664
:109C9000FFE0882349F09091C00095FFFCCF8093AE
:109CA000C60031968491F5CFE7E3F7E084918823ED
:109CB00041F09091C00095FFFCCF8093C600319693
:109CC000F5CF8091C00085FFFCCF8AE08093C6006D
:109CD000FE018491E4E6FFE0882349F09091C00002
:109CE00095FFFCCF8093C60031968491F5CF4091CB
:109CF00083195091841960918519709186198EE2AB
:109D000097E00E94186440918719509188196091DA
:109D1000891970918A198BE297E00E94186440912A
:109D20008B1950918C1960918D1970918E1988E260
:109D300097E00E94186440918F195091901960919A
:109D400091197091921985E297E00E9418648091B0
:109D5000C00085FFFCCF8AE08093C600FE0184919D
:109D6000E4E6FFE0882349F09091C00095FFFCCF26
:109D70008093C60031968491F5CFE0EFF6E08491B0
:109D8000882341F09091C00095FFFCCF8093C600DE
:109D90003196F5CF8091C00085FFFCCF8AE080939B
:109DA000C600FE018491E4E6FFE0882349F090912B
:109DB000C00095FFFCCF8093C60031968491F5CF0B
:109DC00040917B1950917C1960917D1970917E1999
:109DD00087EE96E00E9407644091771950917819B8
:109DE0006091791970917A1984EE96E00E94076467
:109DF0008091C00085FFFCCF8AE08093C600FE0101
:109E00008491E4E6FFE0882349F09091C00095FF3B
:109E1000FCCF8093C60031968491F5CFE1E3F6E064
:109E20008491882341F09091C00095FFFCCF8093EE
:109E3000C6003196F5CF8091C00085FFFCCF8AE047
:109E40008093C600FE018491E4E6FFE0882349F098
:109E50009091C00095FFFCCF8093C600319684910D
:109E6000F5CF40917F1950918019609181197091BF
:109E7000821988E296E00E9407644091631950912C
:109E80006419609165197091661985E296E00E94E7
:109E900007644091B3195091B4196091B51970914C
:109EA000B61982E296E00E941864409167195091B9
:109EB00068196091691970916A198FE196E00E94A2
:109EC000076440916B1950916C1960916D197091F4
:109ED0006E198CE196E00E94076440916F195091D1
:109EE0007019609171197091721989E196E00E9460
:109EF00007644091731950917419609175197091AC
:109F0000761986E196E00E9407648091C00085FF83
:109F1000FCCF8AE08093C600FE018491E4E6FFE076
:109F2000882349F09091C00095FFFCCF8093C60034
:109F300031968491F5CFE4E0F6E08491882341F0F6
:109F40009091C00095FFFCCF8093C6003196F5CF6D
:109F50008091C00085FFFCCF8AE08093C600FE019F
:109F60008491E4E6FFE0882349F09091C00095FFDA
:109F7000FCCF8093C60031968491F5CF40913E0B83
:109F800050913F0B6091400B7091410B8BEF95E02E
:109F90000E9407644091420B5091430B6091440B27
:109FA0007091450B88EF95E00E9407644091460B45
:109FB0005091470B6091480B7091490B85EF95E0EC
:109FC0000E9407648091C00085FFFCCF8AE08093E7
:109FD000C600FE018491E4E6FFE0882349F09091F9
:109FE000C00095FFFCCF8093C60031968491F5CFD9
:109FF000E7EEF5E08491882341F09091C00095FF51
:10A00000FCCF8093C6003196F5CF8091C00085FFCC
:10A01000FCCF8AE08093C600FE018491E4E6FFE075
:10A02000882349F09091C00095FFFCCF8093C60033
:10A0300031968491F5CF4091AD025091AE0260917E
:10A04000AF027091B0028DED95E00E9407646091BF
:10A05000A9027091AA028091AB029091AC020F9478
:10A060004952AB01BC018AED95E00E940764609102
:10A07000A5027091A6028091A7029091A8020F9468
:10A080005552AB01BC0187ED95E00E9407648091B9
:10A09000C00085FFFCCF8AE08093C600FE0184915A
:10A0A000E4E6FFE0882349F09091C00095FFFCCFE3
:10A0B0008093C60031968491F5CFE1ECF5E0849170
:10A0C000882341F09091C00095FFFCCF8093C6009B
:10A0D0003196F5CF8091C00085FFFCCF8AE0809358
:10A0E000C600FE018491E4E6FFE0882349F09091E8
:10A0F000C00095FFFCCF8093C60031968491F5CFC8
:10A1000040919D0250919E0260919F027091A00229
:10A1100087EB95E00E9407646091990270919A0222
:10A1200080919B0290919C020F944952AB01BC011B
:10A1300084EB95E00E94076460919502709196020D
:10A1400080919702909198020F945552AB01BC01F7
:10A1500081EB95E00E9407648091C00085FFFCCFF1
:10A160008AE08093C600FE018491E4E6FFE0882344
:10A1700049F09091C00095FFFCCF8093C6003196C6
:10A180008491F5CFEDE7F5E08491882341F090913B
:10A19000C00095FFFCCF8093C6003196F5CF80912B
:10A1A000C00085FFFCCF8AE08093C600FE01849149
:10A1B000E4E6FFE0882349F09091C00095FFFCCFD2
:10A1C0008093C60031968491F5CF4091240250913E
:10A1D0002502609126027091270283E795E00E9494
:10A1E000076420E030E040E752E460911C02709187
:10A1F0001D0280911E0290911F020F942ADBAB0179
:10A20000BC0180E795E00E94076440912E0B5091BD
:10A210002F0B6091300B7091310B8DE695E00E9411
:10A2200007648091C00085FFFCCF8AE08093C60060
:10A23000FE018491E4E6FFE0882349F09091C0009C
:10A2400095FFFCCF8093C60031968491F5CFE1E471
:10A25000F5E08491882341F09091C00095FFFCCFF8
:10A260008093C6003196F5CF8091C00085FFFCCF6A
:10A270008AE08093C600FE018491E4E6FFE0882333
:10A2800049F09091C00095FFFCCF8093C6003196B5
:10A290008491F5CF40912A0B50912B0B60912C0BA0
:10A2A00070912D0B87E395E00E94076420E030E079
:10A2B00040E752E4609118027091190280911A02ED
:10A2C00090911B020F942ADBAB01BC0184E395E063
:10A2D0000E9407648091C00085FFFCCF8AE08093D4
:10A2E000C600FE018491E4E6FFE0882349F09091E6
:10A2F000C00095FFFCCF8093C60031968491F5CFC6
:10A30000EAEDF4E08491882341F09091C00095FF3C
:10A31000FCCF8093C6003196F5CF8091C00085FFB9
:10A32000FCCF8AE08093C600FE018491E4E6FFE062
:10A33000882349F09091C00095FFFCCF8093C60020
:10A3400031968491F5CF4091330B50E060E070E09E
:10A3500080ED94E00E9418648091C00085FFFCCFDE
:10A360008AE08093C600FE018491E4E6FFE0882342
:10A3700049F09091C00095FFFCCF8093C6003196C4
:10A380008491F5CF80915A0B8823A1F1EDEBF4E095
:10A390008491882341F09091C00095FFFCCF809379
:10A3A000C6003196F5CF8091C00085FFFCCF8AE0D2
:10A3B0008093C600FE018491E4E6FFE0882349F023
:10A3C0009091C00095FFFCCF8093C6003196849198
:10A3D000F5CF409144025091450260914602709140
:10A3E000470283EB94E00E9407648091C00085FFE0
:10A3F000FCCF11C0E7E9F4E08491882341F090910B
:10A40000C00095FFFCCF8093C6003196F5CF8091B8
:10A41000C00085FFFCCF8AE08093C6001A3008F4A4
:10A420003EC0FE01C491E4E6FFE0CC2349F08091F8
:10A43000C00085FFFCCFC093C6003196C491F5CF14
:10A44000EEE7F4E08491882341F09091C00095FFFD
:10A45000FCCF8093C6003196F5CF8091C00085FF78
:10A46000FCCF8AE08093C6004091B2135091B313A1
:10A470006091B4137091B51384E794E00E9407646F
:10A480004091AE135091AF136091B0137091B1131E
:10A490008AE694E0DF91CF911F910C940764DF91DD
:10A4A000CF911F910895AF92BF92CF92DF92EF921A
:10A4B000FF920F931F93CF93DF93CDB7DEB7E09753
:10A4C0000FB6F894DEBF0FBECDBF80E1E2EEF2E042
:10A4D000DE01919601900D928A95E1F780E1E2EF1D
:10A4E000F2E0DE01519601900D928A95E1F780E14C
:10A4F000E2E0F3E0DE01119601900D928A95E1F71A
:10A500006E0181E2C80ED11C83E9E82E89E1F82EA4
:10A510008E010F5E1F4F63EA79E1AE014F5F5F4F1F
:10A5200093E8A92E99E1B92E20E030E0F60181915F
:10A530009191A191B1916F01F70181939193A193B1
:10A54000B1937F01F80181919191A191B1918F0116
:10A55000FB0181939193A193B193BF01FA01819182
:10A560009191A191B191AF01F50181939193A19343
:10A57000B1935F012F5F3F4F24303105B9F60F943F
:10A58000AB2E80E090E4ACE9B4E480937B19909327
:10A590007C19A0937D19B0937E19809377199093BD
:10A5A0007819A0937919B0937A1910927F191092A3
:10A5B0008019109281191092821980E29EE4A0E025
:10A5C000B0E08093B3199093B419A093B519B093E8
:10A5D000B6191092631910926419109265191092AD
:10A5E000661980E090E0A0E7B1E48093671990934A
:10A5F0006819A0936919B0936A1980936B199093A5
:10A600006C19A0936D19B0936E198DEC9CECACECA9
:10A61000BEE380936F1990937019A0937119B09352
:10A62000721980E090E0A0E2B0E4809373199093F7
:10A630007419A0937519B09376191092460B109265
:10A64000470B1092480B1092490B1092420B10923C
:10A65000430B1092440B1092450B10923E0B10923C
:10A660003F0B1092400B1092410B8DE39AE0A1E852
:10A67000B1E48093AD029093AE02A093AF02B09389
:10A68000B0026DEC7CEC84E99FE30F94435260933D
:10A69000A9027093AA028093AB029093AC0265E882
:10A6A0007BEE80E692E40F944F526093A502709384
:10A6B000A6028093A7029093A8020F941A4180E00B
:10A6C00090E0A0E8BFE38093A1029093A202A09340
:10A6D000A302B093A4021092330B80E090E0A0E4B8
:10A6E000B0E48093240290932502A0932602B093B5
:10A6F000270240E050E064E372E440931C02509370
:10A700001D0260931E0270931F0210922E0B109276
:10A710002F0B1092300B1092310B10922A0B1092CB
:10A720002B0B10922C0B10922D0B40E050E060E0B0
:10A7300071E4409318025093190260931A027093C7
:10A740001B0210925A0B8093440290934502A093EF
:10A750004602B09347020E948F7AE4E6FFE08491BC
:10A76000882341F09091C00095FFFCCF8093C600F4
:10A770003196F5CFEEE2F4E08491882341F0909198
:10A78000C00095FFFCCF8093C6003196F5CF809135
:10A79000C00085FFFCCF8AE08093C600E0960FB62C
:10A7A000F894DEBF0FBECDBFDF91CF911F910F9107
:10A7B000FF90EF90DF90CF90BF90AF9008951F93E0
:10A7C000CF93DF93CDB7DEB72C970FB6F894DEBFEB
:10A7D0000FBECDBF162F9C878B8786E591E3A0E047
:10A7E000B0E089839A83AB83BC8344E0BE016B5F96
:10A7F0007F4FCE010B962ED843E050E0BE016B5F39
:10A800007F4FCE0101960F9437E1892B09F0FFC0ED
:10A8100040E163E979E1CE010B961CD840E163EA9F
:10A8200079E1CE010B9616D840E163E879E1CE01DB
:10A830000B9610D80F94AB2E44E06BE779E1CE0174
:10A840000B9608D844E067E779E1CE010B9602D871
:10A8500044E06FE779E1CE010B960E942A4C44E078
:10A8600063E679E1CE010B960E942A4C44E063EB4B
:10A8700079E1CE010B960E942A4C44E067E679E12B
:10A88000CE010B960E942A4C44E06BE679E1CE01A2
:10A890000B960E942A4C44E06FE679E1CE010B96BC
:10A8A0000E942A4C44E063E779E1CE010B960E94B6
:10A8B0002A4C4CE06EE37BE0CE010B960E942A4CC2
:10A8C00044E067E37BE0CE010B960E942A4C44E013
:10A8D0006DEA72E0CE010B960E942A4C44E069EAD0
:10A8E00072E0CE010B960E942A4C44E065EA72E0C9
:10A8F000CE010B960E942A4C44E06DE972E0CE0135
:10A900000B960E942A4C44E069E972E0CE010B9656
:10A910000E942A4C44E065E972E0CE010B960E9449
:10A920002A4C42E0BE01675F7F4FCE010B960E942A
:10A930002A4C41E063E37BE0CE010B960E942A4C57
:10A9400044E064E272E0CE010B960E942A4C44E09F
:10A950006CE172E0CE010B960E942A4C44E06EE25C
:10A960007BE0CE010B960E942A4C44E06AE27BE039
:10A97000CE010B960E942A4C44E068E172E0CE01C1
:10A980000B960E942A4C41E06AE57BE0CE010B96D3
:10A990000E942A4C44E064E472E0CE010B960E94CF
:10A9A0002A4C1A3070F044E062EB73E1CE010B9652
:10A9B0000E942A4C44E06EEA73E1CE010B960E949D
:10A9C0002A4C0E948F7A0F941A41E4E6FFE08491AA
:10A9D000882341F09091C00095FFFCCF8093C60082
:10A9E0003196F5CFE0E5F4E08491882341F0909131
:10A9F000C00095FFFCCF8093C6003196F5CF8091C3
:10AA0000C00085FFFCCF8AE08093C60001C04BDD0B
:10AA10002C960FB6F894DEBF0FBECDBFDF91CF915D
:10AA20001F910895682F772767FD70958091961084
:10AA30009091971085569F4E0F941CE190938D1026
:10AA400080938C1021E0892B09F420E0822F089557
:10AA500080918C1090918D1060E070E001960D94C3
:10AA6000C5DD282F6091431C7091441C90E02A3072
:10AA700018F0895A9F4F01C0C0960D946EE1CF9394
:10AA8000C82F82958F70EDDF8C2F8F70CF91E9CF1B
:10AA9000CF93C82F892FF3DF8C2FCF91F0CF6F92F8
:10AAA0007F928F929F92AF92BF92CF92DF92EF925E
:10AAB000FF920F931F93CF93DF936B017C01EA0109
:10AAC000122F209709F455C0123011F48E2DC9DFD2
:10AAD000C601DEDF6091431C7091441C80E290E06F
:10AAE0000F946EE1702E7C1A8C2F870D09F438C0FC
:10AAF0001130D1F088F0123029F5460157018FEF5F
:10AB0000881A980AA80AB80AEE24D7FCE094FE2C0A
:10AB1000EBBEF601679013C0F60160808FEFC81A94
:10AB2000D80AE80AF80A0FC0460157018FEF881AC1
:10AB3000980AA80AB80AC6010F9465E4682E750140
:10AB4000640101C0612C6091431C7091441C80E23F
:10AB500090E00F946EE1862D92DF219709F0C4CF2B
:10AB60006091431C7091441C8AE090E00F946EE168
:10AB7000A8CFDF91CF911F910F91FF90EF90DF90C1
:10AB8000CF90BF90AF909F908F907F906F900895DF
:10AB9000CF93DF93FB0120E030E0DC01ED018D91EC
:10ABA0008823A1F14115510519F02417350774F5D3
:10ABB0008032A1F38A3051F190ED980F9A3020F451
:10ABC000682F6295607F08C09FE9980F9630A8F4BF
:10ABD000682F6295607F6057CE0102967981A0ED63
:10ABE000A70FAA3018F4762F7A2B0CC0AFE9A70F65
:10ABF000A63018F47755762B05C088279927821B35
:10AC0000930B05C071932F5F3F4FC7CFC901DF91F1
:10AC1000CF9108958AE693E00F94DEE1F894FFCF98
:10AC2000E0918C10F0918D108181882399F082E45D
:10AC3000F9DE882369F0F89428E088E190E00FB607
:10AC4000F894A895809360000FBE20936000FFCF1A
:10AC50000C9400000895F894C0E0D0E06FEFCE01AE
:10AC60000F9495E42196C11580E2D807B9F728E042
:10AC700088E190E00FB6F894A895809360000FBE2D
:10AC800020936000FFCF0F931F93CF93DF93CDB737
:10AC9000DEB762970FB6F894DEBF0FBECDBF81E47A
:10ACA000C1DE8823A9F080918C1090918D10FC0159
:10ACB0002181283741F440E150E060E070E00296E5
:10ACC0000F942DDF03C0C4DE0F94C4D88B0102C0E3
:10ACD00000E010E083E4A6DE882331F0B9DE0F94B3
:10ACE000C4D8262F872F02C020E080E21F71422F98
:10ACF000582F4130F0E25F0710F040E050E2CA0107
:10AD0000800F911F8130904220F040E050E2401BC4
:10AD1000510B88E5498B5A8B85DE49895A898823EE
:10AD2000D1F080918C1090918D1040E150E0BE01E7
:10AD30006F5F7F4F01962CDFAC01009761F0FE0141
:10AD40003196CF01840F951FD801E817F90719F044
:10AD500021912D93FACFB80180E090E000E120E04E
:10AD60009EDE62960FB6F894DEBF0FBECDBFDF91B8
:10AD7000CF911F910F910895AF92BF92CF92DF9222
:10AD8000EF92FF920F931F93CF93DF93CDB7DEB770
:10AD900060970FB6F894DEBF0FBECDBF81E442DEF0
:10ADA0008823A9F080918C1090918D10FC01218155
:10ADB000283741F440E150E060E070E002960F94E3
:10ADC0002DDF03C045DE0F94C4D88B0102C000E024
:10ADD00010E083E427DE882331F03ADE0F94C4D8F4
:10ADE000262F872F02C020E080E21F71E22EF82E6E
:10ADF000F1E0EF16F0E2FF0618F0E12C90E2F92EF8
:10AE0000C701800F911F8130904228F0E12C80E231
:10AE1000F82EE01AF10A88E505DE882361F18091B9
:10AE20008C1090918D1040E150E0BE016F5F7F4F1C
:10AE30000196AEDE7C010097F1F0CE0101965C0137
:10AE4000C12CD12CCE14DF0461F0F50161915F01BA
:10AE5000C601800F911F0F9495E4FFEFCF1ADF0A10
:10AE6000F1CFC80115DE6091431C7091441C8AE04B
:10AE700090E00F946EE1B80180E090E000E121E005
:10AE8000A7010DDE60960FB6F894DEBF0FBECDBFF2
:10AE9000DF91CF911F910F91FF90EF90DF90CF90B6
:10AEA000BF90AF900895CF92DF92EF92FF9280E52E
:10AEB000B9DD882309F44CC0CBDD0F94C4D86B01F5
:10AEC0007C018FEFC816D10411F008F041C086E470
:10AED000A9DD882379F0BCDD0F94C4D86115710514
:10AEE00011F460E004C06130710521F461E08C2D43
:10AEF0000F9469D186E596DD882399F0A9DD0F943A
:10AF0000C4D86115710511F460E004C061307105A9
:10AF1000F9F461E08C2DFF90EF90DF90CF900D94CD
:10AF2000A2D18C2D0F94D7D121E0892B09F420E0F8
:10AF30001F922F93DF92CF928DE793E09F938F9391
:10AF40000F94CDE10F900F900F900F900F900F90F6
:10AF5000FF90EF90DF90CF90089508950895CF92DD
:10AF6000DF92EF92FF92C090BC1AD090BD1AE09091
:10AF7000BE1AF090BF1AC701B6010E944580E09149
:10AF80008C10F0918D1082818F3309F440C088239A
:10AF900009F43DC0813239F561E086EA9FE00F9403
:10AFA00095E462E370E080EB9FE00F94A3E464E635
:10AFB00070E082EB9FE00F94A3E466E970E084EB1D
:10AFC0009FE00F94A3E468EC70E086EB9FE00F94A1
:10AFD000A3E46AEF70E088EB9FE0FF90EF90DF90D2
:10AFE000CF900D94A3E480E51DDD882319F030DDBA
:10AFF0006B017C01C701B6010E9445808AE512DD24
:10B00000882329F0FF90EF90DF90CF9021CDFF9023
:10B01000EF90DF90CF90089566EE87EF9FE00D945C
:10B0200077E460E086E69FE00F9477E460E085E6F1
:10B030009FE00F9477E460E084E69FE00D9477E46E
:10B040000895E0918C10F0918D1085818F3311F06F
:10B0500081112BC080918F131F928F938091901339
:10B060001F928F93809192138F93809191138F935E
:10B07000809194138F93809193138F938091951364
:10B080001F928F93809196131F928F9386E893E07F
:10B090009F938F930F94CDE18DB79EB70E960FB609
:10B0A000F8949EBF0FBE8DBF0895813229F50F948D
:10B0B000331A80918F131F928F93809190131F9258
:10B0C0008F93809192138F93809191138F9380919E
:10B0D00094138F93809193138F9388E993E09F93B8
:10B0E0008F930F94CDE18DB79EB70A960FB6F89463
:10B0F0009EBF0FBE8DBF089582E594DC8111A8DC50
:10B1000088E590DC882339F0A3DC0F94C4D87093D1
:10B1100094136093931389E585DC882339F098DCD8
:10B120000F94C4D870939213609391138CE47ADCDB
:10B13000882329F08DDC0F94C4D8609368020895A9
:10B14000CF93DF93EC0160E08E810F94A2D181E078
:10B1500090E00F94E4CF61E08E810F94A2D181E062
:10B1600090E00F94E4CF60E08E810F94A2D184E64A
:10B1700090E0DF91CF910D94E4CFCF92DF92EF92E8
:10B18000FF920F931F93CF93DF937C01C0E0D0E039
:10B19000C62ED12C87010C0F1D1F61E0F80187819D
:10B1A0000F9469D1B6010C2E02C0759567950A946B
:10B1B000E2F76170F80187810F94A2D12196C43023
:10B1C000D10541F7C701DF91CF911F910F91FF90FA
:10B1D000EF90DF90CF90B4CFCF92DF92EF92FF92BB
:10B1E0000F931F93CF93DF937C01C0E0D0E0C62E76
:10B1F000D12C87010C0F1D1F61E0F80187810F948E
:10B2000069D1B6010C2E02C0759567950A94E2F7D4
:10B210006170F80187810F94A2D12196C830D105C1
:10B2200041F7C701DF91CF911F910F91FF90EF90F0
:10B23000DF90CF9085CF1F93CF93DF93EC01162F34
:10B24000642F8C810F94A2D18D818F3F19F060E023
:10B250000F94A2D18F85612F84FF05C0CE01DF91AD
:10B26000CF911F91B9CF70E084E0759567958A956D
:10B27000E1F7CE0182DF612FCE01DF91CF911F91E7
:10B280007CCF40E0D8CF61E0FCDF80E496E00D9415
:10B29000E4CF62E0F6DF80E496E00D94E4CFCF9354
:10B2A000DF93CDB7DEB728970FB6F894DEBF0FBE99
:10B2B000CDBF28E0E2E1F3E0DE01119601900D92AE
:10B2C0002A95E1F7FC012389421710F04FEF420F56
:10B2D000FE013196E40FF11DE40FF11D2081260FD0
:10B2E0002068622F28960FB6F894DEBF0FBECDBF40
:10B2F000DF91CF91C6CFFC016089262F2460208B7F
:10B300006C60BFCFCF93DF93EC01423018F08F8594
:10B3100088608F874B8B1C8A222329F0413019F4D7
:10B320008F8584608F8780E593EC0F94E4CF60E095
:10B330008C810F94A2D160E08E810F94A2D18D8177
:10B340008F3F19F060E00F94A2D16F8564FD19C0A2
:10B3500063E0CE0112DF84E991E10F94E4CF63E072
:10B36000CE010BDF84E991E10F94E4CF63E0CE01DD
:10B3700004DF86E990E00F94E4CF62E0CE01FDDEC9
:10B3800013C06062CE017DDF84E991E10F94E4CFC8
:10B390006F856062CE0175DF86E990E00F94E4CF9F
:10B3A0006F856062CE016DDF6F856062CE0169DFFF
:10B3B0008CE390E00F94E4CF84E0888BCE019BDF98
:10B3C0008CE390E00F94E4CFCE015DDF88EB9BE04F
:10B3D0000F94E4CF82E0898B66E0CE0152DF8CE3EC
:10B3E00090E00F94E4CF1D8ADF91CF9108956F9282
:10B3F0007F928F92AF92CF92EF920F931F93CF9342
:10B40000DF93CDB7DEB73C01162F842F5E854F85C5
:10B4100038899989F301848325830683E782C0866E
:10B42000A1868286538744873587968761E00F948B
:10B4300069D1F30185818F3F19F061E00F9469D1E3
:10B4400061E0F30186810F9469D1112319F0F301B2
:10B45000178603C080E1F301878720E041E060E1C7
:10B46000C301DF91CF911F910F91EF90CF90AF90DB
:10B470008F907F906F9046CF8F92AF92CF92EF9246
:10B480000F93DC0113961C921E921297E1EBF3E0EE
:10B49000ED93FC931F921F921F921F928C2CAE2C47
:10B4A000C02EE22E042F2FEF462F61E0A0DF0F9079
:10B4B0000F900F900F900F91EF90CF90AF908F90D3
:10B4C0000895CF93DF93EC01423018F08F858860A8
:10B4D0008F874B8B1C8A222329F0413019F48F85EA
:10B4E00084608F8780E593EC0F94E4CF60E08C81DB
:10B4F0000F94A2D160E08E810F94A2D18D818F3FF5
:10B5000019F060E00F94A2D16F8564FD19C063E06B
:10B51000CE0133DE84E991E10F94E4CF63E0CE0104
:10B520002CDE84E991E10F94E4CF63E0CE0125DEC7
:10B5300086E990E00F94E4CF62E0CE011EDE13C0F6
:10B540006062CE019EDE84E991E10F94E4CF6F85C5
:10B550006062CE0196DE86E990E00F94E4CF6F85BD
:10B560006062CE018EDE6F856062CE018ADE8CE382
:10B5700090E00F94E4CF84E0888BCE01BCDE8CE3B6
:10B5800090E00F94E4CFCE0184DE80E496E00F9447
:10B59000E4CF82E0898B66E0CE0173DE8CE390E03D
:10B5A0000F94E4CF40E068E0CE0179DE67E379E014
:10B5B000CE010F943DD241E068E0CE0170DE67E33A
:10B5C00079E0CE010F943DD242E066E0CE0167DE25
:10B5D00065E379E0CE01DF91CF910D943DD2FC017E
:10B5E00060896D7F608B68604CCECF93DF93EC01F8
:10B5F000262F8D898230B0F0FE01E80FF11D658B9A
:10B600003E8980ED860F8A3058F4316081E090E009
:10B610000D8802C0880F991F0A94E2F7382B01C0E9
:10B620003E7F3E8B4D8981E0840F8D8B50E048300A
:10B63000510508F0B6C0FA01EE58FF4F0D946ADDCF
:10B640002B3109F0AEC0AEC01E8A2B3509F0A9C05F
:10B65000A9C0223309F4A6C02F3309F4A3C08E89F0
:10B660007AC08F89823331F08F3349F4223309F065
:10B6700098C098C02A3419F4CE0105DE92C08E8994
:10B6800082FF8FC02B3309F066C08CC08F898F3347
:10B6900041F4888D823309F084C0253309F081C0DC
:10B6A00081C08E8982FF7DC0988D9B3311F480FD0F
:10B6B00079C083FF76C02B3309F073C073C04F8904
:10B6C0004F3371F4888D823309F06BC0898D8533D7
:10B6D00009F067C02C3609F064C0CE0180DF61C07C
:10B6E0008E8982FF5EC0988D9B3339F484FF05C03C
:10B6F000283489F54053698D2CC083FF52C0998D41
:10B700009B3309F04EC027C08E8982FF4AC0488D06
:10B710004B3361F4982F9073903341F4283431F413
:10B720004F8940536A8D6053898D32C083FF39C081
:10B73000998D9B33B1F585FF34C0283461F44053B3
:10B740008F89880F8056982F990F990F980F490F5E
:10B750006A8D605324C080FF24C024C08E89982F36
:10B760009C709C30F1F4998D9B33D9F480768036AF
:10B77000C1F42834B1F4488D40538F89880F805626
:10B78000982F990F990F980F490F6B8D60538A8DE1
:10B79000880F8056982F990F990F980F690FCE0137
:10B7A0007EDD1D8A81E090E0DF91CF910895CF92F8
:10B7B000DF92EF92FF920F931F93CF93DF931F922D
:10B7C0001F92CDB7DEB78C01677088E0689FB0012B
:10B7D00011246064C80149835A8353DD4981C42E12
:10B7E0005A81D52EE12CF12CD6016D916D01D80135
:10B7F000ED91FC910190F081E02DC8011995BFEF0A
:10B80000EB1AFB0AE8E0EE16F10471F70F900F90C7
:10B81000DF91CF911F910F91FF90EF90DF90CF902C
:10B820000895FC012589211102C06B3109F4DDCE98
:10B8300041E001DD81E090E008951F920F920FB684
:10B840000F9211240BB60F922F933F934F935F9358
:10B850006F938F939F93EF93FF938091C00084FF2A
:10B8600003C08091C60019C06091C6002091690A8A
:10B8700030916A0AC90101968F77992740916B0A26
:10B8800050916C0A8417950741F0F901E751F64F82
:10B89000608390936A0A8093690AFF91EF919F9168
:10B8A0008F916F915F914F913F912F910F900BBEB0
:10B8B0000F900FBE0F901F9018951F920F920FB60A
:10B8C0000F9211240BB60F922F933F934F935F93D8
:10B8D0006F938F939F93EF93FF9380916D0A8130C5
:10B8E00001F58091D00084FF03C08091D60019C07B
:10B8F0006091D6002091690A30916A0AC9010196C7
:10B900008F77992740916B0A50916C0A841795079D
:10B9100041F0F901E751F64F608390936A0A8093F2
:10B92000690AFF91EF919F918F916F915F914F9174
:10B930003F912F910F900BBE0F900FBE0F901F9055
:10B940001895CF92DF92EF92FF926A017B01411529
:10B9500081EE58076105710509F463C082E08093A8
:10B96000C00060E079E08DE390E0A70196010F94BC
:10B970004EDD2150310941095109CA01B90122E0C6
:10B9800030E040E050E00F944EDD91E03093C50090
:10B990002093C4008091C10080618093C100809198
:10B9A000C10088608093C1008091C100806880934D
:10B9B000C10080916D0A8130D1F5992341F082E078
:10B9C0008093D00060E079E08DE390E006C01092B3
:10B9D000D00060E874E88EE190E0A70196010F9432
:10B9E0004EDD2150310941095109CA01B90122E056
:10B9F00030E040E050E00F944EDD3093D5002093CE
:10BA0000D4008091D10080618093D1008091D100D9
:10BA100088608093D1008091D10080688093D100AC
:10BA200006C01092C00090E020E130E0AFCFFF9060
:10BA3000EF90DF90CF90089520916B0A30916C0ABF
:10BA40008091690A90916A0A8217930771F0F9014F
:10BA5000E751F64F80812F5F3F4F2F773327309389
:10BA60006C0A20936B0A90E008958FEF9FEF089582
:10BA700080916B0A90916C0A90936A0A8093690A8C
:10BA800008954F925F926F927F928F929F92AF92A2
:10BA9000BF92CF92DF92EF92FF920F931F93CF93BB
:10BAA000DF93CDB7DEB7A0970FB6F894DEBF0FBE19
:10BAB000CDBF5C014115510561057105E9F420E038
:10BAC00030E040E350E060E070E0A0960FB6F894FC
:10BAD000DEBF0FBECDBFDF91CF911F910F91FF90C1
:10BAE000EF90DF90CF90BF90AF909F908F907F901E
:10BAF0006F905F904F905BC08E010F5F1F4FC12C06
:10BB0000D12C76014801422E512C612C712C8FEFE3
:10BB1000C81AD80AE80AF80ACB01BA01A3019201AF
:10BB20000F942CDDCA01F80161938F01A901BC01BA
:10BB3000411551056105710551F7F1E0CF1AD108A2
:10BB4000E108F108F401EC0DFD1D80818A3010F44C
:10BB500040E301C047E3480F552747FD5095652F47
:10BB6000752F20E030E0C50122D081E0C81AD1084D
:10BB7000E108F108EFEFCE16DE06EE06FE0611F73D
:10BB8000A0960FB6F894DEBF0FBECDBFDF91CF9168
:10BB90001F910F91FF90EF90DF90CF90BF90AF90EB
:10BBA0009F908F907F906F905F904F900895211598
:10BBB000310539F48091C00085FFFCCF4093C60069
:10BBC00008952A30310509F43FC05BCF9A01462F12
:10BBD000552747FD5095652F752FE9CFCF93DF93FC
:10BBE000EC0120E030E04DE050E060E070E0DFDFAD
:10BBF00020E030E04AE050E060E070E0CE01DF910C
:10BC0000CF91D5CFFB012191BF01222339F0309193
:10BC1000C00035FFFCCF2093C600F4CFDFCF9A01E0
:10BC2000AB01662757FD6095762FC1CFCF93DF9389
:10BC3000EC019A01AB01662757FD6095762FB7DFBF
:10BC4000CE01DF91CF91CACFCF92DF92EF92FF92D8
:10BC5000CF93DF93EC016A017B0177FF0FC020E0F7
:10BC600030E04DE250E060E070E0A1DFF094E0945D
:10BC7000D094C094C11CD11CE11CF11C2AE0B70176
:10BC8000A601CE01DF91CF91FF90EF90DF90CF9092
:10BC9000F8CE2115310539F48091C00085FFFCCF25
:10BCA0004093C6000895EDCECF93DF93EC019A0147
:10BCB000462F50E060E070E0ECDFCE01DF91CF91E5
:10BCC0008DCFCF93DF93EC019A01AB0160E070E080
:10BCD000E0DFCE01DF91CF9181CFCF93DF93EC01F5
:10BCE000D8DFCE01DF91CF9179CF8F929F92AF9223
:10BCF000BF92CF92DF92EF92FF921F93CF93DF9389
:10BD0000EC016A017B01122F20E030E0A901C7019C
:10BD1000B6010F9455D887FF0CC020E030E04DE20B
:10BD200050E060E070E0CE0142DFF7FAF094F7F8FF
:10BD3000F094B12C60E070E080E09FE3B11641F038
:10BD400020E030E040E251E40F945CD8B394F6CFA9
:10BD50009B01AC01C701B6010F947CD76B017C013C
:10BD60000F94C9D84B015C010F94F5D89B01AC012D
:10BD7000C701B6010F947BD76B017C012AE0B501A6
:10BD8000A401CE017EDE112361F0EDE0F6E08191A9
:10BD9000882339F09091C00095FFFCCF8093C600B6
:10BDA000F6CF112319F120E030E040E251E4C70161
:10BDB000B6010F942ADB6B017C010F94C4D84B01B0
:10BDC000AA2497FCA094BA2CB501A401CE013CDFB3
:10BDD000C501B4010F94F7D89B01AC01C701B601AE
:10BDE0000F947BD76B017C011150DBCFDF91CF919A
:10BDF0001F91FF90EF90DF90CF90BF90AF909F90FA
:10BE00008F90089572CFCF93DF93EC016EDFCE0158
:10BE1000DF91CF91E3CE9091C00095FFFCCF80934E
:10BE2000C60080E090E00895FC01659175918591D0
:10BE300094910895EF92FF920F931F93CF93DF9306
:10BE4000EC01CC0FDD1FCC0FDD1FCE01805C904FCD
:10BE5000EBDF9E01265B344F79018E01025C144FAB
:10BE6000F80120813181428153810F947CD7F70101
:10BE70006083718382839383CE01885A904FD4DF8D
:10BE80009E012C5C3D4F7901F80120813181428176
:10BE900053810F947CD7F7016083718382839383EE
:10BEA000CE01845B904FC0DFC85DDD4FF80120817B
:10BEB0003181428153810F947CD7688379838A834F
:10BEC0009B83DF91CF911F910F91FF90EF90089589
:10BED000CF93C82F40910C0250910D0260910E0239
:10BEE00070910F024093010B5093020B6093030B70
:10BEF0007093040B20915602309157023093B40B8B
:10BF00002093B30B24E630E030935702209356027F
:10BF10000F947ECF6093FC0A7093FD0A8093FE0A13
:10BF20009093FF0A8C2FCF910D94543080E00F94A2
:10BF300054308091010B9091020BA091030BB091B2
:10BF4000040B80930C0290930D02A0930E02B09309
:10BF50000F028091B30B9091B40B90935702809392
:10BF600056020F947ECF6093FC0A7093FD0A809373
:10BF7000FE0A9093FF0A0895682F772767FD709552
:10BF8000809196109091971085569F4E0F941CE1CA
:10BF900090938D1080938C1021E0892B09F420E080
:10BFA000822F089580918C1090918D104AE050E07E
:10BFB00060E070E001960F942DDFCB010895809131
:10BFC0008C1090918D104AE050E060E070E0019696
:10BFD0000D942DDF2091961030919710BC01C9016E
:10BFE00085569F4E0F9454E190938D1080938C1042
:10BFF00021E0892B09F420E0822F08950F931F93ED
:10C00000CF93DF9300918C1010918D1065E470E058
:10C01000C8010F941CE1EC01009751F460E070E05E
:10C02000C8010196DF91CF911F910F910D94C5DD4D
:10C03000188280918C1090918D1060E070E00196D4
:10C040000F94C5DD25E42883DF91CF911F910F91D7
:10C05000089580918C1090918D1060E070E00196B1
:10C060000D94C5DD2F923F924F925F926F927F9217
:10C070008F929F92AF92BF92CF92DF92EF92FF92F8
:10C080000F931F93CF93DF93CDB7DEB760970FB6B3
:10C09000F894DEBF0FBECDBF1C012A013B01480151
:10C0A000590120E030E04CE052E4C301B2010F94AA
:10C0B0007BD725E535E547E052E40F945CD86B016A
:10C0C0007C010F9432D90F94C4D88B0177FF12C032
:10C0D00020E030E040E85FE3C701B6010F9458DA92
:10C0E00018160CF05DC0C12CD12CE0E8EE2EEFE369
:10C0F000FE2E56C066307105DCF02AEA3AE24CE4C6
:10C1000053E4C301B2010F947BD725E535E547E041
:10C1100052E40F945CD86B017C0120E030E0A9016F
:10C120000F9455D887FF3FC0C12CD12C76013BC05E
:10C13000882777FD8095982F0F94F7D825E535E56A
:10C1400047E052E40F942ADB20E030E04CE052E478
:10C150000F947CD79B01AC01C301B2010F947BD734
:10C1600025E535E547E052E40F945CD86B017C018E
:10C1700020E030E0A9010F9455D887FD17C020E0DA
:10C1800030E040E85FE3C701B6010F9458DA1816B3
:10C1900084F4C12CD12C70E8E72E7FE3F72E09C080
:10C1A00000E010E006C005E010E003C0C12CD12C77
:10C1B000760120E030E040EC50E4C501B4010F947A
:10C1C0007BD72BEA3AEA42E052E40F945CD82B0189
:10C1D0003C010F9432D90F94C4D8788B6F8777FFC6
:10C1E00012C020E030E040E85FE3C301B2010F94E9
:10C1F00058DA18160CF05FC0412C512C60E8662EFE
:10C200006FE3762E58C0AF85B8891697E4F026E51F
:10C2100035E549E253E4C501B4010F947BD72BEA1D
:10C220003AEA42E052E40F945CD82B013C0120E052
:10C2300030E0A9010F9455D887FD40C0E5E0F0E05B
:10C24000F88BEF8746C0882777FD8095982F0F944D
:10C25000F7D82BEA3AEA42E052E40F942ADB20E0D6
:10C2600030E040EC50E40F947CD79B01AC01C50159
:10C27000B4010F947BD72BEA3AEA42E052E40F94E0
:10C280005CD82B013C0120E030E0A9010F9455D887
:10C2900087FD1CC020E030E040E85FE3C301B2014D
:10C2A0000F9458DA1816ACF4412C512C50E8652E36
:10C2B0005FE3752E0EC0188A1F860BC0412C512CCF
:10C2C000320125E030E0388B2F8703C0412C512C00
:10C2D0003201A701960160E070E080E89FE30F94CF
:10C2E0007BD769837A838B839C83C80101969E8365
:10C2F0008D83AF85B8891196BA87A987A30192016A
:10C3000060E070E080E89FE30F947BD76B877C87C9
:10C310008D879E8747E02F853889429FF001439F94
:10C32000F00D1124F887EF83E00FF11FEE0FFF1FD0
:10C33000EE0FFF1FE20DF31D2181328143815481F5
:10C3400069817A818B819C810F942ADB4B015C018E
:10C35000EF81F8858D819E81E80FF91FEE0FFF1F99
:10C36000EE0FFF1FE20DF31D2181328143815481C5
:10C37000C701B6010F942ADB9B01AC01C501B401D2
:10C380000F947CD79B01AC016B857C858D859E8548
:10C390000F942ADB4B015C0127E0E985FA852E9F8B
:10C3A000D0012F9FB00D1124B887AF83FD01E00F9E
:10C3B000F11FEE0FFF1FEE0FFF1FE20DF31D218196
:10C3C00032814381548169817A818B819C810F9470
:10C3D0002ADB69837A838B839C83AF81B8858D81C7
:10C3E0009E81A80FB91FAA0FBB1FAA0FBB1FA20DCA
:10C3F000B31D11962D913D914D915C911497C701FC
:10C40000B6010F942ADB9B01AC0169817A818B8193
:10C410009C810F947CD79B01AC01C301B2010F94A6
:10C420002ADB9B01AC01C501B4010F947CD7609657
:10C430000FB6F894DEBF0FBECDBFDF91CF911F9135
:10C440000F91FF90EF90DF90CF90BF90AF909F90B3
:10C450008F907F906F905F904F903F902F900895B6
:10C460004F925F926F927F929F92AF92BF92CF92C4
:10C47000DF92EF92FF920F931F93CF93DF937C0194
:10C480005B018A01E9019090C912911014C0FC016E
:10C4900080819181A281B381FA0180839183A283FB
:10C4A000B383FB0180819181A281B38188839983C9
:10C4B000AA83BB837FC091FE55C0FC0120813181DE
:10C4C000428153816091B9127091BA128091BB126E
:10C4D0009091BC120F942ADB2B013C01F5012081C5
:10C4E0003181428153816091BD127091BE12809161
:10C4F000BF129091C0120F942ADB9B01AC01C301C3
:10C50000B2010F947CD7F801608371838283938397
:10C51000F70120813181428153816091C112709174
:10C52000C2128091C3129091C4120F942ADB6B0146
:10C530007C01F50120813181428153816091C512D6
:10C540007091C6128091C7129091C8120F942ADB85
:10C550009B01AC01C701B6010F947CD76883798336
:10C560008A839B8390FE26C02091A1123091A21253
:10C570004091A3125091A412F801608171818281CF
:10C5800093810F947CD7F8016083718382839383B6
:10C590002091A5123091A6124091A7125091A81295
:10C5A000688179818A819B810F947CD768837983A4
:10C5B0008A839B83DF91CF911F910F91FF90EF9022
:10C5C000DF90CF90BF90AF909F907F906F905F90E3
:10C5D0004F9008952F923F924F925F926F927F9269
:10C5E0008F929F92AF92BF92CF92DF92EF92FF9283
:10C5F0000F931F93CF93DF93CDB7DEB728970FB676
:10C60000F894DEBF0FBECDBF8C011B019E012F5FD2
:10C610003F4FAE014B5F5F4F23DF20E030E0A901C9
:10C620006D817E818F8198850F9455D887FF07C0D3
:10C630001D821E821F821886FF24F39401C0F12CF4
:10C6400020E030E040E850EC69817A818B819C8168
:10C650000F9455D887FF0AC080E090E0A0E8B0ECC6
:10C6600089839A83AB83BC83FF24F39420E030E07A
:10C670004FE753E46D817E818F8198850F9458DA5E
:10C68000181654F480E090E0AFE7B3E48D839E8306
:10C69000AF83B887FF24F39420E030E042E553E411
:10C6A00069817A818B819C810F9458DA18164CF439
:10C6B00080E090E0A2E5B3E489839A83AB83BC83F6
:10C6C00003C0FF2009F483C0C980DA80EB80FC80BE
:10C6D0008D809E80AF80B8847090C91271100BC09D
:10C6E000F80180829182A282B382F101C082D1825C
:10C6F000E282F3826AC070FE1CC02091A1123091C8
:10C70000A2124091A3125091A412C501B4010F943A
:10C710007BD74B015C012091A5123091A61240916C
:10C72000A7125091A812C701B6010F947BD76B01D5
:10C730007C0171FE4AC02091A9123091AA12409149
:10C74000AB125091AC12C501B4010F942ADB2B013E
:10C750003C012091AD123091AE124091AF12509138
:10C76000B012C701B6010F942ADB9B01AC01C301D3
:10C77000B2010F947CD7F801608371838283938325
:10C780002091B1123091B2124091B3125091B41273
:10C79000C501B4010F942ADB4B015C012091B51255
:10C7A0003091B6124091B7125091B812C701B6013C
:10C7B0000F942ADB9B01AC01C501B4010F947CD717
:10C7C000F1016083718382839383FF24F3948F2D1F
:10C7D00028960FB6F894DEBF0FBECDBFDF91CF9184
:10C7E0001F910F91FF90EF90DF90CF90BF90AF908F
:10C7F0009F908F907F906F905F904F903F902F9081
:10C800000895682F87EF9FE00D9477E40895FC0169
:10C810002491222341F03091C00035FFFCCF2093BA
:10C82000C6000196F4CF22E030E088EE99E0EACA33
:10C83000FC012491222341F03091C00035FFFCCF50
:10C840002093C6000196F4CF2AE030E088EE99E00C
:10C8500020CACF9365EB73E088EE99E0D3D9C1E0AD
:10C86000C093B1026FEF89E69FE00F9477E4C09325
:10C87000DE02CF91089565EC73E088EE99E0C2D9AD
:10C880001092B10260E089E69FE00F9477E4109285
:10C89000DE02089586ED93E09F938F930F94CDE190
:10C8A0000F94CF3981E00F94BFB40F94F96A82E0FE
:10C8B0000F94F8B186E69FE00F9465E461E0680F9D
:10C8C00086E69FE00F9477E481E00F94BFB482E0A6
:10C8D0000F94F8B1E0917F0BF0E0EE0FFF1FE559E8
:10C8E000F948859194910F94116C61E08FE19FE07C
:10C8F0000E94F2DD61E089E19FE00E94F2DD0F908D
:10C900000F9061E08BE09FE00C94F2DD1092BF0B82
:10C9100060E08DEB9BE00E9444D781E08093B10200
:10C920000895EF92FF920F931F93CF93DF931F927F
:10C93000CDB7DEB789830F94F96A8981823009F413
:10C9400068C0B4F5882309F442C0813009F0F4C00E
:10C950009FB7F894809102018460809302019FBF89
:10C96000EFEFF1EE24E0E150F0402040E1F700C0AD
:10C9700000009FB7F894809102018B7F80930201A1
:10C980009FBF40E050E0BA018DEE9FE00F9489E434
:10C9900040E050E0BA0181EF9FE00F9489E40F90EE
:10C9A000DF91CF911F910F91FF90EF900D94C8935D
:10C9B000833009F45CC0843009F0BEC00F90DF9171
:10C9C000CF911F910F91FF90EF900D94B1BC9FB745
:10C9D000F894809102018460809302019FBF2FEF41
:10C9E00081EE94E0215080409040E1F700C00000CB
:10C9F0009FB7F894809102018B7F809302019FBFC3
:10CA00000F90DF91CF911F910F91FF90EF900D94B8
:10CA1000A26B0F94A26B80EFF4DE1092DE1B1092DB
:10CA2000DD1B6091DF1B84EC9FE00F9477E46DEDDC
:10CA30007BE181EC9FE00F94276B9FB7F894809186
:10CA400002018460809302019FBF8FEF91EEE4E0CA
:10CA500081509040E040E1F700C000009FB7F8949B
:10CA6000809102018B7F809302019FBF65C08DEF93
:10CA70009EE00F9454824CEE5EE062E081E00F9401
:10CA80004D989FB7F89480910201846080930201D1
:10CA90009FBFFFEF21EE84E0F15020408040E1F79E
:10CAA00000C000009FB7F894809102018B7F8093B3
:10CAB00002019FBF1092E80A1092E70A45EE5EE07D
:10CAC00063E083E00F944D984091E70A5091E80AA3
:10CAD00063E083E00F94046BE12CF12C09E210E099
:10CAE0006FEFC7010F9495E4C701B8010F9419DDEA
:10CAF000892BD9F48091E70A9091E80A01969093E6
:10CB0000E80A8093E70A4EED5EE063E083E00F946D
:10CB10004D984091E70A5091E80A63E083E00F9452
:10CB2000046B8CED9EE00F9454829FEFE91AF90A92
:10CB3000E114E0E1FE06A1F60F90DF91CF911F9185
:10CB40000F91FF90EF90089569ED7AE08CEA9EE0F6
:10CB50000D94A0E18F929F92AF92BF92CF92DF92FD
:10CB6000EF92FF928091DF1B81119DC00F947ECFC9
:10CB70006B017C0120911002222309F48CC04091AA
:10CB80001502509116024130510509F484C080917C
:10CB9000110290911202A0911302B0911402460169
:10CBA0005701881A990AAA0ABB0A30E0A8EEB3E036
:10CBB0000F9470DD86169706A806B9060CF473C0AC
:10CBC0004430510559F13CF4423051050CF463C036
:10CBD000E4E6FFE00EC04530510509F05CC0E4E634
:10CBE000FFE042C09091C00095FFFCCF8093C6004B
:10CBF000319684918111F6CFE6EFFDE08491882390
:10CC000041F09091C00095FFFCCF8093C600319613
:10CC1000F5CF8091C00085FFFCCF3AC0E4E6FFE08D
:10CC20008491882341F09091C00095FFFCCF8093C0
:10CC3000C6003196F5CFE0EEFDE08491882341F007
:10CC40009091C00095FFFCCF8093C6003196F5CF40
:10CC50008091C00085FFFCCF1BC09091C00095FF64
:10CC6000FCCF8093C600319684918111F6CFE9EC18
:10CC7000FDE08491882341F09091C00095FFFCCFA6
:10CC80008093C6003196F5CF8091C00085FFFCCF20
:10CC90008AE08093C600C0921102D0921202E09204
:10CCA0001302F0921402FF90EF90DF90CF90BF90AC
:10CCB000AF909F908F90089580E1EAE4FBE0A5E1BA
:10CCC000BBE001900D928A95E1F708954F925F9233
:10CCD0006F927F928F929F92AF92BF92CF92DF928C
:10CCE000EF92FF92CF93DF9300D01F92CDB7DEB7C4
:10CCF0000F94CF398BE440D9882391F07FD96B0111
:10CD00007C0120E030E0A9010F9458DA87FD08C0CB
:10CD1000C092B213D092B313E092B413F092B51351
:10CD200082E52AD9882359F069D96B017C0120E07A
:10CD300030E0A9010F9455D887FF83C006C0C12CED
:10CD4000D12CE0E8EE2EEFEBFE2E84E415D98823FB
:10CD500021F054D94B015C0106C0812C912C70E864
:10CD6000A72E7FEBB72E87E507D9882321F046D978
:10CD70002B013C0106C0412C512C60E8662E6FEB64
:10CD8000762E88E4F9D8882331F038D969837A83FC
:10CD90008B839C8308C080E090E0A0E8BFEB898390
:10CDA0009A83AB83BC8320E030E0A901C501B401C4
:10CDB0000F9458DA87FD45C020E030E0A901C30197
:10CDC000B2010F9458DA87FD3CC020E030E0A901A1
:10CDD00069817A818B819C810F9458DA87FD31C0FB
:10CDE00020E030E0A901C501B4010F9455D8882393
:10CDF00091F120E030E040E05FE3C501B4010F9421
:10CE00002ADB6B017C0129813A814B815C81C30162
:10CE1000B2010F942ADB4B015C01A7019601C70107
:10CE2000B6010F942ADB2BED3FE049E450E40F9468
:10CE30002ADB9B01AC01C501B4010F945CD86B01E6
:10CE40007C0120E030E0A901C701B6010F9458DA57
:10CE500087FF04C00BC0C12CD12C7601C092AE1349
:10CE6000D092AF13E092B013F092B113E4E6FFE07A
:10CE70008491882341F09091C00095FFFCCF80936E
:10CE8000C6003196F5CFE2E8FAE08491882341F0BC
:10CE90009091C00095FFFCCF8093C6003196F5CFEE
:10CEA0004091B2135091B3136091B4137091B513C4
:10CEB00022E030E088EE99E00E94025F8091C0009D
:10CEC00085FFFCCF8AE08093C600ECE7FAE084910E
:10CED000882341F09091C00095FFFCCF8093C6005D
:10CEE0003196F5CFC090AE13D090AF13E090B01351
:10CEF000F090B11320E030E0A901C701B6010F9412
:10CF000055D8882369F022E030E0B701A60188EE09
:10CF100099E00E94025F8091C00085FFFCCF11C0A4
:10CF2000E7E7FAE08491882341F09091C00095FFF3
:10CF3000FCCF8093C6003196F5CF8091C00085FF6D
:10CF4000FCCF8AE08093C6000F900F900F900F9057
:10CF5000DF91CF91FF90EF90DF90CF90BF90AF9097
:10CF60009F908F907F906F905F904F9008952F9239
:10CF70003F924F925F926F927F928F929F92AF9269
:10CF8000BF92CF92DF92EF92FF920F931F93CF93B6
:10CF9000DF931F92CDB7DEB70F94F96AEFE1FDE79B
:10CFA0004591549161E080E00F944D9881E00F9499
:10CFB00054308983E7E2FFE0E4918E2F9927819531
:10CFC0000CF490951C0184E00F948855A2E5BBE019
:10CFD0001D921D921D921C921397EEE4FBE020819E
:10CFE000318142815381AAE4BBE06D917D918D91A5
:10CFF0009C91F6E5CF2EFBE0DF2EE12CF12C870192
:10D000000F94CE2C59DE8CE39FE00E94145F2DEC30
:10D010003CEC4CE85FE30F942ADB4B015C01B1016F
:10D02000882777FD8095982F0F94F7D89B01AC0146
:10D03000C501B4010F942ADBEDE1FBE020813181D1
:10D04000428153810F947CD72B013C01ADE1BBE0C1
:10D050006D937D938D939C931397E0E6F2E060814E
:10D0600071818281938160930C0270930D02809391
:10D070000E0290930F0220E030E040E752E40F945C
:10D080005CD84B015C01A9E1BBE02D913D914D9134
:10D090005C91E5E1FBE06081718182819381A6E38F
:10D0A000BBE0BF93AF93A1E2CA2EABE0DA2E8301BF
:10D0B00072010F94202082E00F94FD520F94CF391B
:10D0C0000F94085680E00F945430A2E5BBE01D9207
:10D0D0001D921D921C921397EEE4FBE0208131819A
:10D0E00042815381AAE4BBE06D917D918D919C9129
:10D0F000B6E5CB2EBBE0DB2EE12CF12C87010F94A3
:10D10000CE2CDADD8AE0829DB001839D700D112462
:10D11000882777FD8095982F0F94F7D8EDE1FBE0F5
:10D1200020813181428153810F947CD72B013C01B6
:10D13000ADE1BBE06D937D938D939C93139720E0BD
:10D1400030E040E05FE3E0E6F2E0608171818281FF
:10D1500093810F942ADB60930C0270930D028093ED
:10D160000E0290930F0220E030E040E752E40F946B
:10D170005CD84B015C01A9E1BBE02D913D914D9143
:10D180005C91E5E1FBE06081718182819381A6E39E
:10D19000BBE0BF93AF9311E2C12E1BE0D12E830100
:10D1A00072010F9420200F94CF3989810F9454304D
:10D1B00080E090E0A4E5B3E4E2E5FBE080839183C6
:10D1C000A283B383AEE4BBE02D913D914D915C9180
:10D1D000EAE4FBE0608171818281938106E5C02EE3
:10D1E0000BE0D02EE12CF12C04E513E40F94CE2CAF
:10D1F00081E00F900F900F900F900F90DF91CF91E3
:10D200001F910F91FF90EF90DF90CF90BF90AF9064
:10D210009F908F907F906F905F904F903F902F9056
:10D2200008952F923F924F925F926F927F928F92CA
:10D230009F92AF92BF92CF92DF92EF92FF920F93A5
:10D240001F93CF93DF93CDB7DEB729970FB6F8942E
:10D25000DEBF0FBECDBF3C0181E00F9454308F8301
:10D2600082E06816710408F081C2F301EB5DF04FB3
:10D27000E491D301AA0FBB1FAA0FBB1FBA83A983D6
:10D28000A85ABD4FBE83AD838D919D910D90BC91E9
:10D29000A02D80930C0290930D02A0930E02B093E8
:10D2A0000F0281E0062C01C0880F0A94EAF70F9460
:10D2B0008855E981FA81E65BF44FF987E8871082A7
:10D2C000118212821382E090520BF090530B009166
:10D2D000540B1091550B20914E0B30914F0B4091F8
:10D2E000500B5091510B60914A0B70914B0B8091F8
:10D2F0004C0B90914D0BE6E5CE2EEBE0DE2E0F941D
:10D30000CE2CE981FA81EB5EF44F2F0180E090E0B2
:10D31000A0E4B0E480839183A283B38320E030E073
:10D3200040E752E460910C0270910D0280910E0270
:10D3300090910F020F945CD84B015C01E0901D0BA3
:10D34000F0901E0B00911F0B1091200B2091190BD8
:10D3500030911A0B40911B0B50911C0B6091150BD7
:10D360007091160B8091170B9091180BF6E32F2EEE
:10D37000FBE03F2E3F922F92A1E2CA2EABE0DA2EC5
:10D380000F9420200F94CF390F943C3080E00F94FD
:10D390005430A885B9851D921D921D921C92139739
:10D3A000E090520BF090530B0091540B1091550BE1
:10D3B00020914E0B30914F0B4091500B5091510BDF
:10D3C00060914A0B70914B0B80914C0B90914D0BDF
:10D3D000B6E5CB2EBBE0DB2E0F94CE2C80E090E0A8
:10D3E000A0E8BFEBF20180839183A283B38320E0A6
:10D3F00030E040E752E460910C0270910D028091A0
:10D400000E0290910F020F945CD84B015C01E090EA
:10D410001D0BF0901E0B00911F0B1091200B209103
:10D42000190B30911A0B40911B0B50911C0B609102
:10D43000150B7091160B8091170B9091180B3F9262
:10D440002F92E1E2CE2EEBE0DE2E0F9420200F94FF
:10D45000CF3981E00F94543089819A818C5C904F50
:10D460000E94145F2DEC3CEC4CE85FEB0F942ADB40
:10D47000D2016D937D938D939C93139720E030E0C0
:10D4800040E752E460910C0270910D0280910E020F
:10D4900090910F020F945CD84B015C01E0901D0B42
:10D4A000F0901E0B00911F0B1091200B2091190B77
:10D4B00030911A0B40911B0B50911C0B6091150B76
:10D4C0007091160B8091170B9091180B3F922F9231
:10D4D0000F9420200F94CF390F943C3080E00F94AC
:10D4E0005430E885F9851082118212821382E0900F
:10D4F000520BF090530B0091540B1091550B20914F
:10D500004E0B30914F0B4091500B5091510B60914D
:10D510004A0B70914B0B80914C0B90914D0BF6E5A3
:10D52000CF2EFBE0DF2E0F94CE2C80E090E0A0E227
:10D53000B1E4F20180839183A283B38320E030E0E1
:10D5400040E752E460910C0270910D0280910E024E
:10D5500090910F020F945CD84B015C01E0901D0B81
:10D56000F0901E0B00911F0B1091200B2091190BB6
:10D5700030911A0B40911B0B50911C0B6091150BB5
:10D580007091160B8091170B9091180B3F922F9270
:10D59000A1E2CA2EABE0DA2E0F9420200F94CF39EF
:10D5A0000F943C3081E00F94543080E090E0A0E78D
:10D5B000B1ECF20180839183A283B38320E030E059
:10D5C00040E05FE3AD81BE816D917D918D919C9135
:10D5D0000F942ADB60930C0270930D0280930E026D
:10D5E00090930F0220E030E040E752E40F945CD8C3
:10D5F0004B015C01E0901D0BF0901E0B00911F0B86
:10D600001091200B2091190B30911A0B40911B0B9C
:10D6100050911C0B6091150B7091160B8091170B9C
:10D620009091180B3F922F920F9420200F94CF3996
:10D63000C3010E941A5FF301E55CF44F81E080832F
:10D640000F9408560F943C3080E00F9454302AE039
:10D6500037ED43E25FE3E885F9856081718182817E
:10D6600093810F947BD7A885B9856D937D938D9316
:10D670009C931397E090520BF090530B0091540B36
:10D680001091550B20914E0B30914F0B4091500B48
:10D690005091510B60914A0B70914B0B80914C0B48
:10D6A00090914D0BB6E5CB2EBBE0DB2E0F94CE2C2C
:10D6B0002AE037ED43E25FE3E885F9856081718117
:10D6C000828193810F947CD7A885B9856D937D93D2
:10D6D0008D939C931397F20160837183828393836C
:10D6E0002AE939E949E95EE360910C0270910D0283
:10D6F00080910E0290910F020F942ADB20E030E01F
:10D7000040E752E40F945CD84B015C01E0901D0BA4
:10D71000F0901E0B00911F0B1091200B2091190B04
:10D7200030911A0B40911B0B50911C0B6091150B03
:10D730007091160B8091170B9091180B3F922F92BE
:10D74000E1E2CE2EEBE0DE2E0F9420200F94CF39B5
:10D7500010920C0210920D0210920E0210920F0203
:10D760000FB6F894DEBF0FBECDBF62C192E069165E
:10D77000710409F05DC1E7E2FFE074901092520B72
:10D780001092530B1092540B1092550B20914E0B8C
:10D7900030914F0B4091500B5091510B60914A0BBF
:10D7A00070914B0B80914C0B90914D0BF6E5CF2E69
:10D7B000FBE0DF2EE12CF12C87010F94CE2C8CE3C3
:10D7C0009FE00E94145F4B015C01672D772767FD86
:10D7D0007095872F972F0F94F7D82B013C0120E0ED
:10D7E00030E040EC5FE3C501B4010F942ADBA301F4
:10D7F00092010F942ADB69837A838B839C836093E5
:10D800001D0B70931E0B80931F0B9093200B609148
:10D810006002709161028091620290916302609354
:10D820000C0270930D0280930E0290930F0220E081
:10D8300030E040E752E40F945CD84B015C0120914A
:10D84000190B30911A0B40911B0B50911C0B6091DE
:10D85000150B7091160B8091170B9091180BA6E386
:10D860002A2EABE03A2E3F922F92B1E2CB2EBBE0B4
:10D87000DB2EE980FA800B811C810F9420200F940D
:10D88000CF391092520B1092530B1092540B1092EE
:10D89000550B20914E0B30914F0B4091500B5091F6
:10D8A000510B60914A0B70914B0B80914C0B9091F6
:10D8B0004D0B16E5C12E1BE0D12EE12CF12C87017A
:10D8C0000F94CE2C80E39FE00E94145F9058A30138
:10D8D00092010F942ADB69837A838B839C83609304
:10D8E0001D0B70931E0B80931F0B9093200B20E059
:10D8F00030E040E752E460910C0270910D0280919B
:10D900000E0290910F020F945CD84B015C012091A4
:10D91000190B30911A0B40911B0B50911C0B60910D
:10D92000150B7091160B8091170B9091180B3F926D
:10D930002F9201E2C02E0BE0D02EE980FA800B81FD
:10D940001C810F9420200F94CF3980E39FE00E9428
:10D95000145F9B01AC010F947CD7A30192010F943B
:10D960002ADB2B013C0160931D0B70931E0B8093EF
:10D970001F0B9093200B20E030E040E05FE36091CC
:10D9800060027091610280916202909163020F9433
:10D990002ADB60930C0270930D0280930E02909329
:10D9A0000F0220E030E040E752E40F945CD84B01D6
:10D9B0005C012091190B30911A0B40911B0B509177
:10D9C0001C0B6091150B7091160B8091170B9091A9
:10D9D000180B3F922F92830172010F9420200F9415
:10D9E000CF3982E090E00E941A5F8091520B9091B3
:10D9F000530BA091540BB091550B80931D0B90933A
:10DA00001E0BA0931F0BB093200B10920C021092D0
:10DA10000D0210920E0210920F020F943C3081E022
:10DA200080933D0B0F900F900F900F900F900F90E1
:10DA30008F8129960FB6F894DEBF0FBECDBFDF9160
:10DA4000CF911F910F91FF90EF90DF90CF90BF90FB
:10DA5000AF909F908F907F906F905F904F903F908E
:10DA60002F900D945430CF92DF92EF92FF920F934C
:10DA70001F9322D980E090E0D4DB81E090E0D1DBFD
:10DA8000E090520BF090530B0091540B1091550BFA
:10DA900020914E0B30914F0B4091500B5091510BF8
:10DAA00060914A0B70914B0B80914C0B90914D0BF8
:10DAB000F6E5CF2EFBE0DF2E0F94CE2C1F910F91B9
:10DAC000FF90EF90DF90CF900D943C300F947ECF7D
:10DAD0006093FC0A7093FD0A8093FE0A9093FF0AFC
:10DAE000089520E030E0A90168EB71E084E50F942F
:10DAF000D6D369E170E080E090E00F94ADCF84E58B
:10DB00000F94FAD664E170E080E090E00D94ADCF20
:10DB10007F928F929F92AF92BF92CF92DF92EF92BD
:10DB2000FF920F931F93CF93DF9300D01F92CDB737
:10DB3000DEB71092CB1A1092CA1A1092C91A10921C
:10DB4000C81A0F94F96A87E09EE00F9454828E0100
:10DB50000F5F1F4F7E0125E0E20EF11C88EE99E079
:10DB60000E941C5D8F3FEFEF9E07C1F3F801819388
:10DB70008F01EE15FF0591F789809A80AB80BC80FC
:10DB80008091C00085FFFCCF8BE28093C600C12C42
:10DB9000D12C7601ABE27A2E80917E0B882309F49A
:10DBA00050C00AE81AE0C814D904EA04FB04A1F042
:10DBB00088EE99E00E941C5D8F3FFFEF9F07C1F345
:10DBC0002FEFC21AD20AE20AF20AF80181938F01FA
:10DBD000FAE00A3C1F0739F76AE87AE08DEB9BE030
:10DBE0000E9411D68091C00085FFFCCF7092C600C4
:10DBF0000F94BB46C814D904EA04FB0469F671DF2C
:10DC000060E08DEB9BE00E9444D710927E0BE1E632
:10DC1000FCE785919491FC012491222341F03091FD
:10DC2000C00035FFFCCF2093C6000196F4CF809151
:10DC3000C00085FFFCCF8AE08093C60080E090E0C2
:10DC400000C00F900F900F900F90DF91CF911F9118
:10DC50000F91FF90EF90DF90CF90BF90AF909F908B
:10DC60008F907F9008952F923F924F925F926F9284
:10DC70007F928F929F92AF92BF92CF92DF92EF925C
:10DC8000FF920F931F93CF93DF931F921F92CDB7F5
:10DC9000DEB7382E811112C01092C91A1092C81A1C
:10DCA0001092CB1A1092CA1A1092CD1A1092CC1A56
:10DCB0001092CF1A1092CE1A0F944E6B80E00F94F0
:10DCC000BFB48AEC92E10F94BB140E9422F60F9429
:10DCD0000C1410923B0B10923C0B10923D0B81E008
:10DCE0000E94685FE0917F0BF0E0EE0FFF1FE55DA3
:10DCF000F14885919491BE016F5F7F4F0F94FEB400
:10DD0000B2DE35D9882309F471C1E0DE311046C096
:10DD100084E090E09093160280931502E7E0F8E724
:10DD20008591949140E060E00F94B7B6882331F07C
:10DD3000E9EDF9E7859194910F94A7BEE0917F0BEF
:10DD4000F0E0EE0FFF1FEF56F548859194910F9488
:10DD5000A7BE82E090E09093160280931502E091B6
:10DD60007F0BF0E0EE0FFF1FE35BF348859194918A
:10DD7000BE016F5F7F4F0F94FEB441E050E062E060
:10DD800080E00F94046BE0917F0BF0E0EE0FFF1F3B
:10DD9000ED5BF348859194910F94548280E090E07C
:10DDA000A0EAB0E48093520B9093530BA093540BD2
:10DDB000B093550B20E030E040E252E46091600205
:10DDC0007091610280916202909163020F945CD81D
:10DDD0004B015C0120914E0B30914F0B4091500B49
:10DDE0005091510B60914A0B70914B0B80914C0BF1
:10DDF00090914D0BE6E3FBE0FF93EF93E6E5CE2E2B
:10DE0000EBE0DE2EE12CF12C00EA10E40F94202050
:10DE10000F94CF3986E50E94BC5F0F900F90882346
:10DE200061F0E0918C10F0918D108181893039F092
:10DE30008F7D41F00E94D25F03C01A8205C081E04D
:10DE40008A8302C0A1E0AA833320B1F00E94965FCA
:10DE50000E9477F60E9493F80F94670D882309F4C7
:10DE6000C1C087EF9FE00F9465E4803F09F0BAC01E
:10DE700081E00E940164B6C08FEF0E94016460E0FF
:10DE800070E088EF9FE00F9491E41982BE016F5F0C
:10DE90007F4F8A810F94380A3C010E94965F212CA3
:10DEA000312C10EA412E10E4512E2092520B309268
:10DEB000530B4092540B5092550B20E030E040E25F
:10DEC00052E46091600270916102809162029091CF
:10DED00063020F945CD84B015C0120914E0B309192
:10DEE0004F0B4091500B5091510B60914A0B709128
:10DEF0004B0B80914C0B90914D0BA6E3BBE0BF9375
:10DF0000AF9306E5C02E0BE0D02E820171010F9475
:10DF100020200F94CF390F900F9077FC47C01982C3
:10DF20008AEC92E10F94BB140E94E9F581E00E9413
:10DF3000685F99DDAE014F5F5F4F6A8181E00F94AA
:10DF40008D0F3C010E94965F2092520B3092530B32
:10DF50004092540B5092550B20E030E040E252E4E6
:10DF600060916002709161028091620290916302FF
:10DF70000F945CD84B015C0120914E0B30914F0BFC
:10DF80004091500B5091510B60914A0B70914B0B8B
:10DF900080914C0B90914D0BA6E3BBE0BF93AF93E8
:10DFA0000F9420200F94CF390F900F906981C301F7
:10DFB0000F9411BF77FC16C086EE0E9401648FE5B6
:10DFC0009FE00F9465E4813059F0E0917F0BF0E021
:10DFD000EE0FFF1FEB5EF148859194910F94A7BE61
:10DFE00011E001C010E00F94085601C010E081E07C
:10DFF0000F94BFB4812F0F900F90DF91CF911F919D
:10E000000F91FF90EF90DF90CF90BF90AF909F90D7
:10E010008F907F906F905F904F903F902F900895DA
:10E020008F929F92AF92BF92CF92DF92EF92FF9228
:10E030000F931F93CF93DF93159881E08093730B19
:10E0400082E090E09093710B8093700BE0917F0BD6
:10E05000F0E0EE0FFF1FE557F448859194910F947F
:10E06000116C20E030E04CE852E46091560B709166
:10E07000570B8091580B9091590B0F947CD760935C
:10E08000560B7093570B8093580B9093590BE0905D
:10E09000520BF090530B0091540B1091550B2091A3
:10E0A0004E0B30914F0B4091500B5091510B6091A2
:10E0B0004A0B70914B0B80914C0B90914D0BC6E32A
:10E0C000DBE0DF93CF93812C912CE0ECAE2EE0E4EB
:10E0D000BE2EF6E5CF2EFBE0DF2E0F94202020E0B1
:10E0E00030E048EC51E46091560B7091570B8091F1
:10E0F000580B9091590B0F947CD76093560B7093EB
:10E10000570B8093580B9093590BE090520BF09063
:10E11000530B0091540B1091550B20914E0B3091E5
:10E120004F0B4091500B5091510B60914A0B7091E5
:10E130004B0B80914C0B90914D0BDF93CF93812C27
:10E14000912CA0E8AA2EAFE3BA2E0F9420200F94B2
:10E15000CF390F900F900F900F908091DF1B882385
:10E1600031F181E00F94BFB482E00F94F8B1E091F7
:10E170007F0BF0E0EE0FFF1FE559F9488591949170
:10E180000F94116C1092720B1092730B1092710B12
:10E190001092700BDF91CF911F910F91FF90EF9034
:10E1A000DF90CF90BF90AF909F908F900895809117
:10E1B000720B8823B1F2E0917F0BF0E0EE0FFF1FAE
:10E1C000EB59F3488591949141E060E00F94B7B624
:10E1D00091E0811101C090E0C6E3DBE09111C1CF75
:10E1E00081E00F94BFB482E00F94F8B120E030E0FA
:10E1F00048EC51E46091560B7091570B8091580B8D
:10E200009091590B0F947CD76093560B7093570BDA
:10E210008093580B9093590BE090520BF090530B56
:10E220000091540B1091550B20914E0B30914F0BD8
:10E230004091500B5091510B60914A0B70914B0BD8
:10E2400080914C0B90914D0BDF93CF93812C912CAF
:10E25000E0E8AE2EEFE3BE2EF6E5CF2EFBE0DF2E9C
:10E260000F9420200F94CF39E0917F0BF0E0EE0F58
:10E27000FF1FEB59F3488591949141E060E00F94C2
:10E28000B7B60F900F9081116CCFAACF0F947ECFAD
:10E290006093FC0A7093FD0A8093FE0A9093FF0A34
:10E2A000E0919610F0919710E856FF4E80818130F2
:10E2B000B9F4EBE9FAE785919491FC0124912223CA
:10E2C00041F03091C00035FFFCCF2093C60001968D
:10E2D000F4CF8091C00085FFFCCF8AE08093C60018
:10E2E000089588EE99E00E94385DE7EDF9E78591A1
:10E2F0009491FC012491222341F03091C00035FF1C
:10E30000FCCF2093C6000196F4CF40917C10509131
:10E310007D1060917E1070917F104F5F5F4F6F4F47
:10E320007F4F2AE030E088EE99E00E94D75D80912F
:10E33000C00085FFFCCF8AE08093C600A7CF8F92F4
:10E340009F92AF92BF92CF92DF92EF92FF920F9384
:10E350001F93CF93DF93B9EBEB2EB5E0FB2E0AE4CE
:10E360001BE0C5E1DBE085EBC82E8BE0D82EF70182
:10E3700081917F010E94BC5F882319F10E9429606E
:10E380004B015C01F6018081811103C06091000B9B
:10E3900001C061E070E080E090E00F94F7D8F801F0
:10E3A00020813181428153810F942ADB9B01AC0192
:10E3B000C501B4010F947CD7688379838A839B83DA
:10E3C00009C0F80180819181A281B38188839983FA
:10E3D000AA83BB830C5F1F4F2496FFEFCF1ADF0A7F
:10E3E0008DEBE81685E0F80611F686E40E94BC5F26
:10E3F0008823D9F00E9429606B017C016093050B92
:10E400007093060B8093070B9093080B20E030E08D
:10E41000A9010F9458DA181644F4C0920C02D09255
:10E420000D02E0920E02F0920F02DF91CF911F9148
:10E430000F91FF90EF90DF90CF90BF90AF909F90A3
:10E440008F9008957CDF89E40E94BC5F882359F097
:10E450000E9429606093090B70930A0B80930B0B49
:10E4600090930C0B08C01092090B10920A0B10929B
:10E470000B0B10920C0B8AE40E94BC5F882359F0AE
:10E480000E94296060930D0B70930E0B80930F0B0D
:10E490009093100B089510920D0B10920E0B10928A
:10E4A0000F0B1092100B0895CF92DF92EF92FF9214
:10E4B000CF93DF93EC01BC016C5F7F4F0E94EA6257
:10E4C00020E030E0A90160913C0270913D02809112
:10E4D0003E0290913F020F947CD76B017C019B011F
:10E4E000AC01688579858A859B850F9455D887FF0F
:10E4F00004C0C886D986EA86FB86C0903002D090D8
:10E500003102E0903202F0903302A7019601688553
:10E5100079858A859B850F9458DA181624F4C88665
:10E52000D986EA86FB86DF91CF91FF90EF90DF904E
:10E53000CF9008952F923F924F925F926F927F9269
:10E540008F929F92AF92BF92CF92DF92EF92FF9203
:10E550000F931F93CF93DF93CDB7DEB7AB970FB673
:10E56000F894DEBF0FBECDBF9F878E87798B688BF7
:10E570005B8B4A8B3D8B2C8B1F8B0E8BED82DC01D2
:10E580008D909D90AD90BC9040904A0B50904B0B5D
:10E5900060904C0B70904D0BDB018D919D910D9017
:10E5A000BC91A02D88879987AA87BB87C0904E0B06
:10E5B000D0904F0BE090500BF090510B2091520BEC
:10E5C0003091530B4091540B5091550BEA89FB89C4
:10E5D00060817181828193810F947BD7688F798F5D
:10E5E0008A8F9B8F8091CA12811173C0AE89BF89B7
:10E5F0008D909D90AD90BC90EA89FB89E080F18080
:10E6000002811381A889B9892D913D914D915C9129
:10E61000EE85FF856081718182819381FE0135964F
:10E62000FF93EF93CC88DD880F942020EE85FF8543
:10E6300080819181A281B38180934A0B90934B0B8F
:10E64000A0934C0BB0934D0BE889F989808191819F
:10E65000A281B38180934E0B90934F0BA093500BEC
:10E66000B093510BEA89FB8980819181A281B381AA
:10E670008093520B9093530BA093540BB093550B74
:10E68000EC89FD8980819181A281B3818093560BB1
:10E690009093570BA093580BB093590B0F900F907A
:10E6A000AB960FB6F894DEBF0FBECDBFDF91CF9112
:10E6B0001F910F91FF90EF90DF90CF90BF90AF90A0
:10E6C0009F908F907F906F905F904F903F902F9092
:10E6D0000895A3019201C501B4010F947BD72B01CA
:10E6E0003C0120E030E0A9010F9458DA53014201C7
:10E6F000181624F0B7FAB094B7F8B094A7019601B1
:10E70000688579858A859B850F947BD7688779870B
:10E710008A879B8720E030E0A9010F9458DA28858A
:10E7200039854A855B8518160CF05058C501B4012F
:10E730000F947CD76B017C0120E030E0A9010F949D
:10E7400058DA18160CF052CF20E030E040EF51E4D8
:10E75000C701B6010F945CD80F9442D80F94C4D867
:10E760007D876C87623071050CF440CF2091560B89
:10E770003091570B4091580B5091590BAC89BD8982
:10E780006D917D918D919C910F947BD76C8F7D8F36
:10E790008E8F9F8F22242394312C8C859D85AA27D0
:10E7A00097FDA095BA2F88A799A7AAA7BBA7DE01B6
:10E7B0001596BF83AE83B101882777FD8095982F8A
:10E7C0000F94F7D86B017C0168A579A58AA59BA554
:10E7D0000F94F7D89B01AC01C701B6010F945CD828
:10E7E0006B017C01EE89FF8980809180A280B380DB
:10E7F0002C8D3D8D4E8D5F8D0F942ADB9B01AC01DE
:10E800006091560B7091570B8091580B9091590B5A
:10E810000F947CD769837A838B839C83288D398D71
:10E820004A8D5B8DC701B6010F942ADB2091520BF4
:10E830003091530B4091540B5091550B0F947CD752
:10E8400068A379A38AA39BA3288539854A855B851C
:10E85000C701B6010F942ADB20914E0B30914F0B6C
:10E860004091500B5091510B0F947CD76CA37DA31A
:10E870008EA39FA3A3019201C701B6010F942ADBC7
:10E8800020914A0B30914B0B40914C0B50914D0B0A
:10E890000F947CD7FF81FF932E812F93DE01119679
:10E8A0006D01E8A0F9A00AA11BA12CA13DA14EA1D8
:10E8B0005FA10F942020BFEF2B1A3B0A0F900F90FF
:10E8C000EC85FD852E163F0609F075CF8FCE4F9251
:10E8D0005F926F927F928F929F92AF92BF92CF92F0
:10E8E000DF92EF92FF920F931F93CF93DF93CDB7F9
:10E8F000DEB728970FB6F894DEBF0FBECDBF85E117
:10E900009BE0D2DD0F947ECF6093FC0A7093FD0AEA
:10E910008093FE0A9093FF0A8091150B9091160B3D
:10E92000A091170BB091180B8D839E83AF83B8878E
:10E930009C01AD0160914A0B70914B0B80914C0B87
:10E9400090914D0B0F9455D8811197C04090190BA1
:10E9500050901A0B60901B0B70901C0BA30192013E
:10E9600060914E0B70914F0B8091500B9091510B19
:10E970000F9455D8811181C020E030E040E752E487
:10E9800060910C0270910D0280910E0290910F0225
:10E990000F945CD84B015C01E0901D0BF0901E0BB6
:10E9A00000911F0B1091200B86E39BE09F938F93A8
:10E9B00021E2C22E2BE0D22EA30192016D817E8135
:10E9C0008F8198850F9420200F900F908091150BC8
:10E9D0009091160BA091170BB091180B80934A0BD6
:10E9E00090934B0BA0934C0BB0934D0B8091190B54
:10E9F00090911A0BA0911B0BB0911C0B80934E0BA6
:10EA000090934F0BA093500BB093510B80911D0B23
:10EA100090911E0BA0911F0BB091200B8093520B75
:10EA20009093530BA093540BB093550B8091210BF3
:10EA30009091220BA091230BB091240B8093560B45
:10EA40009093570BA093580BB093590B28960FB681
:10EA5000F894DEBF0FBECDBFDF91CF911F910F9114
:10EA6000FF90EF90DF90CF90BF90AF909F908F90EE
:10EA70007F906F905F904F900895E090360B60917B
:10EA8000560270915702882777FD8095982F0F9432
:10EA9000F7D820910C0230910D0240910E02509156
:10EAA0000F020F942ADB2EE333EC4EE259E30F946E
:10EAB0002ADB69837A838B839C838E010F5F1F4FD0
:10EAC00021E23BE04DE15BE069E17BE085E19BE039
:10EAD00031DD7CCF4F925F926F927F928F929F92A7
:10EAE000AF92BF92CF92DF92EF92FF920F931F935C
:10EAF000CF93C62FE091360BF0E0882309F4D9C0FC
:10EB0000DF01AE5CB44F8C918111AFC180914A0B93
:10EB100090914B0BA0914C0BB0914D0B8093150B2A
:10EB20009093160BA093170BB093180B80914E0B7C
:10EB300090914F0BA091500BB091510B8093190BFA
:10EB400090931A0BA0931B0BB0931C0B8091520B4C
:10EB50009091530BA091540BB091550B80931D0BCA
:10EB600090931E0BA0931F0BB093200BC090560BDD
:10EB7000D090570BE090580BF090590BC092210B9E
:10EB8000D092220BE092230BF092240BEE0FFF1F8A
:10EB9000EE0FFF1FE05CFD4F2081318142815381E8
:10EBA000662349F060912002709121028091220237
:10EBB0009091230208C060912402709125028091F7
:10EBC0002602909127020F945CD89B01AC01C701EB
:10EBD000B6010F947CD76093560B7093570B8093BC
:10EBE000580B9093590B86E59BE00F94792E8090FB
:10EBF0000C0290900D02A0900E02B0900F0220E047
:10EC000030E040E752E460911C0270911D02809157
:10EC10001E0290911F020F942ADB60930C027093E6
:10EC20000D0280930E0290930F02E091360BF0E0FC
:10EC3000EE5CF44F81E080834ADE20912E0B309110
:10EC40002F0B4091300B5091310B6091520B709112
:10EC5000530B8091540B9091550B0F947BD77B01F4
:10EC60008C016093520B7093530B8093540B9093D1
:10EC7000550B20914E0B30914F0B4091500B509102
:10EC8000510B60914A0B70914B0B80914C0B909102
:10EC90004D0BE6E5CE2EEBE0DE2E0F94CE2C17DEEC
:10ECA00080920C0290920D02A0920E02B0920F027E
:10ECB000DCC0EE5CF44F8081882309F4D6C08090DC
:10ECC0004A0B90904B0BA0904C0BB0904D0B809248
:10ECD000150B9092160BA092170BB092180B409048
:10ECE0004E0B50904F0B6090500B7090510B409218
:10ECF000190B50921A0B60921B0B70921C0B6091B7
:10ED0000520B7091530B8091540B9091550B609363
:10ED10001D0B70931E0B80931F0B9093200B009183
:10ED2000560B1091570B2091580B3091590B0093B3
:10ED3000210B1093220B2093230B3093240B209153
:10ED40002E0B30912F0B4091300B5091310B0F94C3
:10ED50007CD77B018C016093520B7093530B809393
:10ED6000540B9093550B36E5C32E3BE0D32EA301F5
:10ED70009201C501B4010F94CE2C1091360BCC2317
:10ED800089F02091260B3091270B4091280B509150
:10ED9000290B6091200270912102809122029091B2
:10EDA000230210C020912A0B30912B0B40912C0B89
:10EDB00050912D0B609124027091250280912602C2
:10EDC000909127020F947CD724E0129FF001112428
:10EDD000E05CFD4F20813181428153810F945CD8EA
:10EDE0009B01AC016091560B7091570B8091580BB1
:10EDF0009091590B0F947BD76093560B7093570BE0
:10EE00008093580B9093590B86E59BE00F94792ED5
:10EE1000C0900C02D0900D02E0900E02F0900F0214
:10EE200020E030E040E752E460911802709119024E
:10EE300080911A0290911B020F942ADB60930C02BE
:10EE400070930D0280930E0290930F02E091360BA7
:10EE5000F0E0EE5CF44F10823ADDC0920C02D092EA
:10EE60000D02E0920E02F0920F02CF911F910F91CE
:10EE7000FF90EF90DF90CF90BF90AF909F908F90DA
:10EE80007F906F905F904F900895AF92BF92CF9216
:10EE9000DF92EF92FF920F931F93CF93DF93D82FC0
:10EEA00020910D0B30910E0B40910F0B5091100BD8
:10EEB0006091090B70910A0B80910B0B90910C0BD8
:10EEC0000F9465DAC62F172F082FF92E609156027E
:10EED00070915702882777FD8095982F0F94F7D867
:10EEE00020910C0230910D0240910E0250910F02C0
:10EEF0000F942ADB20E030E040E752E40F945CD826
:10EF000020E030E048EC52E40F945CD82091360BBE
:10EF10002F93DF93FF920F931F93CF935B016C01AD
:10EF2000B2E0EB2E01E020E049E05BE065E17BE050
:10EF30008AE49BE00F94A0168091150B9091160B1C
:10EF4000A091170BB091180B80934A0B90934B0B29
:10EF5000A0934C0BB0934D0B8091190B90911A0B11
:10EF6000A0911B0BB0911C0B80934E0B90934F0BF9
:10EF7000A093500BB093510B80911D0B90911E0BE1
:10EF8000A0911F0BB091200B8093520B9093530BC9
:10EF9000A093540BB093550B8091210B9091220BB1
:10EFA000A091230BB091240B8093560B9093570B99
:10EFB000A093580BB093590B0F947ECF6093FC0A2B
:10EFC0007093FD0A8093FE0A9093FF0A0F900F90B2
:10EFD0000F900F900F900F90DF91CF911F910F9195
:10EFE000FF90EF90DF90CF90BF90AF900895CF93B8
:10EFF000DF931F92CDB7DEB78C01E0E7FAE0849192
:10F00000882341F09091C00095FFFCCF8093C6000B
:10F010003196F5CF70E04AE050E088EE99E00E942A
:10F02000165EF8940F94C743179A10923B0B169AEA
:10F0300010923C0B149AEAE6FFE08491882341F099
:10F040009091C00095FFFCCF8093C6003196F5CF1C
:10F05000EBE9FCE785919491FC012491222341F096
:10F060003091C00035FFFCCF2093C6000196F4CF4D
:10F070008091C00085FFFCCF8AE08093C600011517
:10F080001105E1F0F8018491F801882349F090918D
:10F09000C00095FFFCCF8093C60031968491F5CFD8
:10F0A0008091C00085FFFCCF8AE08093C600BE013E
:10F0B0006F5F7F4FC8010F94FEB40BC0E0917F0BD0
:10F0C000F0E0EE0FFF1FE354F448859194910F9404
:10F0D0003C6C789406E010E00150110951F068ECA6
:10F0E00070E080E090E00F94ADCF80E00F94F8B135
:10F0F000F3CFF894FFCFCF92DF92EF92FF920F936E
:10F100001F93CF93C82F80919210909193100397E3
:10F1100014F40E949EDF0F947ECF0091F80A1091A4
:10F12000F90A2091FA0A3091FB0AC090FC0AD090AB
:10F13000FD0AE090FE0AF090FF0A6C197D098E0925
:10F140009F09061717072807390740F4012B022BE0
:10F15000032B21F064E085EE97E049DF409108023F
:10F160005091090260910A0270910B02452B462BC7
:10F17000472B19F10F947ECF0091FC0A1091FD0AE4
:10F180002091FE0A3091FF0A601B710B820B930BDA
:10F19000009108021091090220910A0230910B029D
:10F1A000061717072807390740F49091B713809185
:10F1B000B613981302C0CC2349F0CF911F910F9141
:10F1C000FF90EF90DF90CF900D944E1E179A109203
:10F1D0003B0B169A10923C0B149AEFCF0F94C74337
:10F1E0008091EA0A811142C081E08093EA0A80910D
:10F1F0007C1090917D10A0917E10B0917F10809333
:10F20000781090937910A0937A10B0937B10EAE66F
:10F21000FFE08491882341F09091C00095FFFCCFDE
:10F220008093C6003196F5CFE1E9FCE78591949192
:10F23000FC012491222341F03091C00035FFFCCF26
:10F240002093C6000196F4CF8091C00085FFFCCFCB
:10F250008AE08093C600E0917F0BF0E0EE0FFF1F85
:10F26000E550F848859194910D94116C0895809122
:10F27000EA0A0895CF93DF93EC018091360B8093D7
:10F28000EB0A84E50E94BC5F811102C080E084C06B
:10F290000E9429600F94C9D86093EB0A6623B1F3EA
:10F2A000E4E6FFE08491882341F09091C00095FF4F
:10F2B000FCCF8093C6003196F5CFCD36D10509F449
:10F2C00035C064F4C836D105B1F0C936D10509F0AE
:10F2D00052C0E3E7FBE7A591B49124C0CA3DD10534
:10F2E00009F432C0CD3DD10509F045C0EDE5FBE79D
:10F2F000A591B4913DC0E5E7FBE785919491FC01B0
:10F300002491222309F437C03091C00035FFFCCF8F
:10F310002093C6000196F3CF9091C00095FFFCCFDB
:10F320008093C6008D918111F7CF25C0E1E7FBE7FF
:10F33000A591B4918D918823F1F09091C00095FF33
:10F34000FCCF8093C600F6CFEFE5FBE7A591B49123
:10F350008D91882381F09091C00095FFFCCF809320
:10F36000C600F6CF9091C00095FFFCCF8093C600F9
:10F370008D918111F7CF6091EB0A70E04AE050E087
:10F3800088EE99E00E940F5E8091C00085FFFCCF5F
:10F390008AE08093C60081E0DF91CF9108954F927B
:10F3A0005F926F927F928F929F92AF92BF92CF9215
:10F3B000DF92EF92FF92CF93DF9300D01F92CDB7F1
:10F3C000DEB72B013C0129833A834B835C838DEEAE
:10F3D0009FE00F9465E48F3F01F58EEE9FE00F9460
:10F3E00065E48F3FD1F48FEE9FE00F9465E48F3F8B
:10F3F000A1F480EF9FE00F9465E48F3F71F440E04B
:10F4000050E0BA018DEE9FE00F9489E440E050E0B7
:10F41000BA0181EF9FE00F9489E481EF9FE00F94A0
:10F420006DE44B015C018DEE9FE00F946DE46B0188
:10F430007C0169817A818B819C812CE330E040E002
:10F4400050E00F942CDDC20ED31EE41EF51EB70152
:10F45000A6018DEE9FE00F9489E4C301B20128EE6E
:10F4600033E040E050E00F942CDDBA01A901480DD3
:10F47000591D6A1D7B1D81EF9FE00F9489E4109256
:10F48000780B1092790B10927A0B10927B0B0F90E5
:10F490000F900F900F90DF91CF91FF90EF90DF9042
:10F4A000CF90BF90AF909F908F907F906F905F9024
:10F4B0004F900895CF92DF92EF92FF9220915A0BD6
:10F4C0002223F1F020E030E040E05FE30F942ADBFC
:10F4D0006B017C0120E030E0A9010F9455D888230E
:10F4E00079F0A7019601C701B6010F942ADB2BED35
:10F4F0003FE049E450E40F942ADB9B01AC0104C0D7
:10F5000020E030E040E85FE360E070E080E89FE307
:10F510000F945CD8FF90EF90DF90CF9008956091AA
:10F520004402709145028091460290914702C2DFE9
:10F530006093400270934102809342029093430291
:10F540000895CF93DF93EC010F94BB4681E0D3DDA8
:10F5500080E00F94F8B1209799F0C233D10540F0C4
:10F5600062E370E080E090E00F94ADCFE297ECCFE3
:10F57000BE0180E090E00F94ADCFC0E0D0E0E4CFDA
:10F58000DF91CF9108952F923F924F925F926F92A9
:10F590007F928F929F92AF92BF92CF92DF92EF9223
:10F5A000FF921F93CF93DF934B015C01CC24CA944D
:10F5B000DC2C760165E6262E6AE0362E78EE472EA4
:10F5C00073E0572E612C712C1AE08091250B81116C
:10F5D00026C12FEFC216D206E206F20651F0F7FC62
:10F5E0001EC10F947ECF6C197D09683B7B4008F0EB
:10F5F00016C10F947ECF681979098A099B09693E63
:10F6000073408105910508F47FC08091DF1B811153
:10F6100077C0EDE6FAE08491882341F09091C00034
:10F6200095FFFCCF8093C6003196F5CFE091EB0AB1
:10F6300024E0E29FF0011124EE53F54E4081518108
:10F640006281738121E030E088EE99E00E94025FE0
:10F65000E9E6FAE08491882341F09091C00095FF9B
:10F66000FCCF8093C6003196F5CF6091EB0A70E035
:10F670004AE050E088EE99E00E940F5EF10184912B
:10F68000E5E6FAE0882349F09091C00095FFFCCFB1
:10F690008093C60031968491F5CFF7FE03C0E5E470
:10F6A000F9E025C00F947ECF4B015C01C701B60184
:10F6B0006854744F8F4F9F4F681979098A099B09C5
:10F6C000A30192010F942CDDBA01A9012AE030E0D8
:10F6D00088EE99E00E94D75D8091C00085FFFCCF45
:10F6E0000DC09091C00095FFFCCF8093C600819122
:10F6F0008111F7CF8091C00085FFFCCF1093C60029
:10F700000F947ECF4B015C010F94BB4680E0F3DC8D
:10F7100080E00F94F8B1FFEFCF16DF06EF06FF068B
:10F7200009F046C08091E90AE091EB0AF0E0EF01B0
:10F73000CC0FDD1FCC0FDD1FCE53D54EEE0FFF1FBC
:10F74000E653F54E8823D1F080819181BC01882752
:10F7500077FD8095982F0F94F7D820E030E040E8AF
:10F760005FE30F947BD79B01AC01688179818A812B
:10F770009B810F9458DA87FF4DC027CF80819181FC
:10F78000BC01882777FD8095982F0F94F7D820E04B
:10F7900030E040E85FE30F947CD79B01AC016881C7
:10F7A00079818A819B810F9455D818169CF50DCFCD
:10F7B000F7FC0BCFE091EB0AF0E0EF01CC0FDD1F7F
:10F7C000CC0FDD1FCE53D54EEE0FFF1FE653F54E87
:10F7D00080819181BC01882777FD8095982F0F94B7
:10F7E000F7D89B01AC01688179818A819B810F9454
:10F7F0007BD70F94C4D897FF07C0909580957095DC
:10F8000061957F4F8F4F9F4F663071058105910540
:10F810000CF4DBCE0F947ECF6B017C01D6CEDF9152
:10F82000CF911F91FF90EF90DF90CF90BF90AF905E
:10F830009F908F907F906F905F904F903F902F9010
:10F840000895CF93DF931F921F92CDB7DEB7BE010D
:10F850006F5F7F4F88EF9FE00F94386B89819A81AB
:10F860008156904F803A9F4020F11A821982ECE332
:10F87000FAE08491882341F09091C00095FFFCCF7D
:10F880008093C6003196F5CF8091C00085FFFCCFF4
:10F890008AE08093C600BE016F5F7F4F88EF9FE0D4
:10F8A0000F94276B8FEF99E00F94A7BE81E00F9420
:10F8B000BFB40F900F90DF91CF9108952F923F9298
:10F8C0004F925F926F927F928F929F92AF92BF9270
:10F8D000CF92DF92EF92FF920F931F93CF93DF931C
:10F8E000CDB7DEB7CA58D2400FB6F894DEBF0FBE10
:10F8F000CDBFC958DD4F688379838A839B83C757FF
:10F90000D240FE01E75FFD4F88E2DF011D928A953C
:10F91000E9F7E850F24080E991E0DF019C011D9297
:10F9200021503040E1F7C75ADD4F19821882C9557E
:10F93000D240CE01875A9D4F5C014E019FE6891A45
:10F940009EEF990ADE01AF51BE4F3D0190EBC92EEB
:10F950009FE0D92E23E2E22EF12C00E010E0C35903
:10F96000DD4F8882CD56D240CD58DD4F9882C357A7
:10F97000D240B701882777FD8095982F0F94F7D84C
:10F98000D3016D937D938D939D933D01F50161911D
:10F9900071915F01882777FD8095982F0F94F7D894
:10F9A000D4016D937D938D939D934D010F5F1F4FF8
:10F9B0000630110559F0B501C6010F94386BB5E05A
:10F9C000EB0EF11CE2E0CE0ED11CD3CFCF51DE4FB7
:10F9D000288139814A815B81C15ED140C958DD4FA0
:10F9E000688179818A819B81C757D2400F9455D80D
:10F9F00087FD2BC3FE01EF51FE4F7F016E01FFE239
:10FA0000CF1AFEEFDF0A3E012BEB621A2DEF720ACE
:10FA1000C359DD4F0881CD56D240CD58DD4F1881F6
:10FA2000C357D24085E090E0CF58DD4F998388835B
:10FA3000C157D240CF58DD4FA881B981C157D240BC
:10FA40001197CF58DD4FB983A883C157D240F70132
:10FA50002089318942895389648975898689978982
:10FA60000F947BD74B015C01D80150962D913D91AD
:10FA70004D915C91539754966D917D918D919C9190
:10FA800057970F947BD7A50194010F945CD8F6018A
:10FA900092938293729362936F01D301BE92AE925E
:10FAA0009E928E923D0104501109B4E0EB1AF108C8
:10FAB000CF58DD4FE881F981C157D240EF2B09F0D3
:10FAC000B9CF6E01FFECCF1AFDEFDF0A3E0127E44C
:10FAD000621A2EEF720A2E013DE3430E511CCE0135
:10FAE00001967C0101E010E0D6018D909D90AD90D3
:10FAF000BC90139714962D913D914D915C91179761
:10FB0000C501B4010F947CD79B01AC010F947CD745
:10FB1000F70164A775A786A797A70130110541F0E3
:10FB200080A691A6A2A6B3A684829582A682B78259
:10FB30000F5F1F4FD30114962D913D914D915C9114
:10FB4000179718966D917D918D919C911B970F94AD
:10FB50007BD720E030E040EC50E40F942ADBF20148
:10FB60006083718382839383F4E0CF0ED11C2CE2F7
:10FB7000E20EF11C34E0630E711C88E2480E511C49
:10FB80000530110509F0B0CF8E010B5A1F4F6E01E1
:10FB900091E5C90ED11C22242394312C2C0E3D1E3C
:10FBA000A8ED2A0E311CF801B897208131814281DD
:10FBB0005381F80160817181828193810F945CD8B7
:10FBC0004B015C01E12CF12C3601F8E26F1A71084F
:10FBD00026014E0C5F1CF301EE0DFF1D24813581C3
:10FBE00046815781C501B4010F942ADB9B01AC010A
:10FBF000D20114966D917D918D919C9117970F94E0
:10FC00007BD7F2016483758386839783F4E0EF0EDC
:10FC1000F11C24E1E216F104D9F6045D1F4F38E22D
:10FC2000C30ED11C0215130509F0BDCF1E0185EBD3
:10FC3000280E311C6E0191EBC90ED11C3E01A7EEBE
:10FC40006A1AADEF7A0A14E0E12EF12C270100E0E8
:10FC500010E0812C912CA12CB12CF601E00FF11FAA
:10FC6000D301A00FB11F2D913D914D915C91608109
:10FC70007181828193810F942ADB9B01AC01B401D5
:10FC8000C5010F947CD74B015C01BFEF4B1A5B0A97
:10FC90000C5F1F4FE5E04E165104F9F69B01AC01D5
:10FCA000D1016D917D918D919C910F947BD7F6013F
:10FCB00020813181428153810F945CD8D3016D93AF
:10FCC0007D938D939C931397B1E0EB1AF108E8E2D2
:10FCD0002E1A3108FCE2CF1AD10824E0621A71080A
:10FCE000E114F10409F0B2CFCB50DE4F8881998145
:10FCF000AA81BB81C55FD140C957DD4F88839983F5
:10FD0000AA83BB83C758D2408E01075F1D4FDE0117
:10FD1000AF5CBD4FC558DD4FB983A883CB57D240E8
:10FD2000C359DD4F2880CD56D240CD58DD4F3880A5
:10FD3000C357D240FE01EF51FE4FC358DD4FF98348
:10FD4000E883CD57D240C358DD4FA881B981CD5744
:10FD5000D240CD90DD90ED90FD90C358DD4FB9833A
:10FD6000A883CD57D240C958DD4F288139814A81B7
:10FD70005B81C757D240C701B6010F9455D81816FA
:10FD8000B4F0C358DD4FE881F981CD57D2402081CE
:10FD9000318142815381C958DD4F688179818A81DF
:10FDA0009B81C757D2400F9455D81816FCF4CF58F2
:10FDB000DD4F28813981C157D2402430310509F007
:10FDC0001FC1C957DD4F288139814A815B81C758DE
:10FDD000D240C958DD4F688179818A819B81C7579C
:10FDE000D2400F9458DA18160CF00AC1D8011496B4
:10FDF0008D919D910D90BC91A02DC158DD4F8883B0
:10FE00009983AA83BB83CF57D240F80140805180A9
:10FE100062807380C558DD4FA881B981CB57D2402D
:10FE20008D919D910D90BC91A02DC359DD4F88837C
:10FE30009983AA83BB83CD56D240D1018D919D91E8
:10FE40000D90BC91A02DCD57DD4F88839983AA8357
:10FE5000BB83C358D240A7019601C958DD4F6881C2
:10FE600079818A819B81C757D2400F947BD7CD5827
:10FE7000DD4F688379838A839B83C357D24020E018
:10FE800030E040E450E40F948DDB6B017C01A30172
:10FE90009201C158DD4F688179818A819B81CF575A
:10FEA000D2400F947BD74B015C0120E030E040EC66
:10FEB00050E4C359DD4F688179818A819B81CD5699
:10FEC000D2400F942ADB9B01AC01C501B4010F9411
:10FED0005CD8A70196010F942ADB6B017C0120E01E
:10FEE00030E040E05FE3C301B2010F942ADB4B0135
:10FEF0005C01CD58DD4F288139814A815B81C35730
:10FF0000D240CA01B9010F942ADB9B01AC01C501A3
:10FF1000B4010F942ADB9B01AC01C701B6010F9419
:10FF20007CD76B017C01CD57DD4F288139814A8117
:10FF30005B81C358D240F1016481758186819781CC
:10FF40000F947BD7C359DD4F288139814A815B816A
:10FF5000CD56D2400F945CD84B015C01C359DD4FA4
:10FF6000288139814A815B81CD56D240CA01B901CD
:10FF70000F947CD7A30192010F942ADB2B013C0143
:10FF8000C359DD4F288139814A815B81CD56D240EA
:10FF9000C158DD4F688179818A819B81CF57D240DA
:10FFA0000F942ADB9B01AC01C301B2010F947CD7F3
:10FFB00020E030E040EC50E40F945CD89B01AC01B1
:10FFC000C501B4010F947BD7CD58DD4F288139810D
:10FFD0004A815B81C357D2400F942ADB9B01AC015D
:10FFE000C701B6010F947CD7CD57DD4F28813981E9
:10FFF0004A815B81C358D2400F947CD74B015C018E
:020000021000EC
:10000000CF58DD4F28813981C157D2402F5F3F4FF4
:10001000CF58DD4F39832883C157D2400C5F1F4F23
:10002000C558DD4F88819981CB57D2400496C55879
:10003000DD4F99838883CB57D24094E0290E311C41
:100040002530310509F07FCE04C0812C912CA12CE4
:10005000B12CB401C501C657DD4F0FB6F894DEBF11
:100060000FBECDBFDF91CF911F910F91FF90EF9009
:10007000DF90CF90BF90AF909F908F907F906F90C8
:100080005F904F903F902F900895CF92DF92EF9224
:10009000FF926B017C018091B00B8823A1F086EA6E
:1000A0009FE00F9465E4882371F0C701B60106DC78
:1000B00020919B1930919C1940919D1950919E1946
:1000C0000F945CD803C060E070E0CB01FF90EF902C
:1000D000DF90CF9008954F925F926F927F928F92B0
:1000E0009F92AF92BF92CF92DF92EF92FF920F93C7
:1000F0001F93CF93DF93CDB7DEB728970FB6F89451
:10010000DEBF0FBECDBF0F94CF39809156029091C4
:1001100057029093B40B8093B30BE091360BF0E051
:10012000EE0FFF1FE653F54E60817181882777FD42
:100130008095982F0F94F7D86093A40B7093A50B1C
:100140008093A60B9093A70B8091340B9091350B65
:100150009093A30B8093A20B0F947ECF60938A0B96
:1001600070938B0B80938C0B90938D0B80914A0B2B
:1001700090914B0BA0914C0BB0914D0B89839A83BE
:10018000AB83BC838093920B9093930BA093940BBF
:10019000B093950B40904E0B50904F0B6090500BCE
:1001A0007090510B4092960B5092970B6092980B67
:1001B0007092990B8091520B9091530BA091540B1C
:1001C000B091550B8D839E83AF83B88780939A0B34
:1001D00090939B0BA0939C0BB0939D0B6091560B3F
:1001E0007091570B8091580B9091590B60939E0B17
:1001F00070939F0B8093A00B9093A10B20E030E0B5
:1002000040E85FE30F947BD76093560B7093570BD6
:100210008093580B9093590B86E39BE09F938F93A9
:10022000812C912CB8ECAB2EB3E4BB2E16E5C12E7D
:100230001BE0D12EED80FE800F811885A301920175
:1002400069817A818B819C810F94202020E030E0AD
:1002500040EA51E46091520B7091530B8091540B22
:100260009091550B0F947CD72B013C010F900F9070
:1002700020E030E042E553E40F9458DA18164CF0D1
:100280004092520B5092530B6092540B7092550B4C
:100290000CC080E090E0A2E5B3E48093520B909311
:1002A000530BA093540BB093550BE090520BF0906E
:1002B000530B0091540B1091550B20914E0B309124
:1002C0004F0B4091500B5091510B60914A0B709124
:1002D0004B0B80914C0B90914D0BA6E36A2EABE03B
:1002E0007A2E7F926F92812C912CB0E7AB2EB1E4E5
:1002F000BB2EE6E5CE2EEBE0DE2E0F9420201092F2
:10030000CB1A1092CA1A1092CD1A1092CC1A1092CF
:10031000CF1A1092CE1A80E090E0A8E4B2E4809365
:100320004A0B90934B0BA0934C0BB0934D0B80E07A
:1003300090E0AEE3B3E480934E0B90934F0BA09309
:10034000500BB093510BE090520BF090530B009177
:10035000540B1091550B7F926F92812C912CF8E4E5
:10036000AF2EF2E4BF2E9C01AD01C501B4010F9484
:1003700020201092350B1092340B0F900F900F909D
:100380000F9028960FB6F894DEBF0FBECDBFDF9159
:10039000CF911F910F91FF90EF90DF90CF90BF9082
:1003A000AF909F908F907F906F905F904F900D9443
:1003B000CF39E091360B84E0E89FF0011124EE5331
:1003C000F54E4081518162817381ECEFF9E08491B7
:1003D000882341F09091C00095FFFCCF8093C60028
:1003E0003196F5CF22E030E088EE99E00E94025F7E
:1003F000E8EFF9E08491882341F09091C00095FFE7
:10040000FCCF8093C6003196F5CF6091360B70E03B
:100410004AE050E088EE99E00E940F5EE4EFF9E0D8
:100420008491882341F09091C00095FFFCCF809388
:10043000C6003196F5CF4091B01A5091B11A609133
:10044000B21A7091B31A21E030E088EE99E00E9470
:10045000025F8091C00085FFFCCF8AE08093C600D8
:100460000895CF93DF93CDB7DEB72A970FB6F894F0
:10047000DEBF0FBECDBF0F947ECF6F837887898795
:100480009A87179A10923B0B169A10923C0BEFEE3C
:10049000F9E08491882341F09091C00095FFFCCF52
:1004A0008093C6003196F5CF8091C00085FFFCCFC8
:1004B0008AE08093C60083E40F94A4591C01409005
:1004C00074105090751060907610709077100F94A3
:1004D000132F481A590A610871080E94D5E4481A76
:1004E000590A6108710877FE03C0412C512C320172
:1004F0009091B7138091B613981799F0E091B613C5
:1005000027E5E29FF0011124E854FC4E20E030E0A2
:1005100040E752E462A173A184A195A10F942ADB64
:1005200008C060910C0270910D0280910E029091B2
:100530000F020F94C4D87E836D830F94A51E0E9472
:100540007CDD1092BF0B789420E030E040E85FE360
:100550006091560B7091570B8091580B9091590BED
:100560000F947BD769837A838B839C83E090520BB3
:10057000F090530B0091540B1091550B20914E0BA2
:1005800030914F0B4091500B5091510B60914A0BA1
:1005900070914B0B80914C0B90914D0BA6E3BBE0FF
:1005A000BF93AF93812C912CE8ECAE2EE3E4BE2EEA
:1005B000DE0111966D010F94202020E030E040E82C
:1005C0005FE36091560B7091570B8091580B90919F
:1005D000590B0F947BD769837A838B839C832FE895
:1005E00032EC45EF5FE36091520B7091530B8091B9
:1005F000540B9091550B0F947CD76B017C0167E0F5
:1006000074E062197309F4E076956795FA95E1F75D
:1006100080E090E00F94F5D820919B1930919C19BF
:1006200040919D1950919E190F945CD89B01AC018B
:10063000C701B6010F947CD77B018C0120914E0B32
:1006400030914F0B4091500B5091510B60914A0BE0
:1006500070914B0B80914C0B90914D0BA6E3BBE03E
:10066000BF93AF93812C912CA0E2AA2EA2E4BA2EC4
:10067000DE0111966D010F942020B301A20181E9E2
:100680009FE00F9489E40F900F900F900F9005E773
:100690001FE0F12CB3E0EB2E8091CA12882341F1C8
:1006A0008F2D6E2D0F94F8DCB5E18B02F001112433
:1006B00023E09202E00DF11D1124EE0FFF1FEE0F5B
:1006C000FF1FE653FD4E20E030E04AE754E461812D
:1006D0007281838194810F942ADB20E030E040E036
:1006E0005FE30F947CD70F9432D90F94C4D802C023
:1006F00060E070E0C8010F9491E4F3940E5F1F4F27
:1007000089E0F812C9CFB10183E79FE00F9491E42B
:1007100040914A0B50914B0B60914C0B70914D0BDB
:100720008DE99FE00F9489E440914E0B50914F0B5F
:100730006091500B7091510B81EA9FE00F9489E416
:100740004091520B5091530B6091540B7091550B8B
:100750008DE89FE00F9489E4BE016B5F7F4F89E8CD
:100760009FE00F94276BE091360BF0E0EE0FFF1F38
:10077000E653F54E60818CE89FE00F9477E460913A
:10078000C81A8BE89FE00F9477E46091340B88E8F7
:100790009FE00F9477E461E085EA9FE00F9477E4AF
:1007A0000F94CF39EAEEF9E08491882341F09091DB
:1007B000C00095FFFCCF8093C6003196F5CF83E44F
:1007C0000F94A4594AE050E0BC0188EE99E00E94E1
:1007D000615E84E69FE00F9465E461E0680F84E663
:1007E0009FE00F9477E4EFEDF9E08491882341F0E6
:1007F0009091C00095FFFCCF8093C6003196F5CF55
:100800008091C00085FFFCCF8AE08093C6000F94E2
:100810007ECFAB01BC018F819885A985BA85481B25
:10082000590B6A0B7B0B2AE030E088EE99E00E94BE
:100830006D5EF894FFCF6F987798EAE6F0E08081DC
:100840008F7B8083808180688083EF9A08951F92D8
:100850000F920FB60F9211240BB60F920F931F93A6
:100860002F933F934F935F936F937F938F939F93B8
:10087000AF93BF93EF93FF938091340B9091350B1F
:100880008B3491050CF441C080916A0086FF0BC047
:100890000F947ECF6093860B7093870B8093880BA9
:1008A0009093890B2CC00F947ECF0091860B1091F2
:1008B000870B2091880B3091890B601B710B820B89
:1008C000930B2091340B3091350B253631052CF0EC
:1008D00003E010E020E030E004C004E010E020E09D
:1008E00030E0601771078207930748F08091610B31
:1008F0009091620B02969093620B8093610B8091B2
:100900006A0090E4892780936A00FF91EF91BF917C
:10091000AF919F918F917F916F915F914F913F9197
:100920002F911F910F910F900BBE0F900FBE0F9044
:100930001F9018956C987498EAE6F0E080818160C9
:10094000808380818D7F8083EC9A08951F920F921F
:100950000FB60F9211240BB60F922F933F934F9324
:100960005F936F937F938F939F93AF93BF93EF9317
:10097000FF93EC98EAEDF9E08491882341F090919F
:10098000C00095FFFCCF8093C6003196F5CF8091D3
:10099000C00085FFFCCF8AE08093C6008091BF0B2A
:1009A00081115FDDFF91EF91BF91AF919F918F9189
:1009B0007F916F915F914F913F912F910F900BBE5F
:1009C0000F900FBE0F901F901895BF92CF92DF929D
:1009D000EF92FF920F931F93CF93DF93CDB7DEB7C4
:1009E000E1970FB6F894DEBF0FBECDBF88E89FE059
:1009F0000F9465E4B82EBE01605D7F4F89E89FE0EB
:100A00000F94386BE3E8F8E08491882341F09091EB
:100A1000C00095FFFCCF8093C6003196F5CF68A942
:100A200079A94AE050E088EE99E00E94165E8E01B6
:100A3000015E1F4F85E9E82E8FE0F82ED02EC12EE3
:100A4000C7010F9465E4F80181938F01FFEFEF1A5E
:100A5000FF0A8DE9E8168FE0F80691F71FA2ED2D49
:100A6000FC2D8191882339F09091C00095FFFCCF37
:100A70008093C600F6CF6EE778E08D2D9C2D0F9405
:100A800077E0CF92DF9287E798E09F938F938E0174
:100A90000F5F1F4F1F930F930F9439E20F900F902A
:100AA0000F900F900F900F907E0195E0E90EF11CD2
:100AB000F7018081882349F0992787FD90950F944D
:100AC00066E0F70181937F01F3CF60E0C8010E94E7
:100AD000F2DD81E99FE00F946DE4F62EE72ED82E2B
:100AE000C92EECE5F8E08491882341F09091C00094
:100AF00095FFFCCF8093C6003196F5CF2AE030E019
:100B00004F2D5E2D6D2D7C2D88EE99E00E946D5E3F
:100B100061E088E598E00E94F2DD63E578E0C801D5
:100B20000F9482E08DE99FE00F946DE46CA77DA7A0
:100B30008EA79FA7CE018C960F94AD6FBC01C80104
:100B40000F9411E160E578E0C8010F9477E081EA45
:100B50009FE00F946DE46CA77DA78EA79FA7CE01A1
:100B60008C960F94AD6FBC01C8010F9411E169E43C
:100B700078E0C8010F9477E060E0C8010E94F2DDE0
:100B800064E478E0C8010F9482E08DE89FE00F9460
:100B90006DE46CA77DA78EA79FA7CE018C960F94BE
:100BA000AD6FBC01C8010F9411E160E0C8010E9463
:100BB000F2DD61E089E398E00E94F2DD89A98F937C
:100BC00088A98F9382E398E09F938F931F930F934D
:100BD0000F9439E260E0C8010E94F2DD6BE278E038
:100BE000C8010F9482E08B2D90E09DA78CA7CE01C9
:100BF0008C960F948272BC01C8010F9411E160E0E1
:100C0000C8010E94F2DDCF92DF92EF92FF9282E262
:100C100098E09F938F931F930F930F9439E260E0B6
:100C2000C8010E94F2DD61E08EE198E00E94F2DDF1
:100C30000FB6F894DEBF0FBECDBFE1960FB6F894A5
:100C4000DEBF0FBECDBFDF91CF911F910F91FF90FF
:100C5000EF90DF90CF90BF9008954F925F926F9288
:100C60007F92AF92BF92CF92DF92EF92FF920F935B
:100C70001F93CF93DF93CDB7DEB7E0970FB6F8940D
:100C8000DEBF0FBECDBF2B013C0169017A0180910F
:100C9000890A8111E5C0F8940F94F32E80917410A5
:100CA00090917510A0917610B09177108093850A7D
:100CB0009093860AA093870AB093880A0F94132F03
:100CC0004091850A5091860A6091870A7091880A3E
:100CD000481B590B610971094093850A5093860A94
:100CE0006093870A7093880A0E94D5E44091850A30
:100CF0005091860A6091870A7091880A481B590BA7
:100D0000610971094093850A5093860A6093870AA6
:100D10007093880A9091B7138091B613981799F041
:100D2000E091B61387E5E89FF0011124E854FC4EEA
:100D300020E030E040E752E462A173A184A195A1D4
:100D40000F942ADB08C060910C0270910D02809113
:100D50000E0290910F026093710A7093720A809351
:100D6000730A9093740A0F94A51E80E1EAE4FBE0F5
:100D7000A5E7BAE001900D928A95E1F78091360BD4
:100D80008093700A8091070280936F0A0E947CDD35
:100D90001092BF0B81E08093890A789420E030E0C4
:100DA000A901C301B2010F9455D881110AC020E0F6
:100DB00030E0A901C701B6010F9455D8882309F482
:100DC0004FC069E178E0FE0131965F01CF010F94D9
:100DD00082E0F50101900020E9F78F01015011092F
:100DE00020917D0A30917E0A40917F0A5091800ABD
:100DF000C301B2010F947CD723E048E00F94A5DD36
:100E000066E178E0C5010F9477E0F50101900020DC
:100E1000E9F78F010150110923E046E0C701B6014F
:100E20000F94A5DD63E178E0C5010F9477E0F5014B
:100E300001900020E9F78F010150110960916002D3
:100E400070916102809162029091630223E048E018
:100E50000F94A5DD60E0C5010E94F2DD0E9491DFE4
:100E6000E0960FB6F894DEBF0FBECDBFDF91CF91F5
:100E70001F910F91FF90EF90DF90CF90BF90AF90B8
:100E80007F906F905F904F90089520E030E0A9012F
:100E900060E070E080E291E4E0CE8F929F92AF92AA
:100EA000BF92CF92DF92EF92FF920F931F93CF9357
:100EB000DF9300D01F92CDB7DEB79B01AC018091CC
:100EC000890A882309F497C08091700A8093360BB1
:100ED0008091710A9091720AA091730AB091740A7C
:100EE00080930C0290930D02A0930E02B0930F0218
:100EF0006091810A7091820A8091830A9091840A9C
:100F00000F947BD769837A838B839C83CE01019670
:100F10000F94792E20E030E040E551E460916002CA
:100F20007091610280916202909163020F945CD88B
:100F30004B015C01E0907D0AF0907E0A00917F0AEF
:100F40001091800A2091790A30917A0A40917B0AA7
:100F500050917C0A6091750A7091760A8091770AA7
:100F60009091780AE6E3FBE0FF93EF93E1E8CE2E61
:100F7000EAE0DE2E0F9420200F94CF3980E1E5E7E0
:100F8000FAE0AAE4BBE001900D928A95E1F780E1D6
:100F9000EAE4FBE0A5E1BBE001900D928A95E1F760
:100FA0004091850A5091860A6091870A7091880A5B
:100FB00040935B0E50935C0E60935D0E70935E0EDB
:100FC00086EA9DE00E9466C58091850A9091860A16
:100FD000A091870AB091880A80937410909375103D
:100FE000A0937610B093771081E08093BF0B10929E
:100FF000890A0F900F900F900F900F900F90DF9134
:10100000CF911F910F91FF90EF90DF90CF90BF9005
:10101000AF909F908F90089560E070E0CB013DCF3E
:10102000FBDF81E08093B1020895EEEFF7E0849159
:10103000882341F09091C00095FFFCCF8093C600BB
:101040003196F5CF40914A0B50914B0B60914C0B70
:1010500070914D0B23E030E088EE99E00E94025F32
:10106000EBEFF7E08491882341F09091C00095FF69
:10107000FCCF8093C6003196F5CF40914E0B509136
:101080004F0B6091500B7091510B23E030E088EED4
:1010900099E00E94025FE8EFF7E08491882341F035
:1010A0009091C00095FFFCCF8093C6003196F5CF9C
:1010B0004091520B5091530B6091540B7091550B12
:1010C00023E030E088EE99E00E94025FE6EFF7E06F
:1010D0008491882341F09091C00095FFFCCF8093CC
:1010E000C6003196F5CF8091C00085FFFCCF8AE025
:1010F0008093C6000895EEEDF7E08491882341F0D7
:101100009091C00095FFFCCF8093C6003196F5CF3B
:101110000F943E3AAB01BC0123E030E088EE99E049
:101120000E94025FEBEDF7E08491882341F09091FB
:10113000C00095FFFCCF8093C6003196F5CF81E0CB
:101140000F943E3AAB01BC0123E030E088EE99E019
:101150000E94025FE8EDF7E08491882341F09091CE
:10116000C00095FFFCCF8093C6003196F5CF82E09A
:101170000F943E3AAB01BC0123E030E088EE99E0E9
:101180000E94025FE6EDF7E08491882341F09091A0
:10119000C00095FFFCCF8093C6003196F5CF8091BB
:1011A000C00085FFFCCF8AE08093C6000895EF92CF
:1011B000FF920F931F93CF93DF93E2ECF7E08491BC
:1011C000882341F09091C00095FFFCCF8093C6002A
:1011D0003196F5CF0AEC12E1F0ECEF2EF7E0FF2E9E
:1011E000C0E0D0E0F801EC0FFD1F41815281638126
:1011F000748123E030E088EE99E00E94025FF701FD
:101200008491E0ECF7E0882349F09091C00095FFCD
:10121000FCCF8093C60031968491F5CF2496CC31D3
:10122000D10501F7045E1F4FF3E10E381F07C1F629
:10123000EFEBF7E08491882341F09091C00095FF97
:10124000FCCF8093C6003196F5CF8091C00085FF1A
:10125000FCCF8AE08093C600DF91CF911F910F9160
:10126000FF90EF9008952F923F924F925F926F926E
:101270007F928F929F92AF92BF92CF92DF92EF9226
:10128000FF920F931F93CF93DF93CDB7DEB7C35574
:10129000D1090FB6F894DEBF0FBECDBF82E090E05B
:1012A000909316028093150285EE93E00E94EA5F08
:1012B0008823B1F080918C1090918D106AE270E0DB
:1012C00005960F941CE1009711F0DC011C928091AF
:1012D0008C1090918D1005960F94046C0C9429B588
:1012E00086ED93E00E94EA5F882321F00E944A6421
:1012F0000C9429B58AEE93E00E94EA5F882319F0E6
:101300008FDE0C9429B588EF93E00E94EA5F882372
:1013100021F00E9486640C9429B585E094E00E9437
:10132000EA5F882309F4C4C18BE094E00E94EA5F7D
:10133000882391F08091DF1B882311F40C9429B548
:101340000F947ECF6093B90B7093BA0B8093BB0B55
:101350009093BC0B0C9429B580E194E00E94EA5F65
:10136000882361F060917C0B70917D0B4AE050E026
:1013700088EE99E00E94615E0C9429B584E194E0C6
:101380000E94EA5F882309F446C0E8E1F4E0819115
:10139000882339F09091C00095FFFCCF8093C60060
:1013A000F6CF80915B0B90915C0B2CE3289FB001F2
:1013B000299F700D11244AE050E088EE99E00E94C8
:1013C0000F5E6CE174E088EE99E00E94025EE1E25B
:1013D000F4E08191882339F09091C00095FFFCCF13
:1013E0008093C600F6CF80915D0B90915E0B2CE34D
:1013F000289FB001299F700D11244AE050E088EE2B
:1014000099E00E940F5E6CE174E088EE99E00E9422
:10141000025E0C9429B587E294E00E94EA5F88237B
:10142000C1F08091DF1B882361F06091DD1B70911A
:10143000DE1B4AE050E088EE99E00E94165E0C94B4
:1014400029B56AE274E088EE99E00E94025E0C948D
:1014500029B58CE394E00E94EA5F882379F16091DA
:101460008C1070918D106D5F7F4F21E041E08DEB0E
:101470009BE00E94B4D78091AE0D9091AF0DA091EA
:10148000B00DB091B10D80935B0E90935C0EA09364
:101490005D0EB0935E0E86EA9DE00E949DC4209191
:1014A000C00025FFFCCF8093C6000A9721F760E0BB
:1014B0008DEB9BE00E9444D70C9429B58FE394E018
:1014C0000E94EA5F882399F00E94716D81E0809309
:1014D0007E0B60918C1070918D106C5F7F4F21E0BE
:1014E00040E08DEB9BE00E94B4D70C9429B583E4D7
:1014F00094E00E94EA5F882309F445C08091DF1BD5
:10150000882309F49ECF10926D0AE6E4F4E08191FD
:10151000882339F09091C00095FFFCCF8093C600DE
:10152000F6CF00E010E0FF24F3948091690A9091D7
:101530006A0A20916B0A30916C0A821B930B8F7799
:101540009927892B89F088EE99E00E941C5DF09222
:101550006D0A9091C00095FFFCCF8093C6000F5F8D
:101560001F4F10926D0AE1CF03311105F4F281E0B3
:1015700080936D0A8091C00085FFFCCF8AE0809344
:10158000C6000C9429B589E494E00E94EA5F8823A0
:10159000A9F0EDE4F4E08191882339F09091C00046
:1015A00095FFFCCF8093C600F6CF8091C00085FFE9
:1015B000FCCF8AE08093C6000C9429B588E594E0BE
:1015C0000E94EA5F8823A9F0ECE5F4E0819188238A
:1015D00039F09091C00095FFFCCF8093C600F6CF04
:1015E0008091C00085FFFCCF8AE08093C6000C94F8
:1015F00029B58AE794E00E94EA5F882321F00F94DE
:10160000A26B0C9429B58FE794E00E94EA5F8823CF
:1016100041F060E070E088EF9FE00F94276B0C943E
:1016200029B582E894E00E94EA5F882359F062E8D5
:1016300074E088EE99E00E94025E40E052EC61E0C6
:1016400070E010C08DE894E00E94EA5F882381F08A
:101650006DE874E088EE99E00E94025E40E054E993
:1016600061E170E088EE99E00E94A15C0C9493B671
:1016700089E994E00E94EA5F882361F00F947ECFAD
:101680006093AC0B7093AD0B8093AE0B9093AF0B4C
:101690000C9429B58EE994E00E94EA5F882311F446
:1016A0000C9429B561E080E00E9491640C9429B506
:1016B0008EE50E94BC5F81110C9429B587E40E94DD
:1016C000BC5F882311F40C94269B0E9429600F9420
:1016D000C4D86C34710509F43AC47CF564307105E2
:1016E00009F409C154F46230710509F4ECC00CF03E
:1016F000F6C077FF78C00C9429B56C31710509F4F8
:1017000056C17CF46A30710509F44BC16B30710528
:1017100011F00C9429B560E080E00E946A750C9489
:1017200029B56E31710509F452C36B34710511F09E
:101730000C9429B508E210E000C46735710511F476
:101740000C94A69A14F56035710511F40C947F94ED
:101750006CF46F34710511F00C9429B50FEF10E0A3
:10176000AAE7CA2EACE0DA2E0C946A9461357105B2
:1017700011F40C94ED996635710511F00C9429B5AE
:1017800086EE0E9401640C9429B56C35710511F444
:101790000C94AF9A7CF46A35710511F40C94AB9AF1
:1017A0006B35710511F00C9429B581E08093000B25
:1017B0000C9429B56236710511F40C94119B6336B3
:1017C000710511F00C9429B51092DF1B0F94A76BD3
:1017D0006091DF1B84EC9FE00F9477E482E00F942C
:1017E000F8B10C9429B58091EA0A81110C9429B5BD
:1017F0000E949F716091780B7091790B80917A0BA8
:1018000090917B0B0F94F5D86B017C014090560BA7
:101810005090570B6090580B7090590B8090210B93
:101820009090220BA090230BB090240BA501940163
:10183000C301B2010F947BD720E030E048EC52E4C2
:101840000F942ADB9B01AC01C701B6010F9458DA53
:101850001816E4F4A3019201C501B4010F947BD7DB
:1018600020E030E048EC52E40F942ADB9B01AC010D
:10187000C701B6010F947CD70F94C9D86093780B39
:101880007093790B80937A0B90937B0B8091330B41
:101890008823A9F088E50E94BC5F811110C089E50A
:1018A0000E94BC5F81110BC08AE50E94BC5F811160
:1018B00006C085E40E94BC5F81110C9432B50E9481
:1018C00067740C9429B58091EA0A81110C9429B5AA
:1018D0000E94227281E00E9445770C9429B5809184
:1018E000EA0A81110C9429B50E94227280E00E94BC
:1018F00045770C9429B580E50E94BC5F882339F0B8
:101900000E9429600F94C9D86B017C0103C0C12CCF
:10191000D12C760183E50E94BC5F882361F00E9490
:10192000296020E030E04AE754E40F942ADB0F946A
:10193000C9D86B017C01C114D104E104F10459F050
:10194000E0917F0BF0E0EE0FFF1FED54F34885911F
:1019500094910F94116C0F94CF390F947ECF4B015B
:101960005C018C0C9D1CAE1CBF1C0F947ECF609341
:10197000FC0A7093FD0A8093FE0A9093FF0A0F946D
:101980007ECF681579058A059B0510F00C9429B562
:101990000F94BB4680E00E947B7880E00F94F8B102
:1019A000EECF60E081E00E946A750C9429B50F9437
:1019B000CF39E8EAFDE08491882341F09091C0009E
:1019C00095FFFCCF8093C6003196F5CF2EDBEAE978
:1019D000FDE08491882341F09091C00095FFFCCFF9
:1019E0008093C6003196F5CF86DB81E08093B10B02
:1019F00088E50E94BC5F182F89E50E94BC5F082F14
:101A00008AE50E94BC5F782E101308C0181711F0E9
:101A1000012F04C07724739401E011E00E9422F6A4
:101A20006090CA121092CA1282E00F943E3A6093FC
:101A3000520B7093530B8093540B9093550B711072
:101A40000F94F11340910C0250910D0260910E021F
:101A500070910F024093010B5093020B6093030BA4
:101A60007093040B80915602909157029093B40B9F
:101A70008093B30B84E690E09093570280935602D4
:101A80000F947ECF6093FC0A7093FD0A8093FE0A48
:101A90009093FF0A81E00F94543080E1EAE4FBE088
:101AA000A5E1BBE001900D928A95E1F710920C023E
:101AB00010920D0210920E0210920F02112321F0CB
:101AC00080E090E00E941169002321F081E090E025
:101AD0000E94116988E50E94BC5F882341F00E9442
:101AE000DF5F672B682B692B11F00C9461B589E5DA
:101AF0000E94BC5F882341F00E94DF5F672B682B48
:101B0000692B11F00C9477B5772009F4F1C080911E
:101B10003B0B882321F080913C0B811108C080E0B1
:101B200090E00E94116981E090E00E9411690E949A
:101B300077F6EFE8F0E885919591A591B4918983C6
:101B40009A83AB83BC83EBE8F0E885919591A591EE
:101B5000B4918F8F98A3A9A3BAA329E13BE045E1F3
:101B60005BE0BE016F5F7F4FCE014F960E943062F7
:101B70000E94E9F520E030E040E850EC6091190B5C
:101B800070911A0B80911B0B90911C0B0F9455D8E0
:101B900087FF0CC080E090E0A0E8B0EC8093190BC8
:101BA00090931A0BA0931B0BB0931C0B80E090E05A
:101BB000A0EAB0E480931D0B90931E0BA0931F0B23
:101BC000B093200B20E030E040E251E460916002ED
:101BD0007091610280916202909163020F945CD8CF
:101BE00060930C0270930D0280930E0290930F028B
:101BF0001092520B1092530B1092540B1092550BE3
:101C000080E00F945430E090520BF090530B009111
